:020000040000FA
:100000000212FC022003FFFFFFFFFF02200BFFFF95
:10001000FFFFFF020E5DFFFFFFFFFF02201BFFFF40
:10002000FFFFFF022023FFFFFFFFFF02202BFFFF48
:10003000FFFFFF022033FFFFFFFFFF020EA0FFFFC5
:10004000FFFFFF022043FFFFFFFFFF02204BFFFFE8
:10005000FFFFFF022053FFFFFFFFFF02205BFFFFB8
:10006000FFFFFF022063FFFFFFFFFF02206BFFFF88
:10007000FFFFFF022073FFFFFFFFFF02207BFFFF58
:10008000FFFFFF022083FFFFFFFFFF02208BFFFF28
:10009000FFFF70DFFFFF040000000002000000C847
:1000A0000300030369A5020269A501000000000026
:1000B00004003273000074F8121043900393E06060
:1000C0001590030274FEF0900304744DF0A37405C0
:1000D000F07A011206747F0102116074F712104366
:1000E00074FF1212687E00801F851882851983E0D4
:1000F00064FE70069003877401F085188285198369
:10010000E0F8900384E068F07C017D00AA18AB1948
:10011000120E188B09EA450970030201E98518825D
:10012000851983E064EF70027E07E0C0E0900387EA
:10013000E0F8900385E0FAE82AF8E434001206C7F4
:10014000D0E0F0900387E060A014600E14602A14E1
:10015000603A14605014606680A0900384E4F085D7
:100160001882851983E0900386F0C39480900387FA
:100170004003E4808474028080851882851983E0BE
:10018000900382F090038774030200F9851882853A
:100190001983E0900383F0900386E0601990038751
:1001A00074040200F9900385E004F0F8900386E0FF
:1001B0006860030200FA90038774050200F9900357
:1001C00085E4F0900387F0900384E0F88518828539
:1001D0001983E06860030200FA900382E0644D60D6
:1001E000030200FA12031E8002EEF97401121234A7
:1001F0007F0202116074F712104374FB121268EA56
:10020000FEEBFF75080475090078081212CC740221
:100210001212E57A907B007904120EC17402121258
:1002200034120666121336E0687003A3E069701298
:10023000851882851983E0F47003A3E0F46003025B
:1002400002FE74041212DD1206D38A088B09A80874
:10025000A9097402121336E8F0A3E9F0740412132A
:1002600036E0600879011200B6020317851882850E
:100270001983E0687003A3E0697076851882851998
:1002800083E0F47003A3E0F470197402121336745F
:1002900010F0A37420F08518828519837410F0A3E0
:1002A0007420F075080175090078081212CC7402E8
:1002B0001212E57A247B08120F467402121234756A
:1002C000080478081212CC74021212E57A907B00AE
:1002D0007904120EC1740212123412066612133619
:1002E000E0687003A3E069700479028006790480F5
:1002F0000279031200B68E828F83741E80058E826F
:100300008F83E4F0120666121336E0687003A3E0F0
:1003100069700479018002790074050201ED74EDC1
:1003200012104374F8121268900307E0FA90030663
:10033000E0FB8B08EAF8E4C8F9EB28FEE93408FF93
:10034000751001880C750D068F0974027808121259
:1003500093C39508F8E49509F9740228F50E74031F
:1003600039F50F8E088F09740978081212EDE50827
:10037000F511EE2410F508E43FF509EEF50AEF5407
:1003800001F50B900383E0146054147003020453CE
:100390001470030204CE14601024FE700302058959
:1003A000147003020639020649750D03794E120CCA
:1003B0005890030712065C7402F0A3744012065AA8
:1003C000740812065AF0A3F0751012AA10A90C12A4
:1003D0000674A90D74081212347F0C021160750D99
:1003E00004794E120C58EE450B7005A911120FAC92
:1003F000C3EE9425EF9408503CC3E5089424E50926
:1004000094084031E50E2496F8E50F3420F98882EF
:100410008983E0701BA3AA82AB83E07013900388EA
:100420007401F08882898374A5F08A828B838004AA
:10043000900388E4F075081075090078081212CC52
:100440007C087D03EEFAEFFB120F467402121234A1
:100450000203CB750D05E511C394794006750C01B7
:100460000203CB75124075130078121212CC7C096E
:100470007D037402780A121293AA0AAB0BA9111217
:100480000EC17402121234900307E0A3F090030629
:10049000E0A3F0751043C3EE9425EF9408400302E7
:1004A00003CBC3E5089424E509940850030203CB69
:1004B000900388E070030203CBE50E2497F8E50F64
:1004C0003420F988828983E4F0A3F00203CB750815
:1004D0000475090078081212CC74021212E57A90A1
:1004E0007B007904120EC1740212123474021213CA
:1004F00036E0F8A3E0F9851882851983E068700377
:10050000A3E069851882851983700BE0F47003A35A
:10051000E0F470578009E0F47003A3E0F4700D85F7
:1005200018828519837410F0A37420F012066612E5
:100530001336E8F0A3E9F075080178081212CC74BC
:10054000021212E57A247B08120F4674021212344A
:1005500075080478081212CC74021212E57A907BA6
:10056000007904120EC174021212341206661213BC
:1005700036E0687003A3E0697006750D010203CBD5
:10058000750D02750C070203CB900391E0600764C0
:100590000260030203CBEAFF7A017900120674E0DD
:1005A000600302062D8003120D19120D23E970F766
:1005B000740412133612064E74041213367808129D
:1005C000131A85080C85090D850A0E850B0F9005F9
:1005D000A2780C1212B97404121336780C12130B91
:1005E000E5084509450A450B70CE8EC2E5C554E0C5
:1005F0004FF5C5740412133612064E7404121336E6
:10060000780812131A85080C85090D850A0E850BCA
:100610000F9005A2780C1212B97404121336780CDC
:1006200012130BE5084509450A450B70CE7A01798E
:100630000012067479080203D4EB900393F0700360
:100640000203CB750D090203CB79060203D4E4F053
:10065000A37426F0A3E4F0A3F022F0A3E4F0A3F047
:10066000A3F0A3F0A322851882851983E0F8A3E004
:10067000F974022274F6121043EAFE900305E0D2E8
:10068000E7F0E9A3F0EE900303F08E0A74042AFE6B
:100690007A028004E0620A0AEAF83395E01206C79B
:1006A0008E08C3E89508E99400A2D265D03340E4EF
:1006B000E50AF0740128FC3395E0FD7A027B031211
:1006C0000E487F03021160F9740228F58274033921
:1006D000F5832274E91210437582007583FE1211AE
:1006E000FB8A168B177514007515008A828B83E4BC
:1006F000F0900391E07006D2AAD2AF800464027039
:100700000579001200B6750C00750D20750E007588
:100710000F00900391E0600464027015120D19122D
:1007200000DBE9F87409686003020803790012002D
:10073000B675080075090278081212CC74021212FC
:10074000E5850C08850D09AA08E5095407FB850E07
:100750000A850F0B740B780812124FA908120EC1EC
:1007600074021212347E007F009005AAC0828E109F
:10077000EFF5113395E0F512F513850C08850D0999
:10078000850E0A850F0B780879101212A69005A61F
:1007900078081212B9758305D08278081211DC50DE
:1007A0001D851882851983E5822EF582E5833FF544
:1007B00083E0F9AA14AB151208328A148B150EEED9
:1007C00070010FC3EF940240A09005AE780C121296
:1007D000B99005B2780C1211DC40030207127900BF
:1007E000AA14AB1512083279001208328B15900347
:1007F00091E07004C2AFC2AAEA451570277AA57BC2
:10080000A58021E8700302073174066870030207AF
:100810003174076870030207318516828517837467
:1008200001F080BA7582007583021211FB7F1002FD
:100830001160C008C0097C088A088B09740F780809
:100840001212EDEA25E0FAEB33FBE9A2E75004745B
:10085000014AFAE508A2E0500874216AFA74106BA4
:10086000FBE9C333F91CEC70CFD009D0082274F730
:1008700012104378007900802374942508F582E4EF
:100880003403F583E08A828B83F09004141209F319
:100890004005900414E4F008E87001099004141273
:1008A000095D6007C3E89CE99D40CEE8FAE9FB7F5B
:1008B0000202116074F5121043900498E0FEA3E068
:1008C000FF8F08EEC39508F895E0F9EFC39EE85056
:1008D0000B120ADA701178007900801B247F500116
:1008E00009C39CE99D50EF7A007B008041E004F051
:1008F000D2E908E8700109C3E89CE99D502C8A827E
:100900008B83E0C0E0900499E0FE74182EF582E439
:100910003404F583D0E0120ACA90049AE4F09004FB
:1009200099E0C3947F40C6E480C5E8FAE9FB7F0400
:1009300002116074F7121043C2E990049812095D25
:10094000601874182508F582E43404F583E0F5C1D5
:10095000900498120AF14002E4F00208AFE0F508B2
:10096000A3E065082274F71210437800790090051F
:100970001DE07063A3E0705F75F900C28FC284A2AE
:100980008340FCA28F4004A28350F8E5F9C28FA2F5
:10099000835004D2848040C0E0E0FE749D2EF58236
:1009A000E43404F583D0E0F090051E120AF140D340
:1009B000E4F080CF749D2508F582E43404F583E0EB
:1009C0008A828B83F090051D1209F3400590051D66
:1009D000E4F008E870010990051D12095D6007C385
:1009E000E89CE99D40CEE8497006E4F090051DF0D2
:1009F0000208ABE004120ACEC394802274F81210ED
:100A0000439005A0E0FF8F82A88290059FE0FEEF53
:100A1000C39EE0500DC398F895E0F9120AD97018FA
:100A20008012C398F895E0F9E8247F500109C39C2F
:100A3000E99D4004EC4D70077A007B00020AC58AEC
:100A4000828B83E0F5F9A3AA82AB837801790080D9
:100A500008E004F008E8700109C3E89CE99D50270C
:100A60008A828B83E0C0E09005A0E0FE741F2EF523
:100A700082E43405F583D0E0120ACA9005A0E0C3F1
:100A8000947F40CDE480CCC28FA28340FCC284A27C
:100A90008F4004A28350F890059F120AE4E0F5F914
:100AA000C28F90059FE0FAA3E06A90059F7005123F
:100AB0000AE48005120AF14002E4F0A28350D0D289
:100AC00084E8FAE9FB7F01021160120ACE22F08A63
:100AD000828B83A3AA82AB8322E824FF18E934FF28
:100AE000F9E84922E0FA741F2AF582E43405F58317
:100AF00022E004F0C394802274FB1212687E0090FE
:100B000005CA780812131A9005CA7401F0A3F0A35D
:100B10007469F0A374A5F09005B6780812127E707F
:100B2000030E80159005BA780812127E6008E59DC4
:100B3000541864107003022000120C7EEEA2E050E4
:100B400003020BFBAA18AB191201F5E97003020BA3
:100B5000FB851882851983E0C3943C500CE0F8743F
:100B60003CC398FA95E0FB80047A007B00120D3CB0
:100B7000E97003020BFB900391E06401700C75F8BF
:100B800000C2AB539AF7D2EA805E79071200B680B2
:100B900003120D19120D23E970F77401121336E4D4
:100BA000F0A37426F0A3E4F0A3F0740112133678D6
:100BB0000812131A85080C85090D850A0E850B0F7E
:100BC0009005A2780C1212B97401121336780C1227
:100BD000130BE5084509450A450B70CE758600C222
:100BE000AAC28B539AFBC2E990000174CDF0022097
:100BF00000C2AF75C9AB75C95B80FE750800750989
:100C000000750A00750B00900391E0701BD2AAD208
:100C1000AF79051200B6E07003120D191200DBE97E
:100C2000F8740968700980E9794E120C5880ED74E7
:100C3000016870E2E07017120D199005BE78081275
:100C400012B99005C278081211DC50EBC2AAC2AFEB
:100C500075C9AB75C95B80FEC082C08378109005F2
:100C6000A1E0C399501575B60FE5B4A2E750FAE5B7
:100C7000BBC39940F118E870EDE9F0020D37C0826E
:100C8000C08353BEFBE59DA2E650FA0078F87901D7
:100C900000120AD970FA75C6807480659E70FA4396
:100CA000BE049062707408F0794A120C58900001EA
:100CB00074F5F07403F5D575D489A2A0E4339003DC
:100CC00091F0A2E05029D28453F3F753F3EF53FD90
:100CD000F743FD10538FF753F7DF43FC2043F10236
:100CE00053F5DF75F82043F4F0D2FED2AB802853E1
:100CF000FF3F85FFFF53F1FE43F30C53F2F375867C
:100D00008075C48090049BE4F0A3F075C2D875C5CB
:100D10000B75C402438640801E8003120933A2E98A
:100D200040F922C082C083900498E0F8A3E0686094
:100D300004790180027900D083D0822274F11210EC
:100D40004374FF1212687E00900391E06401706B9F
:100D5000C2849003927401F07508388E098E0A8E51
:100D60000B7C017D00AA18AB19120E188B0DEA45F9
:100D70000D6018851882851983E06410602CE0648A
:100D8000EF70088E088E098E0A8E0B85080C850977
:100D90000D850A0E850B0F9005A278081212B9E591
:100DA0000C450D450E450F70330E900391E0640124
:100DB0007056D284900392E4F08051D2AAD2AF8AC6
:100DC000088B09E4F50AF50B9005C6780C12131A86
:100DD0007808790C120FC379061200B6900391E0DF
:100DE0006003020D61120D191200DBE9F874096845
:100DF000700779061200B680927407686085E86013
:100E00008A74066870A48083C2AFC2AAEEF9740126
:100E10001212347F08021160C082C083900391E0F7
:100E2000700512086E801E900392E06015A28F502C
:100E30000BE5F98A828B83F07A0180027A007B00CD
:100E40008003120965020D37C082C083900391E0D0
:100E500070051208B480031209FC020D37C0E0745B
:100E6000F21210A9900001E064CD700512201380E9
:100E70002AE064F57024E5C1C28BC0E0900415E05F
:100E8000F8749428F582E43403F583D0E0F09004FC
:100E900015120AF14005E4F08001007F01021108FB
:100EA000C0E074F21210A9900001E064CD70051248
:100EB000203B800BE064F57005120933800100804F
:100EC000DA74F51210438908740F5508F50A750B8A
:100ED00000740B780A121293EA2400F8EB3480F9BC
:100EE000E82400E9350BF9E5C7F509A2AFE433F5CD
:100EF0000AC2AFE508C4540FFAE5C754F84AF5C76B
:100F0000740B121336E0FAA3E0FB801C88828983FD
:100F1000E08C828D83F088828983A3A882A9838C48
:100F2000828D83A3AC82AD83EAFEEBFFEE24FF1A31
:100F3000EF34FFFBEE4F70D48509C7E50AA2E092BB
:100F4000AF7F0402116074F7121043ED900389F033
:100F5000ECA3F0A37462F0A37473F0A3E0541FF049
:100F60007409121336E0F508A3E0F509E5083333F8
:100F700054FC90038EF0740678081212EDE5089088
:100F8000038DF090038F7412F0A37442F075D1FEBC
:100F900075D601EA906271F0EBA3F0906270E0D236
:100FA000E1F0E0A2E740FB7F02021160C082C08353
:100FB000E9C333906272F0906270E0D2E0F0D083C7
:100FC000D08222080808EAC0E0EBC0E086F0E7A47F
:100FD000FA180986F0E7A42AFA180986F0E7A42A85
:100FE000FA180986F0E7A42AFA1986F0E7A4FBE5C7
:100FF000F02AFA190886F0E7A42BFBE5F03AFA1973
:101000000886F0E7A42BFBE5F03AFA18180986F0F9
:10101000E7A4C5F02BFBE43AFA1908E7C5F0C6A42B
:1010200026F6E5F03BFBE43AFA1886F0E7A4F6E58D
:10103000F00826F6E43B08F6E43A08F6D0E0FBD0E8
:10104000E0FA222518C582C0E0E51934FFC583C047
:10105000E0E518C3958224F910AF088583198582CD
:10106000188008858319858218D2AFCEF0A3E520B9
:10107000F0A37808E608F0A3DEFAEFF0A3E58124F8
:10108000FBF8E608F0A3E608F0A30808E608F0A3DA
:10109000E608F0A315811581D0E0FED0E0F81581B7
:1010A0001581E8C0E0EEC0E022C0D02518C582C09E
:1010B000E0E51934FFC583C0E0E518C3958224F349
:1010C00010AF088583198582188008858319858269
:1010D00018D2AFC8F0A3E9F0A3EAF0A3EBF0A3792C
:1010E00008E709F0A3D8FAECF0A3EDF0A3EEF0A323
:1010F000EFF0A3D0E0F0A3D0E0F0A3D0E0F0A3E5C0
:1011000020F0A3E5F0F0A322851983851882E0C0C2
:10111000E0A3E0F9A3E0FAA3E0FBA37808E0F60877
:10112000A3DFFAE0FCA3E0FDA3E0FEA3E0FFA3E061
:10113000C0E0A3E0C0E0A3E0F5D0A3E0F520A3E089
:10114000A3F5F010AF088583198582188008858380
:1011500019858218D2AFD082D083D0E0F8D0E032A7
:10116000851983851882E0A3FEE0A3F5207808E0C6
:10117000A3F608DFFAE0A3FFE0A3C0E0E0A3C0E02D
:10118000E0A3C0E0E0A3C0E010AF0885821885832B
:10119000198008858218858319D2AFD083D0822226
:1011A000E490030278A179038002F0A3D8FCD9FA75
:1011B0007AA27B0590008E782979018015E493A3AB
:1011C000AD82AE838A828B83F0A3AA82AB838D82A9
:1011D0008E83D8E9D9E7120AF8121340C008C3E099
:1011E00096F50808A3E096420808A3E0964208088E
:1011F000A3E09645087001D3D00822C5822518C502
:1012000082C583351910AF07F5198582188007F557
:1012100019858218D2AFC583222518F58210AF0830
:10122000F518400C15198008F51840021519D2AFB1
:101230008519832200C0D0251810AF08F518500C6E
:1012400005198008F51850020519D2AFD0D02260D8
:1012500016080808C6C313C618C613C618C613C690
:1012600018C613C6D5E0EA22251810AF08F51840B5
:101270000C15198008F51840021519D2AF22E06646
:10128000701008A3E066700A08A3E066700408A363
:10129000E06622700422600D18C6C333C608C63348
:1012A000C6D5E0F41822E627F60809E637F608095D
:1012B000E637F60809E637F622E026F608A3E03618
:1012C000F608A3E036F608A3E036F62274028000A2
:1012D000C0E0F404121219D0E0121329222518FAE2
:1012E000E43519FB222518FCE43519FD22600C08B1
:1012F000C6C313C618C613C6D5E0F42275D0007550
:10130000813F7518027519030211A0E6F008A3E6E3
:10131000F008A3E6F008A3E6F022E0F608A3E0F662
:1013200008A3E0F608A3E0F622CAC0E0E6F0A308AE
:10133000DAFAD0E0FA222518F582E43519F583228D
:1013400000000080FBFFFFFFFFFFFFFFFFFFFFFF2D
:10135000FFFFFFFFFFFFFFFFFFFFFFFFFFFFFFFF9D
:10136000FFFFFFFFFFFFFFFFFFFFFFFFFFFFFFFF8D
:10137000FFFFFFFFFFFFFFFFFFFFFFFFFFFFFFFF7D
:10138000FFFFFFFFFFFFFFFFFFFFFFFFFFFFFFFF6D
:0A1FF600CA05094338860000000008
:020000040003F7
:01FFF000F020
:020000040000FA
:10200000022C420221EBFFFFFFFFFFFFFFFFFFFF5C
:10201000FFFFFFFFFFFFFFFFFFFFFFFFFFFFFFFFD0
:10202000FFFFFFFFFFFFFFFFFFFFFF02291CFFFF76
:10203000FFFFFFFFFFFFFFFFFFFFFFFFFFFFFFFFB0
:10204000FFFFFF022749FFFFFFFFFFFFFFFFFFFF2B
:10205000FFFFFF022127FFFFFFFFFFFFFFFFFFFF43
:10206000FFFFFFFFFFFFFFFFFFFFFF0228F4FFFF5F
:10207000FFFFFFFFFFFFFFFFFFFFFFFFFFFFFFFF70
:10208000FFFFFF02218701FFFFFFFFFFFFFFFFFFB1
:102090001020102001FF01010503010F10FEFFC0F9
:1020A0004D00000000584D00000000FF000000FF40
:1020B00000010000333A000000008539713BCD3942
:1020C000E73A0000BB3900000000000000000000FB
:1020D0000000000000000000000000000000FF0100
:1020E0000100AA07000000E803FFFF250803E8033A
:1020F00064006400B8010202000800000502070441
:1021000001051E02051E020A0A0103B80B02803EE9
:102110000102FEFFE8030A050001FFFF0A01E09645
:102120005118000206FFFFC0E074F2122568A2AF4A
:10213000E433FED2AFE5A7FFE5A1F5085F541060D8
:102140000612451375A1EFE5085F540860081245B3
:102150001975A1F78024E508A2E092F0EFA2E082D1
:10216000F05017906198E0F8900DE3E0C398A2D288
:1021700065D0335002E8F075A1FE751A00EEA2E0BA
:1021800092AF7F010225C7C0E074F2122568A2AFAA
:10219000E433FED2AF9061A4E0F8759B00E591585E
:1021A000540860087591F71245618023E5915854F1
:1021B0001060087591EF1245678014E591A2E092D6
:1021C000F0E8A2E082F05007E0C2E0F01246BD90D5
:1021D00061A3E0F8E5E9585404600E12469375E9EE
:1021E000FB906193E0A2E640F2808FC0E074F212AF
:1021F0002568A2AFE433FED2AF9061A5E0F8E5BF59
:10220000585404600675BFFB1246D502217AC3E418
:1022100098F8E499F912224F8026C3E49AFAE49BD5
:10222000FBE920E7E912224FE498F8E499F922C388
:10223000E498F8E499F912224FE498F8E499F9C384
:10224000E49AFAE49BFB22EB20E7CFE920E7E0B930
:102250000010BB0008E88AF084F8AAF022E4FBC86A
:10226000FA22EB70227B10C833C8C933C933500738
:10227000C39AC3DBF280069A50012ADBEAC833F422
:10228000C8C933F4C9FA2275F008E4C833C8C933A1
:10229000C933C99AC99B5004C92AC93BD5F0ECFB84
:1022A000C833F4C8E4C9FA2274F512250274FA128C
:1022B0002AC87508047509007808122A21740412C6
:1022C0002AAA7AF87B0779031243ED7402122A34A2
:1022D0009080B07808122C707402122CC778081203
:1022E0002ADE70497508027509007808122A2174DF
:1022F00002122AAA7AF67B0779031243ED740212BE
:102300002A34851882851983E0F47003A3E0F46011
:102310001C851882851983E0F8A3E0F988828983F7
:102320007402F0A3F0A37469F0A374A5F0C2AF75B2
:10233000D69F0200007406122A347F0402278C08FC
:102340000808EAC0E0EBC0E086F0E7A4FA180986C6
:10235000F0E7A42AFA180986F0E7A42AFA180986F1
:10236000F0E7A42AFA1986F0E7A4FBE5F02AFA19A7
:102370000886F0E7A42BFBE5F03AFA190886F0E7A7
:10238000A42BFBE5F03AFA18180986F0E7A4C5F08B
:102390002BFBE43AFA1908E7C5F0C6A426F6E5F0E7
:1023A0003BFBE43AFA1886F0E7A4F6E5F00826F6D7
:1023B000E43B08F6E43A08F6D0E0FBD0E0FA22E489
:1023C000CFC0E0E4CEC0E0E4CDC0E0E4CCC0E07536
:1023D000F020E626F608E633F608E633F608E6339C
:1023E000F6181818EC33FCED33FDEE33FEEF33FF37
:1023F000C3EC9709ED9709EE9709EF971919194062
:102400000FFFEC97FC09ED97FD09EE97FE191906F1
:10241000D5F0BFECF709EDF709EEF709EFF7191959
:1024200019D0E0FCD0E0FDD0E0FED0E0FF2225187E
:10243000C582C0E0E51934FFC583C0E0E518C39547
:102440008224F810AF088583198582188008858357
:1024500019858218D2AFCEF0A3E520F0A37808E664
:1024600008F0A3DEFAEFF0A3E58124FAF8E608F01D
:10247000A3E608F0A3E608F0A30808E608F0A3E640
:1024800008F0A315811581D0E0FED0E0F815811584
:10249000811581E8C0E0EEC0E022122CBCB9000337
:1024A0000224ECE49004D1789B79118002F0A3D847
:1024B000FCD9FA781A9020867A01BA00028007E4E3
:1024C00093A3F608DAF97A6B7B15902094789479C7
:1024D000018015E493A3AD82AE838A828B83F0A33F
:1024E000AA82AB838D828E83D8E9D9E77582EB759A
:1024F00083FD74041229E07582E975834A74001221
:1025000029E02518C582C0E0E51934FFC583C0E085
:10251000E518C3958224F910AF08858319858218C0
:102520008008858319858218D2AFCEF0A3E520F00C
:10253000A37808E608F0A3DEFAEFF0A3E58124FB18
:10254000F8E608F0A3E608F0A30808E608F0A3E61A
:1025500008F0A315811581D0E0FED0E0F8158115B3
:1025600081E8C0E0EEC0E022C0D02518C582C0E0FE
:10257000E51934FFC583C0E0E518C3958224F31044
:10258000AF0885831985821880088583198582188C
:10259000D2AFC8F0A3E9F0A3EAF0A3EBF0A3790867
:1025A000E709F0A3D8FAECF0A3EDF0A3EEF0A3EF67
:1025B000F0A3D0E0F0A3D0E0F0A3D0E0F0A3E520BA
:1025C000F0A3E5F0F0A322851983851882E0C0E02E
:1025D000A3E0F9A3E0FAA3E0FBA37808E0F608A3E0
:1025E000DFFAE0FCA3E0FDA3E0FEA3E0FFA3E0C070
:1025F000E0A3E0C0E0A3E0F5D0A3E0F520A3E0A3D2
:10260000F5F010AF08858319858218800885831935
:10261000858218D2AFD082D083D0E0F8D0E03208E3
:1026200075F0108E218F228582268583258518825C
:10263000851983E0CEA3E0CF852682852583EBC96B
:10264000EAC8EDCBECCAC3E833C8E933C9EA33CAF8
:10265000EB33CBC3EA9EF524EB9FF523B35004ABD9
:1026600023AA24EC33CCED33CDD5F0DAAE21AF2262
:1026700022D083D082ECC0E0EDC0E0E493A3FCE480
:1026800093A3FDED4C600D1227CCEC24FFFCED3440
:10269000FFFD80EFE493A3FCE493A3FDED4C600DFC
:1026A00012289FEC24FFFCED34FFFD80EFD0E0FD0D
:1026B000D0E0FCE493A3C0E0E493C0E0228519835A
:1026C000851882E0A3FEE0A3F5207808E0A3F608D1
:1026D000DFFAE0A3FFE0A3C0E0E0A3C0E0E0A3C016
:1026E000E0E0A3C0E0E0A3C0E010AF088582188559
:1026F00083198008858218858319D2AFD083D08250
:102700000229E6D083D082E9C0E0E493A3C386F037
:10271000C5F095F0F908E493A386F0C5F095F07044
:102720000BE493A3C3994005E9048002A3E475F088
:1027300002A42582F582E5F03583F583D0E0F9E443
:1027400093A3C0E0E493C0E022C0E074F2122568D5
:10275000A2AFE433FED2AFC2C0901463E0700BE5C9
:10276000D1A2E4501D1244718018E5D1A2E35006B5
:1027700075D1F7124447E5D1A2E4500675D1EF12A6
:10278000444DEEA2E092AF7F010225C785198385F3
:102790001882E0A3FEE0A3F5207808E0A3F608DFA6
:1027A000FAE0A3FFE0A3C0E0E0A3C0E0E0A3C0E044
:1027B000E0A3C0E010AF08858218858319800885E2
:1027C0008218858319D2AFD083D08222C0E0C3E4BF
:1027D0009396087401939618400FE4936670080866
:1027E000740193661870007019A3A3C3E49396084C
:1027F0007401939618A3A3400DD0E0D0E0D0E0027E
:1028000026ADA3A3A3A3A3A3D0E022D083D082C5E7
:10281000F0E493A3C5F0C395F0F5F0E493A3C3955A
:10282000F04005E5F0048001E475F002A42582F58E
:1028300082E5F03583F583E493A3C0E0E493C0E040
:10284000227404800474028000CCC0E0EDC0E0E596
:1028500018C39CCCAD1950011D10AF068C188D19F2
:1028600080068C188D19D2AF122962D0E0FDD0E01D
:10287000FC2274028000CCC0E0EDC0E0E518C39CEF
:10288000CCAD1950011D10AF068C188D1980068C27
:10289000188D19D2AF122940D0E0FDD0E0FC22C043
:1028A000E0C0F088F0E4936670080874019366183D
:1028B0007000A8F0A3A3700BD0F0D0E0D0E0D0E07F
:1028C0000226ADA3A3D0F0D0E022D083D082CCC02A
:1028D000E0E493A360061229A21470FAE493A360C3
:1028E00006122AB21470FAD0E0FCE493A3C0E0E42C
:1028F00093C0E022C0E074F2122568758900C2C559
:10290000901463E0700E7A007B1090071EE0F912BD
:102910003D0380031249517F010225C7C0E0C0D0AA
:10292000E8C0E0E9C0E0E5A8D2AFC2C7751A00A2CE
:10293000E7A2E792AFD0E0F9D0E0F8D0D0D0E03213
:10294000CAC0E0E493A3C582CCC582C583CDC5834C
:10295000F0A3C582CCC582C583CDC583DAE5D0E0BE
:10296000CA22CAC0E0E0A3C582CCC582C583CDC55A
:1029700083F0A3C582CCC582C583CDC583DAE6D0FA
:10298000E0CA22C008C3E096F50808A3E096420812
:1029900008A3E096420808A3E09645087001D3D04A
:1029A0000822C0E0E493A3D39C5010E493A3C39CFB
:1029B000400AD0E0D0E0D0E00228E7A3A3A3D0E013
:1029C000227009080808226016181818C6C333C6F2
:1029D00008C633C608C633C608C633C6D5E0EA22E1
:1029E000C09FF59FE473D09F22D083D082C09FE424
:1029F00093C0E0740193C0E0740293F59F22251800
:102A0000F58210AF08F518400C15198008F518402C
:102A1000021519D2AF851983227404800A740380C9
:102A200006740280027401C0E0F4041229FED0E0B2
:102A3000122C7F2200C0D0251810AF08F518500CBA
:102A400005198008F51850020519D2AFD0D022BB65
:102A50000102E722C082C08389828A83BB0003E02F
:102A60008002E493D083D082226016080808C6C38F
:102A700013C618C613C618C613C618C613C6D5E0A3
:102A8000EA22C3E0C696F608A3E0C696F608A3E0DD
:102A9000C696F608A3E0C696F6222518F8E435197E
:102AA000F9222518FAE43519FB222518FCE435191A
:102AB000FD22C0E0E493A36C7009D0E0D0E0D0E048
:102AC0000228E7A3A3D0E022251810AF08F518408C
:102AD0000C15198008F51840021519D2AF22E066CE
:102AE000701008A3E066700A08A3E066700408A3EB
:102AF000E06622C3E09608A3E09608A3E09608A348
:102B0000E096A2D265D03322E76670100809E76626
:102B1000700A0809E76670040809E76622C3E096B0
:102B2000F008A3E096F008A3E096F008A3E096F082
:102B300022C3E697F60809E697F60809E697F6082D
:102B400009E697F622C3E4939608740193960874F5
:102B5000029396087403939622E647F60809E6471F
:102B6000F60809E647F60809E647F622E056F008B7
:102B7000A3E056F008A3E056F008A3E056F022E0E8
:102B800026F008A3E036F008A3E036F008A3E0360C
:102B9000F022E627F60809E637F60809E637F608D0
:102BA00009E637F622E657F60809E657F60809E679
:102BB00057F60809E657F622E056F608A3E056F65F
:102BC00008A3E056F608A3E056F622E026F608A38E
:102BD000E036F608A3E036F608A3E036F6227004E5
:102BE00022600D18C6C333C608C633C6D5E0F41834
:102BF00022E4C396F608E496F608E496F608E4960E
:102C0000F622C6F4C608C6F4C608C6F4C608C6F45A
:102C1000C622600D08C6A2E713C618C613C6D5E0C3
:102C2000F322C3E7960809E7960809E7960809E73B
:102C30009622C3E09608A3E09608A3E09608A3E0D6
:102C4000962275D00075813F7518D1751904000260
:102C5000249A600C08C6C313C618C613C6D5E0F480
:102C600022E6F008A3E6F008A3E6F008A3E6F022C7
:102C7000E0F608A3E0F608A3E0F608A3E0F622CA0F
:102C8000C0E0E6F0A308DAFAD0E0FA22EAF0A3EB1B
:102C9000F0A3ECF0A3EDF022E0FAA3E0FBA3E0FC4C
:102CA000A3E0FD22E0F8A3E0F9A3E0FAA3E0FB2211
:102CB000E8F0A3E9F0A3EAF0A3EBF022E5C754F8AB
:102CC0004401F5C77901222518F582E43519F58309
:102CD000221229E978AC021229E98CAC021229E906
:102CE000A0AC021229E9DCAC021229E90CAD0212F7
:102CF00029E9A5AE021229E961AF021229E919B04A
:102D0000021229E96EB0021229E9D1B0021229E9B2
:102D10000FB1021229E939B1021229E9C5B1021233
:102D200029E91EB2021229E97FB2021229E9BEB4D2
:102D3000021229E992B6021229E971B7021229E9B1
:102D4000AAB8021229E95DBB021229E970BE02127B
:102D500029E97FBE021229E90BBF021229E9C1BF8E
:102D6000021229E908C0021229E951C0021229E918
:102D70008DC0021229E903C1021229E96FC10212B2
:102D800029E98BC1021229E9BCC1021229E9FBC160
:102D9000021229E9FCC2021229E9ABC3021229E995
:102DA0003CC6021229E995C7021229E928C8021275
:102DB00029E9B2C8021229E9D6C8021229E987C94D
:102DC000021229E938CA021229E9B5CB021229E90F
:102DD00040CC021229E97FCC021229E9F5CC02127B
:102DE00029E94ACE021229E9EDCE021229E921CFC2
:102DF000021229E939CF021229E9DCCF021229E9AE
:102E000066D2021229E907D4021229E925D4021256
:102E100029E943D4021229E913D5021229E968D815
:102E2000021229E90080031229E95A80031229E9D4
:102E3000C480031229E94D81031229E90982031292
:102E400029E95182031229E98C82031229E9E282DD
:102E5000031229E94A83031229E9CE83031229E9DF
:102E6000E783031229E90C84031229E92B84031256
:102E700029E96984031229E9B884031229E9E18464
:102E8000031229E93085031229E9DC85031229E9B7
:102E9000A486031229E90987031229E9D6870312B8
:102EA00029E91C88031229E93888031229E96A886C
:102EB000031229E9128A031229E9E98A031229E98E
:102EC000158B031229E94B8B031229E96C8B031232
:102ED00029E97B8B031229E9868B031229E93A8CB5
:102EE000031229E9AD8C031229E91F8D031229E988
:102EF000278D031229E9A28D031229E9FB8D031204
:102F000029E93E8E031229E9D090031229E916928D
:102F1000031229E9A694031229E98E95031229E9DF
:102F2000C195031229E98396031229E93297031206
:102F300029E97A97031229E9DC97031229E9019814
:102F4000031229E91298031229E98A98031229E940
:102F50001299031229E97699031229E95B9A03125F
:102F600029E9809A031229E9A19B031229E9BF9B51
:102F7000031229E9D29B031229E9459C031229E98E
:102F8000549C031229E9DC9C031229E9249D0312B5
:102F900029E9319D031229E93A9D031229E93A9F53
:102FA000031229E98EA0031229E99EA0031229E940
:102FB000BAA1031229E933A2031229E969A3031272
:102FC00029E9ABA3031229E9E7A3031229E9BBA569
:102FD000031229E920A8031229E934A8031229E9D8
:102FE0003EA8031229E948A8031229E952A80312AE
:102FF00029E95CA8031229E975A8031229E97FA829
:10300000031229E989A8031229E993A8031229E9DF
:10301000C2A8031229E9EAA8031229E9F5A80312B4
:1030200029E93FA9031229E949A9031229E954A969
:10303000031229E978A9031229E99CA9031229E9B5
:10304000FDA9031229E948AA031229E964AA031277
:1030500029E9CEAA031229E91AAB031229E962ABC6
:10306000031229E9DDAB031229E977AC031229E940
:103070003BAE031229E9A9AE031229E9DBAF031223
:1030800029E901B0031229E971B1031229E925B533
:10309000031229E925B7031229E9FDB8031229E92A
:1030A00096B9031229E9A8BB031229E96ABC0312E5
:1030B00029E9B6BC031229E91CBD031229E92EBD7A
:1030C000031229E97EBF031229E96DC0031229E921
:1030D000ACC1031229E9FEC1031229E9A3C20312FC
:1030E00029E95EC4031229E98FC5031229E9ADC598
:1030F000031229E902C6031229E900C7031229E9CC
:1031000028C7031229E98BC7031229E98CC80312C7
:1031100029E9FFC8031229E92DCA031229E998CA2F
:10312000031229E988CB031229E9EECD031229E91C
:103130001CCE031229E917CF031229E9B5D00312D7
:1031400029E905D1031229E9BDD1031229E972D277
:10315000031229E9D6D2031229E98FD3031229E9F0
:103160002FD4031229E993D4031229E9DDD40312E1
:1031700029E91AD5031229E982D6031229E91D810A
:10318000011229E95F81011229E95A84011229E912
:10319000AD84011229E9F384011229E93486011270
:1031A00029E99986011229E9D986011229E91C88A1
:1031B000011229E95E8B011229E9878C011229E9A4
:1031C000C897011229E96898011229E95B9B01124D
:1031D00029E9929C011229E9089D011229E9329EF0
:1031E000011229E9829F011229E969A0011229E946
:1031F000D2A2011229E9E0A4011229E971A5011264
:1032000029E945A6011229E9D1A6011229E9DBA67F
:10321000011229E903A7011229E9B0A7011229E93E
:103220009BA8011229E96EA9011229E9FBA9011243
:1032300029E911AA011229E975AA011229E99EAA10
:10324000011229E9CBAA011229E910AD011229E9DD
:10325000EBAD011229E92FAE011229E9A0AE01124E
:1032600029E959AF011229E98BAF011229E9D2AF3F
:10327000011229E905B0011229E96AB0011229E910
:10328000B9B0011229E9BEB0011229E912B1011247
:1032900029E95CB1011229E958B2011229E9BDB24C
:1032A000011229E91BB3011229E965B6011229E9C6
:1032B00039B7011229E9C6B8011229E9A0BB0112E8
:1032C00029E953BC011229E97ABE011229E91FBF7D
:1032D000011229E95DBF011229E92DC1011229E975
:1032E00040C1011229E949C1011229E952C1011263
:1032F00029E967C1011229E986C1011229E9BBC385
:10330000011229E90EC4011229E918C4011229E9A0
:1033100022C4011229E97DC4011229E9D9C401128C
:1033200029E9F1C5011229E952C6011229E9A1C70B
:10333000011229E9EAC7011229E9C2C8011229E9E3
:10334000EDC9011229E9A3CA011229E9A5CB01128D
:1033500029E9A7CC011229E98CCD011229E9A3CDD5
:10336000011229E9E0CD011229E9EACD011229E98A
:10337000F4CD011229E9FFCD011229E91DCE011278
:1033800029E95FCE011229E9BDCE011229E9E2CE79
:10339000011229E9FCCE011229E989CF011229E99C
:1033A000C2CF011229E912D1011229E969D1011212
:1033B00029E983D2011229E9B9D2011229E955D3A9
:1033C000011229E9D1D3011229E941D5011229E9D4
:1033D0005CD6011229E922D7011229E9CCD70112C2
:1033E00029E951D8011229E9B9D8011229E96ED980
:1033F000011229E9C0D9011229E935DA011229E9B6
:10340000FEDA011229E921DB011229E9E5DB0112CB
:1034100029E909DC011229E92BDC011229E98CDCFC
:10342000011229E9D7DE011229E9B2DF011229E9E7
:103430005CE0011229E99DE2011229E9EBE20112A7
:1034400029E92EE3011229E986E3011229E9E4E3DF
:10345000011229E90EE4011229E932E4011229E9F5
:1034600063E4011229E98DE4011229E9D4E401128F
:1034700029E932E5011229E98EE5011229E98FE6F1
:10348000011229E9F9E7011229E937E8011229E9CE
:1034900060E8011229E9F1E8011229E93BE901128A
:1034A00029E95FE9011229E9B5E9011229E9D0E921
:1034B000011229E98BEA011229E9B5EA011229E989
:1034C000F8EA011229E94EEB011229E953EE011243
:1034D00029E986EE011229E943EF011229E91EF0DC
:1034E000011229E9AEF0011229E9EFF0011229E9F0
:1034F00065F3041229E99DF3041229E9BEF30412CD
:1035000029E900F4041229E964F4041229E96EF4AB
:10351000041229E97EF4041229E9B5F4041229E918
:103520005EF8041229E926FA041229E91AFC0412A9
:1035300029E9B8FC041229E93FFD041229E94D806C
:10354000041229E9F680041229E9D581041229E937
:10355000F082041229E91083041229E9328404124A
:1035600029E9CF85041229E93C86041229E912874A
:10357000041229E91888041229E97D88041229E92E
:10358000B988041229E91289041229E94B89041225
:1035900029E99489041229E9268A041229E9C38AAF
:1035A000041229E9988B041229E9658C041229E98F
:1035B000F28C041229E9188D041229E9458D0412B0
:1035C00029E9768D041229E94B8E041229E95B8ED4
:1035D000041229E9AE8E041229E9BB8E041229E9EE
:1035E000C88E041229E9D18E041229E9358F0412FC
:1035F00029E9938F041229E9DE8F041229E9F98F52
:10360000041229E92090041229E93D90041229E9C5
:103610004990041229E9ED91041229E90692041255
:1036200029E98292041229E99592041229E9A592C6
:10363000041229E94B93041229E9BB94041229E9E5
:10364000CE95041229E96E96041229E9789604129F
:1036500029E9E696041229E9F796041229E9369732
:10366000041229E96497041229E93198041229E91E
:103670008898041229E9CD98041229E923990412A3
:1036800029E94199041229E98F99041229E95D9ADF
:10369000041229E9AB9A041229E9ED9A041229E9E6
:1036A000709B041229E99A9B041229E9D09B041209
:1036B00029E9DF9B041229E93D9C041229E9B59C04
:1036C000041229E9F69C041229E9459D041229E90E
:1036D000709D041229E98A9D041229E9A49D04120F
:1036E00029E9799E041229E9839E041229E9BE9EE4
:1036F000041229E9CE9E041229E9D79E041229E971
:10370000289F041229E93C9F041229E95AA00412B7
:1037100029E96DA0041229E984A0041229E999A0DD
:10372000041229E933A1041229E9B2A1041229E9FA
:1037300055A2041229E960A2041229E9ADA30412DA
:1037400029E9C9A3041229E921A4041229E98FA4B3
:10375000041229E9DBA4041229E9F5A4041229E9D9
:1037600055A5041229E9F3A5041229E93EA604127D
:1037700029E9A1A8041229E939A9041229E9B0A963
:10378000041229E9F6AB041229E90EAC041229E966
:1037900011AC041229E91DAC041229E931AC041260
:1037A00029E939AC041229E970AC041229E964ADA5
:1037B000041229E9EEAD041229E970AE041229E9D8
:1037C000E5AE041229E9BDAF041229E9DFAF041206
:1037D00029E976B0041229E982B0041229E9DFB0A0
:1037E000041229E9E2B0041229E90FB1041229E90F
:1037F00024B1041229E993B1041229E9DFB20412B9
:1038000029E9F2B3041229E97DB4041229E990B53B
:10381000041229E95AB6041229E98BB6041229E9DF
:10382000B1B6041229E9BAB6041229E9E9B60412BC
:1038300029E999B7041229E949B8041229E9BCB861
:10384000041229E96EB9041229E9E1B9041229E93F
:1038500020BA041229E969BA041229E99EBA0412AD
:1038600029E91FBD051229E98ABD051229E9D1BD43
:10387000051229E947BE051229E997BE051229E973
:103880001BBF051229E95FC1051229E98AC3051288
:1038900029E967C7051229E9E4C7051229E91FC804
:1038A000051229E93DC8051229E99DC8051229E933
:1038B000C5C8051229E9F5C8051229E926C9051266
:1038C00029E953C9051229E9ACC9051229E9F7C943
:1038D000051229E9CAA2051229E946A3051229E918
:1038E0006CA3051229E9A3A3051229E9FCA405127A
:1038F00029E918A5051229E95DA5051229E9EDA513
:10390000051229E945A6051229E91AA7051229E990
:10391000F8A7051229E942A8051229E9A3A805126A
:1039200029E927A9051229E950A9051229E991A930
:10393000051229E93FAB051229E90FAC051229E967
:10394000D6AC051229E9A9AD051229E9E3AD0512A6
:1039500029E93BAE051229E95DAE051229E9F1AE70
:10396000051229E9A4AF051229E94C8D061229E9AF
:10397000B18D061229E9588E061229E9908E061299
:1039800029E9B0F1011229E95BF2011229E9F8F302
:10399000011229E974F4011229E9ACF4011229E9B0
:1039A00097F7011229E929F9011229E993F901127E
:1039B00029E9CBFC011229E96CFE011229E992AE3A
:1039C000061229E9BAAE061229E9A6AF061229E9BC
:1039D000DCE1051229E95FE2051229E976E2051228
:1039E00029E9E9E2051229E94FE3051229E978E31B
:1039F000051229E9FDE3051229E99FE4051229E9E9
:103A000002E5051229E967E5051229E987E50512AE
:103A100029E9B7E5051229E9D3E5051229E902E606
:103A2000051229E932E6051229E968E6051229E9B5
:103A3000C8E6051229E9F8AF051229E9C8B0051250
:103A400029E9EDB0051229E90DB1051229E921B1E5
:103A5000051229E989B1051229E9ADB1051229E953
:103A60002BB3051229E951B4051229E932B5051223
:103A700029E996B5051229E9C2B5051229E946B624
:103A8000051229E997B6051229E9B8B6051229E900
:103A900030B7051229E9D4B8051229E937B905125A
:103AA00029E9C7BA051229E994BB051229E9CFBB58
:103AB000051229E9F4BB051229E914BC051229E90C
:103AC0003ABC051229E94EBC051229E9B7BC05121A
:103AD00029E90BBD051229E99FA3061229E9A9A32B
:103AE000061229E9CAA3061229E92C94051229E92C
:103AF0003A97051229E96798051229E9429A0512B1
:103B000029E9CC9A051229E9859B051229E9AE9B82
:103B1000051229E9F89B051229E9BDA4021229E939
:103B2000269D051229E9299D051229E92C9D0512DA
:103B300029E92F9D051229E94F9D051229E9529D7A
:103B4000051229E96B9D051229E9CF9D051229E986
:103B5000C19E051229E9F69F051229E943A0051225
:103B600029E94AA1051229E91CA2051229E9F5D67D
:103B7000031229E92DD7031229E964AC021229E9BD
:103B8000BDDC031229E944DD031229E975DD0312C6
:103B900029E9A3DD031229E9F7DD031229E925DE6E
:103BA000031229E946DF031229E974DF031229E928
:103BB000A2DF031229E9D8DF031229E985E0031205
:103BC00029E9ABE0031229E90AE1031229E980E2BD
:103BD000031229E91AE3031229E90BE4031229E984
:103BE000E8E4031229E932E5031229E981E5031229
:103BF00029E9EDE5031229E955E6031229E9A2E6D0
:103C0000031229E912E7031229E923E8031229E93B
:103C100017E9031229E9C8E9031229E9FDE90312AA
:103C200029E952EA031229E9F4EA031229E922EB0D
:103C3000031229E9A7EC031229E92CED031229E963
:103C40006CED031229E9ABED031229E9C4ED03126F
:103C500029E973EE031229E93DEF031229E9E4EFA4
:103C6000031229E978F0031229E91EF1031229E968
:103C700088F1031229E913F2031229E9A6F20312CB
:103C800029E9C4F2031229E997F3031229E955F44B
:103C9000031229E90BF5031229E9A9F5031229E911
:103CA0004079001229E98179001229E9EA790012A4
:103CB00029E90B7A001229E9247A001229E9DE7A2F
:103CC000001229E9E77A001229E9387B001229E974
:103CD000617B001229E9787B001229E9DC7B001264
:103CE00029E96E7C001229E99F7C001229E9FB7CFE
:103CF000001229E9617D001229E9957D001229E968
:103D0000087E001229E94A7E001229E98A7E001203
:103D100029E9C27E001229E9D47E001229E9E67E53
:103D2000001229E9177F001229E9577F001229E9BB
:103D3000807F001229E92AF2051229E96DF30512A4
:103D400029E993F3051229E9A4F3051229E9BCF541
:103D5000051229E9DBF5051229E9ECA5061229E986
:103D600022A6061229E96DA6061229E9B9A70612AC
:103D700029E90080051229E93E81051229E97A81A5
:103D8000051229E93F83051229E96983051229E90A
:103D9000EF85051229E92F86051229E9C487051246
:103DA00029E95988051229E9B788051229E94889BE
:103DB000051229E98089051229E9C289051229E934
:103DC0003C8B051229E9C58C051229E9FB8E0512E9
:103DD00029E9298F051229E9558F051229E95E8FF6
:103DE000051229E9B48F051229E94490051229E941
:103DF0004B93051229E9CF93051229E904B806125D
:103E000029E91AB8061229E924B8061229E974B872
:103E1000061229E9D084061229E9E984061229E963
:103E20008E85061229E9CE85061229E9E785061254
:103E300029E91B86061229E96886061229E99C866B
:103E4000061229E9DE86061229E9B488061229E954
:103E50001F89061229E90FB1061229E964B1061279
:103E600029E9BDB1061229E9B5B6061229E908B754
:103E7000061229E94AB7061229E95AB7061229E9B2
:103E800006BB041229E95EBB041229E9FEBB041239
:103E900029E916BD041229E902BE041229E9CFBEA0
:103EA000041229E9E4BE041229E92EBF041229E90B
:103EB00085BF041229E9F1BF041229E904C00412E4
:103EC00029E95CC0041229E9CBC0041229E962C3C4
:103ED000041229E95EC4041229E9B9C4041229E9CB
:103EE0000DC5041229E929C7041229E979C704126A
:103EF00029E9FAC7041229E9CCC8041229E905C93D
:103F0000041229E924C9041229E96FC9041229E914
:103F100085C9041229E992C9041229E9CBC90412FE
:103F200029E9DDC9041229E9CCCA041229E9D7CA52
:103F3000041229E95CCB041229E9B4CB041229E963
:103F400000CC041229E937CD041229E95FCD04120F
:103F500029E9DBCF041229E903D0041229E915D19C
:103F6000041229E944D1041229E9BCD1041229E937
:103F70007ED2041229E9B2D2041229E922D3041212
:103F800029E9FFD3041229E938D4041229E942D4DB
:103F9000041229E945D4041229E94FD4041229E96D
:103FA0006BD4041229E9E7D4041229E920D50412BC
:103FB00029E93CD5041229E968D5041229E9A3D5D9
:103FC000041229E9BED5041229E9C8D5041229E949
:103FD000F7D5041229E90DD6041229E929D60412CD
:103FE00029E958D6041229E978D6041229E9C1D65C
:103FF000041229E90AD7041229E914D8041229E97C
:1040000048B4061229E959B4061229E9E2B40612A5
:1040100029E9B4DA051229E903DB051229E9C1DC33
:10402000051229E994DE051229E9D2DE051229E9F3
:10403000A8DF051229E9ADE0051229E9CFE0051254
:1040400029E92BE1051229E9ACE1051229E9A5507E
:10405000001229E9C750001229E91952001229E972
:104060006252001229E9DB52001229E9565300126C
:1040700029E9BF53001229E90654001229E97454B2
:10408000001229E91955001229E99F55001229E962
:10409000DB55001229E92F5A001229E93D5C001274
:1040A00029E9705C001229E9AF5C001229E9BC5DC6
:1040B000001229E9A560001229E94F61001229E9DF
:1040C000FA62001229E92D64001229E94365001201
:1040D00029E9B865001229E98466001229E91B67FD
:1040E000001229E92B67001229E9E267001229E989
:1040F0001869001229E95C6B001229E9FF6D0012B2
:1041000029E9DD6E001229E91A70001229E95F73AE
:10411000001229E96F73001229E9A674001229E937
:104120005975001229E98A76001229E9F8760012F9
:1041300029E92F78001229E98478001229E95FD94A
:10414000041229E906DA041229E978DA041229E9C5
:1041500088DA041229E90ADB041229E961DB041276
:1041600029E956DC041229E97DDC041229E922DD63
:10417000041229E971DD041229E9CFDD041229E9CD
:104180002ADE041229E905E1041229E9BEE104123C
:1041900029E923E2041229E9B6E3041229E956E4E5
:1041A000041229E9EFE4041229E94CE5041229E993
:1041B000C2E5041229E9BEE6041229E9B1E70412B6
:1041C00029E90AE8041229E920E8041229E941E86A
:1041D000041229E980E8041229E910E9041229E906
:1041E00053EA041229E910EC041229E95AED0412E9
:1041F00029E994EE041229E99FEF041229E93FF01E
:10420000041229E9AEF0041229E9CBF1041229E9DC
:1042100086D8021229E9EFD8021229E937D9021209
:1042200029E97BD9021229E9EED9021229E948DAF3
:10423000021229E983DA021229E91DDB021229E9B7
:1042400077DB021229E9E3DC021229E95CDD0212C4
:1042500029E986DD021229E99ADE021229E9A8DF9E
:10426000021229E9D0DF021229E9CEE0021229E97F
:10427000DFE0021229E9F5E0021229E9F6E1021273
:1042800029E919E2021229E9E6E2021229E90EE31C
:10429000021229E925E3021229E94BE3021229E976
:1042A00086E3021229E9A6E3021229E9CDE302120C
:1042B00029E9E5E3021229E9C2E4021229E925E528
:1042C000021229E9A8E6021229E937E7021229E9D0
:1042D0005BE7021229E972E7021229E946E80212B5
:1042E00029E9E2E8021229E908E9021229E95DEA6E
:1042F000021229E97BEA021229E9F6EA021229E907
:104300002CEB021229E969EB021229E9F5EB021202
:1043100029E961EC021229E945ED021229E923EFAE
:10432000021229E9F8EF021229E944F0021229E900
:104330007CF1021229E9C9F2021229E93FF40212C2
:1043400029E94DF4021229E947F5021229E9EEF5AF
:10435000021229E937F6021229E94CF6021229E97C
:104360005BF7021229E974F8021229E9D2F8021265
:1043700029E904ED051229E941ED051229E9DAEDF3
:10438000051229E9E5EE051229E92DF1051229E9C1
:10439000A9F1051229E9E294061229E910960612FC
:1043A00029E9D896061229E92D97061229E9B0972E
:1043B000061229E95DFE041229E91CFF021229E90F
:1043C0002DFF021229E9CDFF021229E9E7FF0212AF
:1043D00029E9E8FF011229E93BB5061229E94BB5A5
:1043E000061229E960B5061229E9F1B5061229E994
:1043F00044B3061229E9C9B3061229E92FB40612FB
:1044000029E9EF7F001229E9D67F001229E9E67F2A
:10441000001229E9E97F001229E9EC7F001229E95D
:10442000F87F001229E91CA8061229E93EA8061205
:1044300029E9ACA9061229E930AA061229E9BFFF29
:10444000011229E9C8FF011229E9D1FF011229E966
:10445000DFFF011229E973F9021229E9DFF90212DB
:1044600029E9A7FA021229E9A0FB021229E98DFD28
:10447000021229E9E7FD021229E93AFE021229E9AE
:104480004BFE021229E95DFE021229E9C9FE021261
:1044900029E9DDFE021229E9E8FE021229E9F6FE09
:1044A000021229E908FF021229E97CE7051229E92D
:1044B000A8E7051229E94FEA051229E9A4EA05123D
:1044C00029E9E0EA051229E9F4EA051229E90DEBE8
:1044D000051229E900EC051229E9DCEC051229E9AD
:1044E000F0EC051229E9C2AB061229E9E6AB061287
:1044F00029E9FFAB061229E93EAC061229E971ACA5
:10450000061229E9A1AC061229E9ABAC061229E989
:1045100013AD061229E916AD061229E920AD0612DF
:1045200029E92DAD061229E9F1A0061229E919A100
:10453000061229E95AA1061229E978A1061229E9E9
:1045400093A1061229E9FBA1061229E907A2061286
:1045500029E966A2061229E98AA2061229E94BA3D3
:10456000061229E958A3061229E969A3061229E9C6
:10457000A2B8061229E9BAB8061229E9E0B806126B
:1045800029E973F7051229E9BCF8051229E9C2F8EF
:10459000051229E9D9F8051229E9FAF8051229E9DD
:1045A00010F9051229E924F9051229E9A3F90512E0
:1045B00029E908FA051229E990FA051229E909FB07
:1045C000051229E9E2FB051229E9F2FB051229E9A6
:1045D00001FC051229E96BB7061229E98FB706120B
:1045E00029E9B7B7061229E9DFB7061229E9329E91
:1045F000061229E99E9E061229E9BD9E061229E9A6
:10460000239F061229E9699B061229E9829B06125B
:1046100029E9999B061229E9A29B061229E9C09B68
:10462000061229E9CA9B061229E9D49B061229E938
:10463000E79B061229E9749C061229E9E39C0612FD
:1046400029E9119D061229E9629D061229E9AE9D0C
:10465000061229E9C99D061229E9D39D061229E906
:10466000E49D061229E9279E061229E929B90612B6
:1046700029E974B9061229E96EF6031229E99AF6B6
:10468000031229E9B8F6031229E9CBF6031229E946
:10469000E6F6031229E945F7031229E973F7031235
:1046A00029E97FFB031229E9C1FC031229E9F3FC84
:1046B000031229E95EFD031229E9E2FE031229E94A
:1046C0000AFF031229E91FFF031229E92FFF031232
:1046D00029E96FFF031229E9B1FF031229E9C1FF9C
:1046E000031229E9D7AF061229E9E7AF061229E933
:1046F00005B0061229E920B0061229E947B00612D2
:1047000029E968B0061229E982B0061229E9BAB08F
:10471000061229E9DDB0061229E901B6061229E9D7
:1047200047B6061229E94A91061229E95A9106125A
:1047300029E97892061229E9AA92061229E9CC926F
:10474000061229E9F492061229E90D93061229E9C5
:104750004993061229E9B293061229E9EE9306124B
:1047600029E93594061229E96294061229E98E9402
:10477000061229E933AA061229E96AAA061229E9CA
:1047800092AB061229E995AB061229E931B206125D
:1047900029E9A3B2061229E9E1B2061229E922B3F6
:1047A000061229E9ABD2051229E9B1D2051229E98D
:1047B000F8D2051229E904D5051229E934D50512E4
:1047C00029E99ED5051229E959D6051229E9A0D66D
:1047D000051229E9D3D6051229E95DD7051229E981
:1047E00074D7051229E981D7051229E98BD705125B
:1047F00029E92BD9051229E91DDA051229E97BDA05
:10480000051229E92ECA051229E944CA051229E927
:10481000F6CA051229E920CC051229E915CD0512A1
:1048200029E9ACCD051229E9E7CD051229E959CED0
:10483000051229E9B7CE051229E9C7CE051229E9E3
:10484000EECE051229E940CF051229E9AFD00512B5
:1048500029E9B4D0051229E9D6D0051229E92C8915
:10486000061229E94A89061229E98E89061229E9E0
:10487000B489061229E9D689061229E9EE890612B9
:1048800029E9068A061229E91E8A061229E9C48A3C
:10489000061229E9068B061229E9108B061229E96E
:1048A000258B061229E92C8C061229E9478C061261
:1048B00029E9508C061229E9598C061229E9628CE3
:1048C000061229E96C8C061229E9E98C061229E9FD
:1048D0000080061229E94584061229E9618406123E
:1048E00029E96684061229E932FC051229E948FC07
:1048F000051229E9E6FD051229E931FE051229E92B
:104900009BFE051229E99AFF051229E9C9FF051244
:1049100029E9DBFF051229E937AD061229E942989A
:10492000061229E99E98061229E9DE98061229E95D
:10493000E099061229E9F899061229E90D9A06125A
:1049400029E9399A061229E9709A061229E9809A0A
:10495000061229E9969A061229E9BB9A061229E954
:10496000469B061229E9AA7F001229E989A40212AE
:1049700029E95EA4021229E93AA4021229E95DA3F9
:10498000021229E927A3021229E9E7A2021229E962
:10499000B5A2021229E926A2021229E9D8A0021220
:1049A00029E95EA0021229E99B9F021229E9919E42
:1049B000021229E9489E021229E9229E021229E9DF
:1049C0005E9D021229E9A89B021229E9489B021266
:1049D00029E9199B021229E9169B021229E9DC999F
:1049E000021229E9C898021229E98897021229E9D6
:1049F000BA96021229E93296021229E950AC021243
:104A000029E9BCAB021229E9D4AA021229E94CAA6D
:104A1000021229E999A9021229E948A7021229E9F3
:104A20001DA7021229E95295021229E9B99402122E
:104A300029E91394021229E9D593021229E9BEA6A5
:104A4000021229E93B93021229E9FA92021229E99A
:104A50009D92021229E96A92021229E9EBDB031204
:104A600029E9FE91021229E92FA5021229E9CB9129
:104A7000021229E97091021229E93F91021229E9F3
:104A8000088E021229E91A8D021229E9D48B02122A
:104A900029E9808B021229E9748B021229E9DB8A49
:104AA000021229E9A989021229E9FA86021229E9E2
:104AB0009D84021229E95184021229E936830212E7
:104AC00029E9CB82021229E9F381021229E9AF8197
:104AD000021229E90080021229E96B80021229E9F9
:104AE0003280021229E9B39C0500000080FBE473C8
:104AF0008F0001009B09870001009A092400020031
:104B0000C51525000200C71526000200C91527009B
:104B10000200CB1528000100CD1529000100CE159B
:104B200084000400CF1586000100D3152A0001007F
:104B3000D4152B000100D5152C000100D9152D002E
:104B4000080082092E000100DA152F000100DB1594
:104B500030000100DC1531000100DD1532000100DC
:104B60008A09330001008B0934000100DE1536008C
:104B700001008C0938000100DF1539000100D8154B
:104B800083000200F1156300010097096400010031
:104B9000D61565000100D7156D0001009809710058
:104BA00008007A0966000100F01543000100E115D4
:104BB00044000200E21545000100E4154600020031
:104BC000E515470008008F0948000100E7154B0074
:104BD0000100E81504000100F315A1000100F5151E
:104BE00037000100F415880001009C093C00010019
:104BF0008D093D000100E01549000200E91567003C
:104C0000010099094D000200EB154E000100ED1561
:104C10004F000200EE153E0001008E09000000006A
:104C2000000000013636010100010201000103010C
:104C30000001040106060502000007010034080116
:104C4000000F090401010D0100FF0E08000017020A
:104C50000000190100FF1A0100011B0100FE1C01E8
:104C600000081D0200001F010001200100012102B7
:104C700000002301000F240200002601000127018B
:104C80000008280200FF2A0100072B0102402C0126
:104C900000002D0100012E0100012F0100FF300155
:104CA0000B1C310800003A0100083B01000F3C01D9
:104CB00000013D0100FF3E040000420400004604E4
:104CC00000004A0400004E04000052040000560494
:104CD00000005A0400005E20FFFF360001000600BD
:104CE00000000F00000000000000000000000000B5
:104CF00003FFFF00000403FFFF0000FFFF0FF401AC
:104D00000005C4040320000100000B0000000000A7
:104D100000000003010F0000000000000000000080
:104D20000000000000000000000000000000000083
:104D30000000000000000000000000000000000073
:104D40000000000000000000000000000000000063
:104D500000000000000000000103710301030103D3
:104D600001030103010322030203010310030003F3
:104D700000030003000300030003000342030003D9
:104D80002403060300030003040312032503230383
:104D90002503230304030403000300030003440367
:104DA000000300032303000365032100350381038F
:104DB000000305030003000300030003250323038E
:104DC0000300710030016000110070003102200307
:104DD00050048000100061000000140063007300A4
:104DE0007200620043000000130006000000000093
:104DF0000400120000000000000000000400040095
:104E0000370037003C0244000000000000000000B2
:104E100065000000350081000000050000008300EF
:104E200000000101710101010101110101013101C4
:104E3000010101018001100161013B0014006301C7
:104E400073017201620143010001130106013D017A
:104E500035000401120100010001000100010401FC
:104E60000401330133013C014401320136000001E9
:104E70000001650100013500810100010501820189
:104E8000830100010302710230016002110270020D
:104E90000102020202028002100261023A00410095
:104EA00063027302720262024302000213023800BC
:104EB00000020002040212020002000200020002CC
:104EC00004020402370037003C02440200023900A9
:104ED00000020002650200023502810200020502A2
:104EE00082028302000203047104020460041104BC
:104EF00070040204020401040204100461040004AA
:104F0000140463047304720462044304000413046D
:104F10000604000400040404120400040004000455
:104F2000000451046400000400040004440400046C
:104F300000040004000465040004350481046400D6
:104F4000050400048304000400007D411300ED40CB
:104F500001007D4102006F400300754004007B406A
:104F60000500814006008D403000B1403100AB406B
:104F70003200BD403300C3403500C9403400CF404B
:104F80003600D5401100E1401400E74015009F4075
:104F90001F00A540FFFF000001C33106F93108F3EF
:104FA000310B1132102D310A233202C93105E7319C
:104FB00007CF310CAB310DB731642F2FFF00000745
:104FC000ECFDFDFDECDCDCCCBCACAC9C9C8C7C7CBE
:104FD0006C6C5C5C5C4C4C3C3C2C2C1C1C03EAF563
:104FE000E5D5D5C5B5A59595858575756565555581
:104FF00045453535252515150500160F00000B15FF
:105000000B020002220F3300000E01030507090BFB
:105010000D0F00020406080A0C0D5A696742656507
:10502000416C6C69616E6365303930301718192135
:10503000301B1D1F30303016181920231A1C1E304B
:1050400000034A49434E181A250502000119161893
:105050001616182303000C0E020B040B0A07080097
:105060000F00393D3F373C3C362C442D02040201F1
:105070000101010902E803000000BE040A7F003CB0
:1050800000000000000E00E8033C00100C0A0C03B6
:10509000150900040009FF1E1E0305010C05040488
:1050A0000810080328C082C08390081DE4F0A3F014
:1050B0007CD57D047A8E7B0712479B122F35124ACE
:1050C000D1122F3B026E8074F312242E74F5122A33
:1050D000C889098A088B0AE9705F74026508703E06
:1050E0009007AD7408F0750C00780C122A25ECF5C9
:1050F0000C780C122A25EBF50C780C122A25901549
:10510000CF1228419015D3E0F97C8F7D099015F1DD
:10511000126E91122F5F7407122A340251D9740152
:10512000650860030251DC9007AD7408F07B00AAAB
:105130000AA90A122FA10251D974016509600974E4
:1051400002650960030251DCEA60067403650870B9
:10515000409007AD74021251FD122C98122F4D9001
:1051600007B5E0A2E34010E9700D900821E004F0DB
:105170006404700312520774036508705C9008227F
:10518000E0F8740128F0E8C39405404D12520780FE
:1051900048740165087045740165099007AD702E6B
:1051A000740AF07401122CC7E4F07402122CC77454
:1051B00003F004122CC7E4F0A3F0A3F0A3F07408EA
:1051C000122CC7E4F0AA18AB191231D58025740A45
:1051D0001251FD122C98122F83E960179080A412AF
:1051E00028417A017B009007AAE0F9123E29740455
:1051F000122A34740B122A347F050226BDF0901552
:10520000D3E0F99015CF229015CFE4F0A374F8F015
:10521000A374FFF0A37407F02274F612242EE9FFA2
:10522000EAFE7AD1F9123CDF8A828B83E5824583DC
:10523000702A7A027B00123CC1EA4B700E7A107B16
:10524000009007AAE0F9123D0380148A828B8374D0
:10525000D1F0EFA3F0EEF9123CCD8003EFA3F00202
:10526000546F74F712242E890890070712754DFFAA
:105270009015C0E0F47003A3E0F4703690071EE0D0
:105280009015C0F0A3E4F080298E828F83A3A3122F
:10529000793B60168E828F83A3A3A3E0F583888277
:1052A000A312793BFAA9081240578E828F83127895
:1052B00063FFEE4F70D39015C0E0F47003A3E0F4E9
:1052C000600A9015C0E0FAA9081240571232DD902A
:1052D00007781259E01232D702768574F112242E23
:1052E000890A8C08750900750B00740F122CC712FF
:1052F00061397411122CC7125A078049AE0E12532D
:10530000A7F50CA3E0F50DAE0BEE2EFEE433FFEA9D
:105310002EF582EB1266F2650C7004A3E0650D7049
:1053200019AE09EE2EFEE433FFEC2EF582ED3FF5CB
:1053300083E50CF0A3E50DF00509050EE50EC39518
:105340000840B9050BE50BC3950A5005750E0080A2
:10535000EBA909026D9D74F412242E890B7D007453
:105360000C122CC712613980010DEDC3950B503220
:10537000750A008002050AE50AC39C50ECED25E0A1
:10538000FEE433FFEA2EF582EB3F1253B7F509AE88
:105390000A1253A765087004A3E0650970D7790164
:1053A00080027900026B44EE2EFEE433FFE82EF516
:1053B00082E93FF583E022F583E0F508A3E022745B
:1053C000F612242E12545A7003A3E06D701775085C
:1053D000B37509077808122A21EEFA124183740284
:1053E000122A34801F7508027509807808122A2154
:1053F0008C088D097808122A2112544D1241A77485
:1054000004122A34806974F612242E12545A70033E
:10541000A3E06D70177508C07509077808122A2176
:10542000EEFA1241897402122A34801F750803753E
:1054300009807808122A218C088D097808122A21FF
:1054400012544D1241A77404122A348022125DA80E
:10545000F583E0FD7C801267C6221266FB12787528
:10546000FCE439FD900778E06C227402122A347F44
:10547000020226BD74F612242E74FE122AC8EAFE19
:10548000EBFF851882851983E4F0A3125C3712675D
:1054900012E0FCA3E0FBECFA88828983A3A3E0F985
:1054A000750900750800600574FF6970057508824C
:1054B000803D900778E06A7003A3E06B701AAA1829
:1054C000AB191238A1E9F509851882851983126B89
:1054D0004F701C750883801790099AE0600464017E
:1054E00070057508818008E0640270037508808586
:1054F0001882851983125A07A908EEFAEFFB1241A8
:105500008FE5096011851882851983126B4F60063B
:10551000126E8B123D6902546A74F212242EEAFE56
:10552000EBFF750A00750B0012558B1232DDEA6530
:10553000087003EB650970121238B3E914F50A79A3
:10554000017AE97B071238B98003750B801266EC8B
:10555000F50C780C122A25750CE9750D07780C12DC
:105560002A21780A122A257808122A21E50BF50843
:105570007808122A251265AD1266EFF97A057B804C
:105580001241957407122A340262F51277AE126145
:105590003D88828983127874F508E439F50922740C
:1055A000F612242EE9FE7F0080298A828B83125313
:1055B000B9F8E4C8F9E50828E439F509EF25E0F879
:1055C000E433F9EC28F582ED125DB1EA2402FA50D9
:1055D000010B0FEFC39E40D202546F74E812242EC9
:1055E00074FB122AC88A168B17851882851983E4E2
:1055F000F07403122CC7E4F0A3F004122CC7E4F0FB
:10560000A3F012612A3517125C09F50B850A82F5A1
:1056100083127870FEE439FF850A82850B83A3A389
:10562000E0FA850A82850B83A3A3A3E0F9EAF508D3
:10563000E439F509E50A2404F50A5002050BEEFAEF
:10564000EFFB123379E964016016EEFAEFFB1233D7
:1056500079E9703D900778E06E7003A3E06F6031E8
:10566000126909122A25E4F508F5097808122A2199
:105670007808122A2590077812284575088078083E
:10568000122A251259E61241957407122A3402593A
:10569000D6125A0D8810602B12748A123D6374035F
:1056A000122CC71259E07403122CC7126B4F6013EF
:1056B0007403122CC71259FFA9101240878A0A8B53
:1056C0000B8003751000125A0D880F602712748A20
:1056D000123D637401122CC71259E07401122CC7D9
:1056E000126B4F600F7401122CC71259FFA90F12D1
:1056F00040878003750F00900707805D850A8285CB
:105700000B83A3A3A3A3A3A3A3A3E4F0A3F0AA0AD8
:10571000AB0B851482851583A3A3125A1D12793B06
:10572000F9123CCD851282851383E0C0E085188292
:10573000851983E0F874E928F582E43407F583D00D
:10574000E0126B5304F0E511A2E05007AA12AB136C
:10575000123D69851482851583E0F514A3E0F515E3
:10576000E51445157003025943851482851583A3FA
:10577000A312793B60DD851482851583A3A3A3A3BF
:10578000A3A3A3A3E0A2E050CA851482851583A336
:10579000A3A3A3126B4F851482851583A3A3601F57
:1057A00012793BFA7901851482851583A3A3A3A3FB
:1057B000126DC6124AEE8A128B13751101800F12F8
:1057C0005A1DA3A3E0F512A3E0F513751100E5122D
:1057D00045137003025746851282851383A3E06543
:1057E000087004A3E06509600F74FF650870047415
:1057F000FF65096003025746851282851383A3A3C0
:10580000A3A3A3A3A3122845851282851383A3A370
:10581000A3A3A3A3E0FC7405122CC7126E91A910D8
:105820001240697402122A34E9703C851282851391
:1058300083A3A3A3A3A3A3A3A3A3A3122845851271
:1058400082851383A3A3A3A3A3A3A3A3A3E0FC74B0
:1058500003122CC7126E91A90F1240697402122A0A
:1058600034E97003025746E50F2510C333240AFAC2
:105870007B00123CC18A0A8B0BEA450B700302576E
:10588000248A828B8374D2F0851682851783A3A322
:105890001261398A828B83A3A3E8F0A3E912776BA4
:1058A000A3E51012787CE50FF0E510603CEA2405D2
:1058B000FAE4350BFBE50A240AF8E4350BF98A8291
:1058C0008B831261437403122CC7125A22122A1DB1
:1058D000AC10EC2CFCE433FD8A828B83126E9112A7
:1058E0003C9D7403122A34800D8A828B83A3A3A368
:1058F000A3A3E4F0A3F0E50F70030256FCA810E8A0
:1059000028F8E433F9E50A28F8E50B39F9E8240A20
:10591000FAE439FB850A82850B83A3A3A3A3A3A37F
:10592000A3A31259E07401122CC7125A22122A1D85
:10593000AC0FEC2CFCE433FD123C9D7403122A34B2
:1059400002570E851882851983E0602712690912B3
:105950002A257508E97509077808122A21740312A7
:105960002CC7126912122A2590077812284575084B
:10597000008029EEFAEFFB123379E9702F126909E2
:10598000122A257508E97509077808122A21750871
:10599000007808122A259007781228457808122ADC
:1059A000251259E61241957407122A347403122CF9
:1059B000C7126B4F600B7403122CC7126E91123D0D
:1059C000697401122CC7126B4F600B7401122CC743
:1059D000126E91123D697405122A347F100226BDA1
:1059E000EAF0A3EBF022E5162402FCE43517FDE50E
:1059F0001612653D3517F583E0F97A067B80221291
:105A00005A07AA0AAB0B22E0FCA3E0FD22850A821A
:105A1000850B83E0F8A385820A85830B22126DC66D
:105A2000A322E0F50CA3E0F50D750E00780C2274AE
:105A3000F112242E74F4122AC88A088B09ECFEEDA8
:105A4000FF740B122CC77403F0122AA212479B1288
:105A500032D7EAFCEBFD7403122AA2124795E960E3
:105A60000FEE24131266EF64036010E06401600B14
:105A70008518828519837484025BC18E828F83A30B
:105A8000A3A3A3A3A3A3A3E06018F46015EE2413BB
:105A90001266EF64037016EE24141266EF6003F4CE
:105AA000700B8518828519837482025BC112763966
:105AB000E064217002A3E06003025B988518828590
:105AC0001983748C125C3764036003025B82740177
:105AD000122AAA1262DD124A47E96003025B8212AF
:105AE0003FEB8A0A8B0BEA450B7003025BC28E0CFC
:105AF0008F0D750E00780C122A1D7C157D00123C4E
:105B00009D7403122A34850882850983A3A3E50ABC
:105B10002415FCE4350BFD7409122962127298C039
:105B2000E0E50A241EF582E4350BF583D0E012612E
:105B300049C0E0E50A241FF582E4350BF583D0E087
:105B4000F0E50A2420F582E4350BF5837405F0EEC8
:105B5000240BFE50010FFAEFFB12395B7D007C0035
:105B60007900EEFAEFFB12414D9080A41228417AA1
:105B7000007B109007AAE0F9123E297404122A341F
:105B80008078125BFF122A25125C11124A7174018F
:105B9000122A34E9702C8014125BFF122A25125C41
:105BA00011124A6B7401122A34E9700D851882852E
:105BB0001983E4F0123FBB8009851882851983742C
:105BC00088F0127298F50A780A122A257401122AAE
:105BD0009A880A890B780A122A21E508240CF58292
:105BE000E43509125C094480F50B780A122A211267
:105BF000666F1241417405122A34740C026D9AEEDC
:105C00001262EAE0F50A780A22F583E0F50AA3E0D9
:105C100022EE240BFCE43FFD8E828F83A3A3A3A37B
:105C2000A3A3A3A3A3126ECE8E828F83A3A3A3A349
:105C3000A3A3A3A3E0F922F01277AEE022C082C0B2
:105C40008374F3122AC8851882851983E4F004123C
:105C50002CC71259E07403122CC7AA82AB83122EF0
:105C600057AA18AB19122E93740D122A34026E80A3
:105C700074F612242E1266F7FAA3E0F9EAF89007F8
:105C8000BBE058F508A3E059F509E5084509601C93
:105C90007808122A219007781228451266ECFD7CBC
:105CA000001267C21241A17404122A3402546F74A4
:105CB000F412242E74FF122AC8EAFEEBFF85188224
:105CC000851983E4F090098EE06021EE240B1266C2
:105CD000EF640160178E828F83A3A3126139EE24D3
:105CE000151266EF687003A3E0696003025DA312FA
:105CF000659D126137E8FAE9FB88828983A3A3A333
:105D0000A3A3A3A3A3E0FC88828983A3A3A3A3A343
:105D1000A3A3A3127815EC28F508E439F509EC459E
:105D2000096010EC9471E99408500890099AE064B5
:105D300002700A85188285198374808038122ECFEC
:105D40008A0A8B0BA80AA90BE849602188828983FB
:105D5000A3A3A3A3E06016C394035011E824121276
:105D60005DAEE82414125DAE123FBB800985188237
:105D70008519837481F0125DA8126910122A2574A6
:105D800001122A9A880889097808122A2175081FA1
:105D90007509807808122A211265A3124141740501
:105DA000122A347401026B41EE1276603F22F582B2
:105DB000E439F583E508F0A3E509F02274EA12243A
:105DC0002E74DB122AC88A148B1575120075130005
:105DD000127933F50EAC18AD197A007B00799C125C
:105DE0002FB37A047900122EA5EAF50C8518828566
:105DF0001983E02AF0F8E50EC3984003025FDBE068
:105E0000C3950EF509C394044003750903E50975AC
:105E1000F01AA4FAABF0123D638A128B13EA451311
:105E20007003025FDE750D00AE12AF13850E0880A1
:105E30007E126046123CA9850A82850B83A3A3A328
:105E4000A3E0702D850A82850B83126B4F700C12B4
:105E50006FDBF0EE2418126FDE8010126054F090A9
:105E60000567E014C0E012602ED0E012607FE4808D
:105E700034900567E004C0E012602ED0E012607735
:105E8000C39403EE4003025F421262E674021260A2
:105E90007764017003025F4FEE2415126057F0EE35
:105EA0002416126057F0EE241AFE50010F050DE57E
:105EB0000DC395094003025F7AE508C3950C4003C2
:105EC000025F5885080AAA0A7B00122F178A0A8BDC
:105ED0000B050890055412606012479B850A828565
:105EE0000B8312613912603CE8F0A3E912609185DE
:105EF0000A82850B83A3A3A3A3A3A3A3A3A3A3E0C5
:105F0000C0E0126024D0E0F07401122CC7E4F085E8
:105F10000A82850B831261397402122CC712614305
:105F20007401122AA2122E81E964016003025E311B
:105F30007404122CC7AC82AD8312604C12479B02D2
:105F40005E3712605512607764036003025E98EE5C
:105F50002415126FDE025E9EE50CC3950E4005759A
:105F60000800801DE50EC3950CF5088014126054DE
:105F7000F0EE241AFE50010F050DE50DC3950950F2
:105F80005D740E122AAA85080AAA0A7B0079871274
:105F90002FB305087418122CC712606012479B12A9
:105FA0006046123CA9EE2412F8E43FF9740E122C5C
:105FB000C7126E9188828983EAF0A3EB12607F7426
:105FC00003126091741D122CC7E0C0E0126024D04F
:105FD000E0126DF87097126FDB8095750900750AF5
:105FE00000780A122A257812122A217809122A2505
:105FF000E50EF5097809122A257405122CC7E0FD73
:106000007C001265291241DD7405122A34E512451F
:10601000136007AA12AB13123D697425122A347F4C
:106020000E0226BDEE2419F582E43FF583221260AC
:106030003222EE2418F582E43FF58322EE2412F595
:1060400082E43FF583227C087D0079FFEE240AFA82
:10605000E43FFB22EE2414F582E43FF58374012231
:1060600012613D8E828F83E8F0A3E9F07C687D05A4
:10607000EE1267DD3FFB221277D0A3A3A3E022F04C
:10608000EE126FD27402F0EE2416F582E43FF5832F
:1060900022F0EE2417F582E43FF5837402F01260DB
:1060A0003274FFF02274F612242E74F9122AC88A70
:1060B000088B0912612A35091278FD123CB5EAF8FD
:1060C000EBF9ECFAEDFB851882851983122CB0EE02
:1060D0002404FE50010F8E828F83E0C0E07404120E
:1060E0002CC7D0E0126DCFFA7405122CC77401F0E2
:1060F0007406122CC77401F0900782F090078B048D
:106100001277E7A3126139900783126143EA90077F
:106110008C126149900781F0AA18AB19122F53E92C
:106120006003122F59740702546CEA12612F221275
:10613000670C2212753639F58312613D22E0F8A30F
:10614000E0F922E8F0A3E9F022F0127745E02274AA
:10615000F212242E74FF122AC87508007E007F00F8
:106160001232058A0A8B0B1232058A0C8B0DA80C91
:10617000A90D80050508126133E84970F790099A66
:10618000E060076401600302625A1232058A0C8BD8
:106190000DA80CA90D8003126133E849603688828E
:1061A0008983126E91900554E06A7003A3E06B60DE
:1061B0000D12753639F583126E91EA4B70D98882CB
:1061C0008983126139900554E0687003A3E0697017
:1061D0000302625A7A167B00123D638A0C8B0DAE65
:1061E0000CAF0DEE4F60739005541261398E828FA3
:1061F00083126143900549E08E828F83A3A3F0123E
:106200003361E98E828F83A3A3A3A3A3F09015D457
:106210001277C4F07C687D051262DD12479BAA18D4
:10622000AB197941124867851882851983E06008A7
:10623000900778126139800478FE79FF8E828F830F
:10624000A3A3A3A3A3A3A31261431262E5E50AF0EB
:10625000A3E50BF08E0A8F0B050890078CE0F8E59C
:1062600008C39850047A008022E508C398FAC394C2
:106270000640027A057900800DE50A127537350B64
:10628000125C09F50B09E9C39840EE75090078091D
:10629000122A25780A122A21EAF5097809122A25F4
:1062A00090078CE0F5097809122A25AD087C007A60
:1062B000837B07900781E0F91241D77405122A34D5
:1062C00090099AE060046401700BEE4F6007EEFAEB
:1062D000EFFB123D69122F597401025585EE240B14
:1062E000FAE43FFB22EE1262EA221275373FF58391
:1062F00022EEFAEFFB7F060226BD74EC12242E7408
:10630000FF122AC88A0A8B0B7E008E0E8E0F126136
:106310002A350B127939FFAC18AD197A007B007958
:106320009D122FB3851882851983E0F8EFC398403A
:10633000030263D5E0C39FFEC3940B40027E0AEEC6
:1063400075F007A4FAABF0123D638A088B098A0E38
:106350008B0FEA450F607C750C00801A85088285DA
:106360000983A3A3A3A3A37403F0E5082407F508F6
:1063700050020509050CE50CC39E5059AC08AD0947
:10638000850C10E5102FFAE43400FB798B122FB343
:10639000850882850983A3A3A3A3A3E0146008143E
:1063A000601314601F80B5850882850983A3A3A3A9
:1063B000A3A3E480B4850882850983A3A3A3A3A330
:1063C000740180A5850882850983A3A3A3A3A37470
:1063D0000280967E007508007808122A25780E1231
:1063E0002A21EEF5087808122A25EFF50878081218
:1063F0002A257405122CC7E0FD7C00E50A1267DD32
:10640000350BFBE50A12653D350BF583E0F91241CA
:10641000E37405122A34E50E450F6007AA0EAB0F90
:10642000123D697401122A347F0C0226BD74EA12EF
:10643000242E74FE122AC88A148B15750A00750B57
:1064400000127933F508AC18AD197A007B0079A3F6
:10645000124A5F85080C851882851983126139C339
:10646000E50C98E499507D851882851983E0C395E1
:106470000CFEA3E09400FFC3EE9404EF94004006EA
:106480007E037F008004EE4F605AEEFAEFFBEA7560
:10649000F015A4FAA8F075F015EBA428FB123D63E3
:1064A0008A0C8B0D8A0A8B0BEA450B603775090045
:1064B000750E00850E10C3E5109EE49F502BAC0CAA
:1064C000AD0D850E12850810E5122510FAE4340092
:1064D000FB79A2124A5FE50C2415F50C5002050D5C
:1064E000050E80CF75098B7E00750C00780C122A82
:1064F00025780A122A21EEF50C780C122A25780844
:10650000122A257405122CC7E0FDAC091265291268
:1065100041E97405122A34E50A450B6007AA0AAB63
:106520000B123D69740202601CE5141267DD35151B
:10653000FBE51412653D3515F583E0F922240FF5CE
:1065400082E42274F612242E74FF122AC8EAFEEBAB
:10655000FF12659D12767DA3A3A3A3A3A3A3A3E02B
:10656000F9122F77E9851882851983F0750800786C
:1065700008122A257401122A9A88088909780812B3
:106580002A217508357509807808122A211265A319
:106590001241417405122A34740102546CEE1261E6
:1065A0002F3F2279011265ADFAE43FFB22EE24026F
:1065B000FCE43FFDEE240F2274F412242E74FA1230
:1065C0002AC88A088B09EA12753D12754DFFEEFA4A
:1065D000EFFB122E5DE960131232D7EAFCEBFDEE01
:1065E000FAEFFB124795E96401700A7401122CC797
:1065F000E4F0A380097401122CC7EEF0A3EF127827
:1066000003A3A3A3A3A3E0F8A2E650087403122CEB
:10661000C77401F0E8A2E750087404122CC7740193
:10662000F07405122CC7E4F004122AA2122FA7E975
:10663000851882851983F07A007B001232FB750A77
:1066400000780A122A257401122A9A880A890B787E
:106650000A122A21750A34750B80780A122A21122F
:10666000666F1241417405122A347406026B417937
:1066700001E5082402FCE43509FDE508240FFAE4ED
:106680003509FB2274F612242E74FF122AC81266F2
:10669000F7F509A3E0F508A909122F65E985188225
:1066A000851983F090099AE0700B740165087005F4
:1066B000A9091242A3EE240B1266EF702C75080094
:1066C0007808122A257401122A9A880889097808FC
:1066D000122A217508367509807808122A21126558
:1066E000A31241417405122A34026598EE240EF576
:1066F00082E43FF583E0221266FB22EAFEEBFF1202
:10670000670B3FF583E0126712E022EE2413F58257
:10671000E422F8A3E0F98882898322C082C08390B2
:10672000099AE070031242A9026E8074F412242EBA
:1067300074EF122AC8EAFEEBFF12558B900778E03F
:1067400065087004A3E065097052A818A919880AA1
:10675000890B780A122A21750A11750B00780A1222
:106760002A217C007D007A817B00123DED740412A9
:106770002A34E97027750A00780A122A2574011252
:106780002A9A880A890B780A122A21AC08AD0912C4
:1067900067C212419B7403122A348021750A117555
:1067A0000B80780A122A217808122A211266ECFD41
:1067B0007C841267C21241A77404122A3474110235
:1067C0006B411267C622EE1267DD3FFBEE240FF528
:1067D00082E43FF583E0F922FCEFFDE5082402FAAC
:1067E000E42274F112242E74EB122AC81266F7FC0C
:1067F000A3E0FAE4CAFBEC2AF508E43BF5099007AC
:1068000078E065087004A3E0650960030268B18858
:10681000828983A3A3E09410500F88828983A3A365
:10682000E08518828519838008851882851983740C
:1068300010F0E0C0E07404122CC7D0E012766EA312
:10684000A3A982AA83890C8A0D750E00780C122ADE
:106850001D7407122CC7E0FC7D007408122CC7AA17
:1068600082AB83123C9D7403122A347404122A9A58
:10687000880A890B780A122A21750A11750B00788B
:106880000A122A217C007D007A817B00123DE77488
:1068900004122A347404122CC7E09007B36005E098
:1068A000D2E48003E0C2E4F0851882851983E48095
:1068B000088518828519837484F0E0C0E0740112A1
:1068C0002CC7D0E0F07402122CC7E508F074031254
:1068D0002CC7E508F0125DA8126910122A2574026F
:1068E000122A9A880889097808122A2175081475CD
:1068F00009807808122A2179031265A51241417492
:1069000005122A347415026D9AE516127660351751
:10691000F583E0F50878082274F412242E74E0124E
:106920002AC88A088B09AC18AD1912412F90099A10
:10693000E0640270337402122CC7AE82AF8312324D
:10694000D7EEFCEFFD124795E9601D1232DD8A0A91
:106950008B0BA80AA90B851882851983E068700340
:10696000A3E0697003026B3F1234937402122CC7C8
:10697000126E871233A9E964017003026B3F741829
:10698000122AA21232E97402122CC7AC82AD8374AF
:1069900018122AA2124795E960321232E38A0A8B52
:1069A0000BA80AA90B851882851983E0687003A3D8
:1069B000E069601885188285198312613990054A4B
:1069C0001261437A4A7B05794B12486D90099AE02F
:1069D000600764016003026A7D12745CC082C08338
:1069E0001232DD8A088B09D083D082E065087004FA
:1069F000A3E06509605C7402122CC7AA82AB831203
:106A00002ECF8A088B09A808A909E8496026888240
:106A10008983A3A3A3A3E06401600D88828983A373
:106A2000A3A3A3E06402700C7402122CC7AA82AB69
:106A300083122EDB9005E8126B4F601690098EE0F2
:106A40006401700E126E8B9005E9E0F58388821266
:106A50004AEE1232DD8A088B09A808A90985188236
:106A6000851983E0687003A3E06960117402122C39
:106A7000C7126E87122EB1E96003123FBB74021277
:106A80002CC7126E871234817900126E8B1230F788
:106A9000740B122CC7E4126B53F8A3E0F9740C12B8
:106AA0002CC7126143740B122AA2122E81E9603F97
:106AB0007C087D0079007418122AA2123CA9740E79
:106AC000122CC7AC82AD837418122AA2124795E922
:106AD000601D7402122CC7AC82AD83740E122CC7D9
:106AE000AA82AB83122E57740B122AA2122E937411
:106AF00002122CC7AC82AD83740E122CC7AA82ABD3
:106B000083122E57740B122AA2122E87E96030745A
:106B10000C122CC7126139851882851983E06870C0
:106B200003A3E0696019851882851983126139749D
:106B30000C122CC7126143740B122AA2122E9374EA
:106B400020122A347F040226BDF582E438F5831230
:106B5000701222F0851882851983E02274F11224C4
:106B60002E74F6122AC8EAFEEBFF75080090081F83
:106B7000126B4F70507A377B00123D6390081FEA0A
:106B8000F0A3EB12734760197C377D007900123C4B
:106B9000A9EEFCEFFD90081F126E911240FFE97004
:106BA0000B8518828519837488026D031276411251
:106BB0006DA27401F07C0B7D419004D3126E911292
:106BC0004ACB026D98E0C8126DA27402F0EEFCEFA1
:106BD000FD12729D1240FFE9700C851882851983A1
:106BE0007488F0750801750AE9750B07780A122A8E
:106BF00021126EA11228451276412428127290FCAF
:106C0000126ED41276412414127290F912406374F9
:106C100004122A34126DAF126DD5243112729060B5
:106C200043127331FAE433FB123D6390081FE024F2
:106C300032126DEA6022750CE9750D07750E007849
:106C40000C122A1D127331FCE433FD126EBF123C8C
:106C50009D7403122A34800C8518828519837488E8
:106C6000F0750801780A122A21126E951228451231
:106C700076412411127290FC126EB6127641242BCA
:106C8000127290F91240637404122A34127641246D
:106C900034126DD524341272906035127328FAE4E0
:106CA00033FB123D6390081FE02435126DEA604209
:106CB000750CE9750D07750E00780C122A1D1273FC
:106CC00028FCE433FD126EAD123C9D7403122A348D
:106CD000E508A2E04025126DAF127290700890088E
:106CE0001F1272F460157B007A00790012410502D0
:106CF0006D988518828519837488F08518828519A6
:106D0000837486F07409122CC774021274A0126D79
:106D1000BE122CC7E8F0A3E9126DCFF5087808126F
:106D20002A257401122A9A880889097808122A21CA
:106D30007508207509807808122A217901740612D5
:106D40002AAAEEFAEFFB1241417405122A3412729C
:106D5000E370427409122CC77402F0126DB8122C41
:106D6000C712734E122A257401122A9A88088909BB
:106D70007808122A217508207509807808122A21BE
:106D800079017406122AAA90081F126E91124141CD
:106D90007405122A341240F9740A122A347F070249
:106DA00026BD126DA622242EF582E438F5832290AA
:106DB000081F1272B924312290081F126DC6A3A3B6
:106DC00012613D740122E0F8A3E0F583888222126B
:106DD00074A0A3E022F582E438F583126DE0C822A6
:106DE000E9F090081FE0F8A3E022F8A3E03400F9EE
:106DF00088828983EAF0A3EB12767712701222C0A0
:106E000082C08390081F126B4F6075E0C824351252
:106E10006B496006126EAD123D6912764124321242
:106E20006B496006126EBF123D6912764124121240
:106E30006B496009126E95126E91123D691276418E
:106E40002415126B496006126ED4123D6912764108
:106E50002429126B496009126EA1126E91123D69CC
:106E6000127641242C126B496006126EB6123D69EF
:106E700090081F126E91123D6990081FE4F0A3F074
:106E8000D083D0820229E6AC82AD83851882851931
:106E900083126ECE221272B62412F582E438F58384
:106EA000221272B62429F582E438F583221272B6D2
:106EB0002435126EC8221272B6242C126EC8221209
:106EC00072B62432126EC822F582E438F583E0FAF5
:106ED000A3E0FB221272B62415126EC82274F112BE
:106EE000242EEAFEEBFF8C088D09750A018C0C8DAF
:106EF0000D750E00780C122A1D7C177D00123C9D2A
:106F00007403122A34EE2412126FDEF0A3F0EE2482
:106F100015126FDEF0A3F012745CE0603AEE2412FA
:106F2000F8E43FF9880C890D127485123D63126FE5
:106F3000FF6021E5082412126FF2122A1DE50824D1
:106F400011126FE612603D126E91123C9D74031295
:106F50002A348003750A00E50812746A6035EE244D
:106F600015F8E43FF9880C890D127485123D6312FF
:106F70006FFF6055E5082415126FF2122A1DE5080F
:106F80002414126FE6126FCE126E91123C9D7403A0
:106F9000122A34E50AA2E0402BEE2412F582E43FE7
:106FA000126B4D600912603C126E91123D69EE2425
:106FB00015F582E43F126B4D600AEE126FCE126E31
:106FC00091123D69A90A026D9D750A0080CB126F6E
:106FD000D2222415F582E43FF58322EE2414F582B3
:106FE000E43FF583E422127631E025E0FCE433FD52
:106FF000EE22127631E0F50CA3E0F50D780C228537
:107000000C82850D831259E0850C82850D831270E8
:107010001222E0F8A3E0F9E8492274EE12242E745B
:10702000ED122AC8890A8A0E8B0F750C00750D00A7
:10703000750BFF7510FF7511FF7508007509008548
:107040001882851983E412734760177403650A6018
:10705000067402650A7010E0C82430127290650F41
:10706000600579000272867C0B7D417A007B0012FC
:107070004ACB7401650A700A851882851983748564
:10708000803DE50A60067403650A701990081F12B6
:1070900072C3F07403650A7029E50E6029851882B1
:1070A000851983801A7402650A701BE50E90081F0B
:1070B00070051272C380081276441272DA7402F0FC
:1070C0008004E50A601E1272C970191272ED600523
:1070D000126DB2800A1272F4600A127641243412E0
:1070E000729014F01272ED60221253B9F509127306
:1070F00031F8E433F990081FE0FAA3E0CA24321211
:107100007305241D1272AA2425802E1272F4602E9B
:1071100090081FE02417F508A3E03400F509127366
:1071200028F8E433F990081FE0FAA3E0CA243512E6
:10713000730524061272AA240E127290F50B7409BC
:10714000122CC77402126B5360030271F4E50845F8
:107150000970030271F41272C970047E2280027EEB
:1071600021850882850983126DBE122CC7126143E6
:10717000900823E0C0E01276412430F582E438F52F
:1071800083D0E0F07412122CC77403F0AC0CAD0D78
:10719000740A122AA212479B850882850983A3E0FC
:1071A000F50C780C122A25780B122A25740C122A59
:1071B0009A880C890D780C122A217810122A21E560
:1071C000082406F50CE43509F50D780C122A211275
:1071D0007298F97409122AAAEEFA7B001241B3746C
:1071E00008122A347C0B7D419004D3126E91124A0E
:1071F000CB027284126DB8122CC712734E122A255C
:107200007401122A9A880889097808122A217508B7
:10721000207509807808122A2179017406122AAA99
:1072200090081F126E911241417405122A34127295
:10723000E3704E1276412419F582E438F583126D1D
:10724000C0122CC7E8F0A3126DDB2418F582E438D5
:10725000126910122A257401122A9A88088909785D
:1072600008122A217508207509807808122A2179C8
:10727000017406122AAA12729D1241417405122A43
:10728000341240F979017413122A347F0A0226BDA0
:10729000F582E438F583E022127755E02290081F4A
:1072A000E02417FAA3E03400FB22F50CA3E034003D
:1072B000F50D1272B62290081F1272BD22E0F8A3DB
:1072C000E0C8221272D374012290081F1272D3E018
:1072D0006401221272BD1272DA22242FF582E43880
:1072E000F583221272B6126DA6E064022212733781
:1072F00090081F221272F8221272BD2434F582E423
:1073000038F583E022F582E43AF583E028F8A3E03B
:1073100039F9E824FEF582E934FFF583E0F510A39E
:10732000E0F51190081FE02290081F1272F825E086
:107330002212733725E02290081F1272BD2431F506
:1073400082E438F583E022126DE1F9E84922E8F0A1
:10735000A3126DE0F5838882A3E0F508780822C0C7
:1073600082C0837B007A857901124105026E8074A8
:10737000F412242E8C088D09EA240F127809127752
:107380005F1261398C828D83A3A3126143EA240EBC
:10739000127809A3F01275441274911276535001B9
:1073A0000FFCEFFDE5082406FAE43509FB12479BC4
:1073B000EE2408FE50010F8E828F83E0C0E012772A
:1073C00051D0E0127552F8127741E8127657500109
:1073D0000FE5082412127464A3F0E5082415127452
:1073E0006412749AA30EAF83C0E012745CD0E0F014
:1073F0006028E508241212747C123D6312781C6028
:1074000019E508241212746F12745EE0F9124087B5
:107410008A0A8B0BAE0AAF0B8007E50824111274A1
:10742000648E828F83E0A3AE82AF83C0E0127528A2
:10743000D0E0F0601FE508241512747C123D631241
:10744000781C6010E508241512746F12746AF91222
:1074500040878005127528E4F0026B44E50824118A
:1074600012763122127631E4F02212752EE02212C9
:107470007631125A07EEFAEFFBE50822F8E43509F7
:10748000F9880A890BE012748A2225E0FAE433FBBA
:1074900022FF1277B98C828D8322A31274A0E0227E
:1074A000F08E828F832274F612242E8C088D09129E
:1074B0007544FFEEFCEFFDAA08AB0912479BEE24D2
:1074C00008FE50010F8E828F8312786A12755285E2
:1074D0000882850983A3A3A3A3A312765350010FA7
:1074E0008E828F83E0F8E50812753DE812764874C5
:1074F00003687026EEFCEFFDE508240BFAE435097D
:10750000FB12479B8E828F83A3A3A3A3A3A3A3A352
:10751000E0C0E0127528D0E0800A12773512762B91
:10752000E8F0A3E9F002546FE50812752E221275F7
:10753000373509F58322E82414F582E42212612FFD
:10754000127634221277E112754B22F583E0FEA306
:10755000E0221277801277BD2274F212242EEAFE06
:10756000EBFF750A00EE24101266EFC3940C400D79
:107570001277AA127644240B127290F50AA80AE830
:1075800028F8E433F9E8240DFAE439FB123D638A64
:10759000088B09EA4509700302762212659D12776D
:1075A000998A828B8312777C7078EEFCEFFDEA2457
:1075B00003FAE43509FB12479BEE2408FE50010F45
:1075C0008E828F831277B58508828509831276565D
:1075D00050010F127629E4F0E50A6046E508240D13
:1075E000F8E43509F98E828F83E0C0E0127629D065
:1075F000E012773CC0E0127639D0E0127648850A76
:107600000B8E828F83E0FCA3E0FBEC8882898312DF
:107610007666500109EE2402FE50010F150BE50BB2
:1076200070DFAA08AB090262F5E508240B12763177
:1076300022F582E43509F58322E508240C1276311F
:107640002290081F1272B92212764C221277880EED
:10765000AF8322A3A3A3A3F0A3E9F0EE2402FE22AA
:10766000240EF582E4221259E1E82402F82212766F
:107670007222127677A322F08882898322126ECC3E
:107680008A828B83227F010226BD74F212242E127D
:1076900077DD1253B7850882F583E0F50DA3858267
:1076A00008858309A3A3E0F50C1277943400FB123C
:1076B0003D638A0A8B0BAE0AAF0BEE4F60378E82AA
:1076C0008F83E50DF0850882850983E0FA1277F053
:1076D000850882850983A3A3A3A982AA8389088A2E
:1076E00009880A7808122A1D12778F3FFB123C9DE9
:1076F0007403122A340262F174F712242EEA24135E
:10770000F8E43BF988828983E0FAA3E0F5838A8272
:1077100012780F127730126712A3E0FA88828983F9
:10772000A3A3E0F9EA8C828D83A3126144027685DB
:10773000127677E0221277BDF8E5082212764CE047
:107740002212774522E508240FF582E43509F583F6
:107750002212775522E5081276603509F583221248
:107760007764A322F08A828B83A32212776F22F0A0
:107770008A828B83A3A3A322A3A3A3A3127780222D
:10778000127788AE82AF8322F08E828F83A322ACE1
:107790000C7D00EE2404FAE42212779D22F583E0AA
:1077A000FEA3E0FF8E828F83E0221277AE22126763
:1077B0000B3FF583221277BD228E828F83E0FAA3DE
:1077C000E0F9EA22E08E828F83A3A3A3A3A3A322DE
:1077D000F0850A82850B83A3228C088D091277E13C
:1077E00022EA12670C3B22F0850882850983A322D6
:1077F000127815EA8E828F83A3F0A3E9127803E54D
:107800000CF022127788A3A322F582E43BF583E0F3
:107810008C828D8322A3E0F8E4C8F922850A828550
:107820000B831259E0850A82850B83127012227431
:10783000F612242E1277D9F58312786312749112FE
:10784000765750010F1267D83509FB12479B8E827D
:107850008F83A3A3A3A3A3A3A3A312786AA3A3F0D4
:1078600002546F12613DE8FEE922127910A3A322AF
:1078700012787422E0FA127815EA282212776FA3A0
:10788000A3A3A32274F612242E1277D91278FD1224
:107890003CB5EAF8EBF9ECFAEDFB85088285098343
:1078A000122CB0EE2404FE50010F8E828F83E085EF
:1078B0000882850983127778C394065005127915DA
:1078C0008037850882850983A3A3A3A3E064FE60B3
:1078D0000E850882850983A3A3A3A3E0F4701B127D
:1078E0007908127648850882850983A3A3A3A3E0BB
:1078F000F47007127922F0A3E9F002546F12754B6D
:10790000FF7904EEFAEFFB228E828F831279102228
:10791000127915A322E0850882850983A3A3A3A376
:10792000A3221277B9850882850983A3A3A3A3A301
:10793000A3A322EA12612F3515F583126DC6E0224A
:1079400074F712242EEAFEEBFF7409122CC7E0F93B
:10795000A3127AD88E828F83800C122A4FF0E924EA
:107960000109E43AFAA312797270EFAA82AB83029A
:107970007B73ECFEEDFFEE24FF1CEF34FFFDEE4FBA
:107980002274ED12242E89088A098B0A7413122C92
:10799000C7E0F50CA3E0F50DA3E0F50EECF8EDF96A
:1079A000E824FF1CE934FFFDE8496037A908AA096B
:1079B000AB0AE92401F508E43AF509850C10850DB8
:1079C00011850E12E50C2401F50CE4350DF50D12B0
:1079D0002A4FF8A910AA11AB12122A4F6860BD797C
:1079E00000800279017F0B0226BD74F612242EE975
:1079F000FE8C088D097808122A218E08AC087D00BB
:107A00001249637402122A34027D4EC082C0838AF6
:107A1000828B83E0FCA3E0F8E4C8F9EC28FAE439AF
:107A2000FB027B5A74F012242EE9FE74026E700978
:107A30008A828B83127ABC804F74036E70168A829E
:107A40008B83127AB61229C17808790C122B921204
:107A50007AA7803474046E8A828B837041127AB65E
:107A60001229C17808790C122B92127AA7780C127D
:107A700029C17808790C122B928A828B83A3A3A345
:107A8000E0F50CE4F50E7418780C1229C178087929
:107A90000C122B92AA08AB09AC0AAD0B8006E0FAD7
:107AA000E4FBFCFD027F528A828B83A3A3E0F50CEA
:107AB000E4F50D741022127ABC780C22E0F508E48B
:107AC000F509F50AF50BA3E0F50CE4F50DF50EF557
:107AD0000F74082288828983E0FAA3E0FB22C08227
:107AE000C083123E77807374F612242EEAFEEBFFF9
:107AF000EE4F603DEE2405FAE43FFB123D638A0839
:107B00008B09A808A909E849602788828983E4F0DD
:107B1000A3F088828983A3A3EEF0A3EFF088828983
:107B200083A3A3A3A374FFF0E82405FAE439FB8040
:107B3000047A007B00027D4EC082C083EA4B700451
:107B400079058016127BD660047904800DEA24FB47
:107B5000FAEB34FFFB123D697900D083D082022911
:107B6000E674F712242E7C00123CD38006F0EEA2BD
:107B7000E092AF7F010226BD74F712242EE9FEECDD
:107B8000FFEA4B602190811CE0F8EEC39840071299
:107B90003CC77903803E127DE4127CF37005127BB2
:107BA000D66007123CC77905802AEEF074016F7029
:107BB0000DEAFCEBFD7A2D7B07123CF1800BEAFC11
:107BC000EBFD7A2D7B07123CE57A007B80EEF91203
:107BD0003D037900809D127D57E0F42274F2122457
:107BE0002E890A750C00750D007E007F00A2AFE49F
:107BF00033F50BC2AF90072D8015EE4F7006850848
:107C00000C85090DE50824FBF582E509127DEAE003
:107C1000F508A3E0F509E50845096023E50824FF18
:107C2000F582E509127DEAE0650A70CEEE4F700636
:107C3000AE08AF0980CE7A007B80123D03800B7ABC
:107C4000007B80123D09EE4F6015780C122A21EE60
:107C5000FCEFFD7A2D7B07123CF77402122A34E503
:107C60000BA2E092AFEEFAEFFB7F060226BDC082C8
:107C7000C083EAF8A2AFE433FCC2AF90072D8003C3
:107C8000127DE4127CD4600F127D53E06970F18A9A
:107C9000828B83E06870E9ECA2E092AF027B5A74B9
:107CA000F712242EA2AFE433FEC2AF127DEE127C97
:107CB000EF70098A828B83800E127CDC127CCE707E
:107CC000F8127CE8127DEAECF0A3ED027B6D127CE9
:107CD000E8127E03E0FAA3E0FBEA4B22127CE812F2
:107CE0007E03E0F8A3E0F922E824FBF582E9228A8A
:107CF000828B83E0F8A3E0F9E8492274F612242E7F
:107D0000EAF8EBF97A007B00A2AFE433F508C2AFE2
:107D100088828983E0FCA3E0FDEC4D602B127AD4CD
:107D2000EA24FBFCEB34FFFD8C828D83E0FEA3E0B4
:107D3000FF88828983EEF0A3EFF08C828D83E4F0DC
:107D4000A3F0127D5374FFF0E508A2E092AF7F022A
:107D50000226BD127D5722EA24FFF582EB127E0334
:107D60002274F712242EE5A8FEC2AF8A828B8312FA
:107D70007CE2127D8E127DEAE8F0A3E9F08A828B24
:107D800083ECF0A3EDF0EEA2E7A2E7027B71EC2416
:107D9000FBF582ED2274F712242EA2AFE433FEC26B
:107DA000AF8A828B83127CE2EC687002ED69700C02
:107DB000127D8E127CDF8A828B838018127D8E1258
:107DC0007CDF7409122CC7E0FAA3E0CA24FBF58219
:107DD000EA127DEAE8F0A3E9F0127DEE127DF97473
:107DE000FF027B6DEA24FBF582EB127E0322EC247A
:107DF000FB127E00E4F0A3F022EC24FF127E0022AE
:107E0000F582ED34FFF5832274F712242EE9FE7F0C
:107E100000A2AFE433F508C2AF127CEF700C8A8287
:107E20008B838015EE6018127CDC1E127CCE70F401
:107E3000EE600C127CE8127DEAECF0A3EDF00FE5A9
:107E400008A2E092AFEFF9027B7374F712242EE9D7
:107E5000FD90811CE0F8EDC398502AE5A8FEC2AF62
:107E6000ED29F8E433F990076EE028FCA3E0398CA3
:107E700082F583E04AF0A3E04BF0EEA2E7A2E7929E
:107E8000AF790080027903027B7374F712242EE924
:107E9000FE90811CE0F8EEC3985022E5A8FFC2AF27
:107EA000EAF4FCEBF4FDEE29127F05E05CF0A3E0C0
:107EB0005DF0EFA2E7A2E792AF79008002790302BA
:107EC0007B73E9F874FF687006D2AF79008002799D
:107ED000070229E6E9F874FF687006C2AF790080EE
:107EE0000279070229E6C082C083123D5790072D10
:107EF000E4F0A3F0123E11123DF9123E53123D5D23
:107F00007900027B5AF8E433F990076EE028FAA36F
:107F1000E0398A82F5832274F012242E7410122C18
:107F2000C7780C122C708A828B83E50C127F7685C1
:107F30000C08850E0A850F0B74107808122A69E563
:107F400008F0A37418780C122A69E50CF0A3AA8231
:107F5000AB837F080226BD74F012242E7410122CFD
:107F6000C7780C122C70850C088A828B83E5081266
:107F70007F76741080CFF0A3850D09E509F0A32268
:107F800074F612242EE9FDEA4B6016780080010891
:107F9000E8C39C5010EA28F582E43BF583E06D606D
:107FA000EE790080027901027D4EC082C08385187F
:107FB00082851983E0F8A3E0F9E84960128A828B90
:107FC00083ECF0A3E824FF18E934FFF94870F2D0FD
:107FD00083D0820229E6C082C0839009C7E0F9D02D
:107FE00083D0820229E60229E60229E60229E60276
:107FF00029E6FFFFFFFFFFFF851A87000229E6FF42
:10800000EB4833378131D74A4F2D893E1540074819
:10801000E947E1430000000000000000000000000C
:108020000000000000000000000000000000000050
:108030000000000000000000000000000000000040
:108040000000FFFFFFFFFFFFFFFF0008000400022A
:108050000001FFFFFFFFFFFFFFFF00000000000027
:108060000000FFFFFFFFFFFFFFFF02050200080106
:108070007482003A003B0000000000000000000095
:1080800000000002000206020400000019E0FCFFEC
:10809000000000FFE71F030080510100FA0000000C
:1080A000100E0000E803000030000000F8FF0000A0
:1080B0000943388664000000E20400005802000012
:1080C000BC0200003200000000F8FF0760EA000078
:1080D0000000000002000000E90300000B000000A7
:1080E000010000000A0000003C000000FEFFFFFF4E
:1080F0001F00000008000000975118006AAEE7FF5B
:10810000965118009F020000E9FFFFFF0000FF00EA
:10811000FFFFFFFF00000000000000000A74F712DC
:10812000242EE99005A1F0900556E4F012477190D5
:1081300005B5E4F0A3F09005A2F0A3F01234399055
:10814000099AE0600464017006122E9F12306112D9
:108150004777900517E4F0A3F01248A902B15774CD
:10816000F012242EEAFEEBFF548060689005A1E037
:10817000F9123CD98A088B09EA4509604F7C0080D6
:10818000010CEC75F003A4F8A9F0749828F582743A
:108190004F39F583E493F4602CE493F88508828BDF
:1081A00083E06870DCAA08EC75F003A4F8749928E1
:1081B000F582744F39F583E493C0E0740193F5833D
:1081C000D082124AEEAA08AB09123CC7EEFAEF645D
:1081D00080028450EF5420601E12329B8A088B0963
:1081E000EA4509600A1231B7AA08AB09123CC7EE8A
:1081F000FAEF642002845090099AE064027024EE41
:10820000A2E0501F90055BE0640F701179001231FD
:1082100087E960099015C512D33B12319FEE6401C6
:10822000028356EE54207003028327750C007A20D7
:108230007B009005A1E0F9123E3BEA4B4C4D7017D4
:108240009080D41228417A207B009005A1E0F91299
:108250003E2F7404122A347C0079047A007B0012C9
:1082600032658A088B098018850882850983A3A353
:10827000A3A3A3A3A3A3A37401F0850A08850B09F4
:10828000E508450960777C007904AA08AB09123239
:10829000658A0A8B0B750C01E5082404F8E435099E
:1082A000F98882898312EF2C12EA8170CD850882C9
:1082B000850983A3A3A3A3A3A3A3A3A3A3E064010A
:1082C00070A6850882850983A3A3A3A3A3A3E05472
:1082D000047095850882850983A3A3A3A3A3A3A300
:1082E000A3A37406128B52700374B7F0E0FA8508EA
:1082F0008285098312862E12319902827A123235D2
:108300007C0079017A007B001232658B09EA45090D
:108310007010E50C700C7A207B009005A1E0F9123A
:108320003E35EE6420802FE0600764016003028424
:1083300026EE5410600812309DEE64108018EE5442
:10834000406008123115EE6440800BEE5480600BE3
:10835000122F6BEE6480FAEF028450EF5401601626
:108360009005D412CB81600612C5EB124AEEEEFAEC
:10837000EF6401028450EF5408604712306D900999
:108380008AE06401703490098BE0602EF508E4F512
:1083900009F50AF50B9080A4780C122C70780879F6
:1083A0000C12233F7808122A197A007B089005A145
:1083B000E0F9123E2F7404122A34EEFAEF64080238
:1083C0008450EF541060129005B3E06005E4F012A1
:1083D000306DEEFAEF64108077EF544060489005FE
:1083E000DE12CB8160399005E412CB8160319009B7
:1083F0008EE0640170299005DE12C5E8124AEE9005
:1084000005E412C5E8124AEE9080CC1228417A00A9
:108410007B409005A1E0F9123E2F7404122A34EE3D
:10842000FAEF6440802AEF5402600A123403EEFA35
:10843000EF6402801BEF5404601912CA8B12C89DAE
:10844000790190055412D33B122FE9EEFAEF640440
:10845000FB80047A007B0002C128C082C08374EADA
:10846000122AC87C167D007900AA18AB19123CA903
:108470007408122CC77402F090054A12977812847F
:10848000997409122CC712C89D7413122CC7E412D8
:10849000C9E71248977416800EE8F0A3E9F090053A
:1084A0005412D0FC227408122A3402C16074F712EC
:1084B000242E74DF122AC8EAFEEBFFEE4F602DACCB
:1084C00018AD191232BF7406122CC7E0601E741763
:1084D000122CC7E0FD7401122CC7E0FCEEFAEFFB92
:1084E0007900122E03E9600479A4800279007421D6
:1084F00002B15474F412242EEAFEEBFF8E828F83B5
:10850000A3A3A3A3A3A3E054406016128B46123387
:1085100079E960077AFF7BFF0285F512C5E40285E1
:10852000E890099AE06007640160030285CE900537
:1085300041E0A2E140030285CE8E828F831286281D
:1085400012C9ADA3A3A3A3E0FA88828983A3A312CF
:10855000D50E8E828F83A3A3A3A3A3A3A3E054105D
:108560006004794080027900750AFE750BFF780A75
:10857000122A2112B61C122845AC08AD09128B46EE
:108580001230737404122A34E5086A7003E5096B2B
:10859000600B12B6216A7003A3E06B704E750A007F
:1085A000780A122A2579028E828F8312B20CAA08C9
:1085B000AB091233BB7401122A347508CDAA088E98
:1085C000828F8312862E123199E9604C8057900970
:1085D0009AE06402600FE06004640170DD90054180
:1085E000E0A2E140D590054A12D33B74FE6A7003C5
:1085F00074FF6B60C512C5E412DA2F123379E98E6D
:10860000828F83600512AA42800312AA5712AA60C1
:1086100012489DE9F50870A5EE4F60097901EEFA60
:10862000EFFB12324102BEF5E0F812B24E2212ED1B
:10863000F7E0F92274F612242EE9FEEAFF7A0F7BA6
:1086400000123CC1EA4B601F8A828B83740CF0EEEF
:10865000A3A3F0EF8A828B8312AE959005A1E0F977
:10866000123CCD7900802FEEF912326B8A088B090B
:10867000A808A909E849601C88828983A3A3A3A349
:10868000A3A3A3A3A3740612E671E0F9123127EEA7
:10869000F9123247791002C4D474F412242E9005D2
:1086A0005BE0640F7030EA4B602C900556E0640884
:1086B0006005E06404701F8A088B09E4F50AF50B75
:1086C0007808122A197A017B009005A1E0F9123E80
:1086D000297404122A3402986374F212242EEAFEDA
:1086E000EBFF8C088D09890A740E122CC712979221
:1086F000850C82F583E4F0A312C8A3E0F912335588
:10870000E9602612D32E123379E96402701B8E823F
:108710008F83A3A3A3A3A3A3A3A3A312B8B4850C7D
:1087200082850D8312C89D8003750A0012B046141D
:10873000602514603A14605B14606314603F146039
:108740007D24FE70030287D81470030287EC147036
:10875000030287FF02880D780C122A21AC08AD09AC
:10876000EEFAEFFB1230857402122A34028808AC4C
:1087700008AD09EEFAEFFB12308B02881712D32EE8
:10878000123379E9600302880DEEFAEFFB1230D95B
:10879000028817A90AEEFAEFFB1233C1806A12BBF6
:1087A0005C64027068E50A700A12DAE87003A3E0FC
:1087B000697064EEFAEFFBA90A123349804A12DAB3
:1087C000E87003A3E069704512BB5C6402703EEE82
:1087D000FAEFFB123331803F9005D612CB81603720
:1087E000EEFAEFFB12C5EB124AEE802B12DAE870BC
:1087F00003A3E0697017EEFAEFFB1233CD8018EE99
:10880000FAEFFBA90A1233D9E9F50A800A750A00C2
:108810007AD37B0012437BA90A02D10D74F412248F
:108820002E74DB122AC88A088B098A828B83A3A341
:10883000E0F912326B8A0A8B0BAE0AAF0BEE4F7067
:108840000302894D850882850983A3A882A983E054
:10885000C0E012C86BD0E012E68864F1603385088E
:1088600082850983A3E064CD60278508828509831A
:10887000A3E0641A601B850882850983A3E064E98C
:10888000600F850882850983A3E064E16003028AA2
:108890003790099AE06007640160030289668E825E
:1088A0008F83A3A3A3A3A3A3A3E054087003028907
:1088B000668E828F83A3A3A3A3A3A3A3A3A37405FC
:1088C000F090099AE060046401705385088285097C
:1088D00083A3E064E960479005DA12CB8160061259
:1088E000C5EB124AEE9005DC12CB81603190054158
:1088F000E0A2E1502912CD59A3A3A312B05C888253
:10890000898312D33B123469EA4B60128508828551
:108910000983A3E0F99005DC12C5E8124AEE8E82C5
:108920008F83A3A3A3A3A3A3A3A3A3E064027010B4
:108930008E828F83A3A3A3A3A3A3A3A3A37406F0F0
:10894000850882850983A3A3E0F9123247123235E4
:1089500090099AE0640270099015C912D33B123154
:108960009F74250298607900123241E97003028AEF
:108970003790099AE0600764016003028A0C900551
:1089800041E0A2E14003028A0C12CB7C607E8E8221
:108990008F8312D33B7404122AAA12CD761232BFEF
:1089A000850882850983A3E064E97020128B351263
:1089B0002A25850882850983A3E0F50A780A122A08
:1089C0002512D51F1232F57402122A34740D122C9E
:1089D000C712CB7212E9AD12C89D7409122CC7E000
:1089E0006004794080027900740F122CC712B05CC9
:1089F000740D122CC712D33B12307FE9600E8E82A9
:108A00008F83A3A3A3A3A3A3E04420F0EE2404F543
:108A10000AE43FF50B8E828F8312ACEEE0F9850AF3
:108A200082850B8312D33B124783850A82850B8391
:108A3000EAF0A3EB0288C0850882850983A3E0C021
:108A4000E07402122CC7D0E012A4D4EEF0A3EF120F
:108A50008B52C0E07403122CC7D0E012E282E0AA6D
:108A600018AB19702E122FC590099AE060046401AA
:108A700070247402122CC7E0701C128B46123379DA
:108A8000E970369005DA12CB81602E12C5EB124ADE
:108A9000EE800312334F7402122CC7E064E97019A0
:108AA000128B35122A25750AE9780A122A2512D561
:108AB0001F1232F57402122A3490099AE06007649A
:108AC00001600302891E900541E0A2E14003028992
:108AD0001E8E828F83A3A3A3A3A3A3A3A3A3E06457
:108AE0000270398E828F83A3A3A3A3A3A3E05404AF
:108AF000602A128B46123379E98E828F83700F12AF
:108B0000C5E874FFF0A312AD09740502893FA3A361
:108B1000A3A3A3A3A3A3A3740302893F850882850B
:108B20000983A3E064E9600302891EEEFAEFFB12F9
:108B300033DF02891E8E828F8312D0FCE8FAE9FBB4
:108B4000750A01780A228E828F8312B227FAA3E077
:108B5000FB22F0E50812EDED3509F583E02274F40F
:108B600012242EEAFEEBFF7508007509008E828F35
:108B700083A3A3A3A3A3E0603B75080812D32E79B7
:108B8000FF122D5B8B0BEA450B601075082C8E8253
:108B90008F83A3A3A3A3A3E0D2E0F08E828F83A34D
:108BA000A3A3A3A3E0540364016003028C684308F9
:108BB00011028C68EE241812BB5F6049EE241A1271
:108BC000BB5F6003F4701D12DAE87003A3E0697004
:108BD00006750822028C68900556E0640460030262
:108BE0008C68801CEE241BF582E43F12B644241AE4
:108BF00012BB5FFAEE24191298381230EBE9706854
:108C0000750901806312D32E123379E9640270036F
:108C100075080112DAE87003A3E0697006E508D26E
:108C2000E1F508E50860158E828F83A3A3E0700646
:108C3000E508D2E58004E508D2E6F50812D32E1245
:108C40003379E964017006E508D2E0F5088E828F79
:108C500083A3A3E0601212B046F9123355E9640110
:108C60006006E508C2E0F50890099AE06004640136
:108C70007012E508A2E1400CE509A2E04006E50813
:108C8000D2E7F50802BEF574EC12242E74CD122A38
:108C9000C8EAFEEBFF851882851983129B54751074
:108CA0000075110075090090099AE06402701C8E2D
:108CB000828F83A3A3A3A3E060119015C712CB8179
:108CC00060099015C712D33B12319F7405122AAA6E
:108CD0008E828F83A3A3A312CB7412D3391232BF17
:108CE000E97003028E0A79017407122CC7E0C3945D
:108CF000024001197409122CC7E0C39402400279A2
:108D000000740E122CC7E064F87003A3E0F4700343
:108D1000028E0A740E122CC7E064F97003A3E0F40B
:108D20007003028E0A740E122CC7E064FA7003A35B
:108D3000E0F47003028E0A740E122CC7E064FB701C
:108D400003A3E0F47003028E0A7408122CC7E0F843
:108D5000900544E0686003028E0AE9A2E040030245
:108D60008E0A12B8AB7424122CC712C9D6241C1256
:108D7000B8AE7412122CC712C89D740B122CC7E027
:108D8000601D741C122CC7E0FD7406122CC7E0FC99
:108D90008E828F8312D3397901122E03E9703D74CC
:108DA00005122AA21231B1E9F508740B122CC7E0A2
:108DB000702E90053EE060287422550864226020E1
:108DC00074425508644270147422122CC712974FD3
:108DD000600E7422122CC712975560047ACF802C33
:108DE000E9A2E6506E90099AE06004640170259053
:108DF0000541E0A2E1501D7422122CC712B04F129F
:108E000028CA01010A2B8E000A8E7AD37B001243F6
:108E10007B0297337422122CC712B04F24FD600BD3
:108E200014600824FD600424FD70DF7422122CC736
:108E300012979A700E7422122CC712C5EAA3E0642E
:108E40000D60107405122AA21233B5E96401700393
:108E5000029733EE242DF582E43FF583129E2C70A9
:108E600003A3E069701E750A00780A122A25780AA1
:108E7000122A25EE242F1298381297661232F574B2
:108E800002122A34740B122CC7E07003028F3112C5
:108E900097661234698A0A8B0BEA450B7003028FBE
:108EA000DA7406122CC7E0F88E828F83A3A3E02821
:108EB000F8A3E03400F9E8240D12973DF88A828B7C
:108EC00083A3A3A3E068600FE88A828B83A3A3A394
:108ED00012DBCC1297A0F079047406122CC712A2F0
:108EE000C3E02AF8A3E034008882F583A3AA82AB0A
:108EF00083123CB58A0C8B0D8C0E8D0F850A8285F2
:108F00000B83A3A3A3A3780C1229834003029733F6
:108F10009080E0780C122BCB850A82850B83A3A36B
:108F2000A3A3E50CF0A3E50DF0A3E50EF0A3E50F78
:108F3000F090099AE064026015E060076401600344
:108F4000029074900541E0A2E1500302906E9005FA
:108F500056E064046008E064096003029733E508A2
:108F6000A2E54003029015EE242F12BB5FC0E0740F
:108F700002122CC7D0E01297C0C0E07403122CC7B5
:108F8000D0E01297B8C0E07404122CC7D0E0F0749F
:108F900016122CC7E0640170267410122CC71297A9
:108FA0005B7003A3E0697017740E122CC712D33BD9
:108FB000123379E9640270077416122CC7E4F012B8
:108FC00097AE1228417406122AAA7409122AA21214
:108FD0002FCB7404122A3402973390059BE064016E
:108FE0006003028F317422122CC712974F7009E56B
:108FF00008A2E65003028F317412122CC7E0F470FD
:1090000003A3E0F4600CEEFCEFFD7405122AA2123B
:1090100031BD029733A2E650527422122CC712CDF2
:10902000707016741C122CC7E06402703E74051236
:109030002AA2790012334980327422122CC7129767
:10904000557014741C122CC7E06404701E74051251
:109050002AA212333D80147422122CC712979A70E0
:109060000A79007405122AA21233C10297339009BB
:109070009AE06013E064016003029733900541E0D9
:10908000A2E140030297337416122CC7E0601CEE75
:10909000240212B60B129CF51412AE8B129CF5C072
:1090A000E07416122CC7D0E0F07006E508C2E7F5B0
:1090B00008E508A2E35061751110A2E25018740A85
:1090C000122CC7E054E3F0740A122CC7E0131313F8
:1090D000541FF8E0802CA2E4502A740A122CC7E036
:1090E0001313543F5407F86009740768600B18E8BD
:1090F0007007C3E508C2E7F508E8333354FCF8E02D
:1091000054E348F0740A122CC7E0C0E08E828F83CB
:10911000A3A312ADDBD0E0F0900556E06404600834
:10912000E0640960030291F4740E122CC712DAF5A0
:109130007003A3E069601F740E122CC712D33B1298
:109140003379E96402600F740A122CC7E054036497
:109150000160030297337407122CC7E07041EE24BC
:109160002F12BB5FC0E07402122CC7D0E01297C070
:10917000C0E07403122CC7D0E01297B8C0E07404AA
:10918000122CC7D0E01297A91228417406122AAAFD
:109190007409122AA2122FCB7404122A348052743A
:1091A00022122CC712CD707016741C122CC7E064EA
:1091B00002703E7405122AA279001233498032747B
:1091C00022122CC71297557014741C122CC7E0641D
:1091D00004701E7405122AA212333D8014742212E8
:1091E0002CC712979A700A79007405122AA21233BA
:1091F000C10297337461550870030292FBE508A21F
:10920000E0506D12B0537405122AA212311BE9709E
:109210005C1232EFE9F5097416122CC7E0700F7476
:1092200010122CC712975B7003A3E0696042A90972
:1092300012B0537405122AA2123121E96024E50804
:10924000A2E3500C85188285198374FFF0A3800C6B
:10925000740E122CC7129778E8F0A3E9F075100489
:10926000800EE508C2E5F508750900800353089FE4
:10927000E508A2E5503FEE242F12BB5FC0E0740268
:10928000122CC7D0E01297C0C0E07403122CC7D0D4
:10929000E01297B8C0E07404122CC7D0E01297A96E
:1092A0001228417406122AAA7409122AA2122FCB7C
:1092B0007404122A34E508A2E640030295CEA818E9
:1092C000A919880A890B780A122A21A90912974636
:1092D000122AA21231A57402122A34E9F509700388
:1092E0000295CE7422122CC712B04F6401600302A3
:1092F00095CE74104510F5100295CE7407122CC748
:10930000E06401705D7422122CC712B04F640570C6
:109310001EA818A919880889097808122A21129705
:1093200044122AA21231A57402122A34029733740D
:1093300022122CC712979A7029740E122CC712D3BE
:109340003B122EBDE9601BA818A919880A890B7861
:109350000A122A21129744122AA21231A57402126B
:109360002A347416122CC7E070257407122CC7E03B
:109370006401700C7422122CC7E0F812979A600CEA
:10938000EEFCEFFD7405122AA21231BD02973312D2
:10939000323BE96003029733741D122CC7E070035F
:1093A0000294497420122CC712B05C741F122CC78F
:1093B000E0FA741E122CC7E0F91230EBE9607D74FC
:1093C0001F122CC7E0701E740E122CC71297781251
:1093D000BC42FAA3E0FB122EC98B0BEA450B6003DB
:1093E0000295C880517420122CC712D33B741F12EF
:1093F0002CC7E0F91230E585188285198312DA2F1F
:109400007808740D122CC7E060027810740C122CCE
:10941000C7E06004740828F8740A122CC7E06001E1
:1094200008088E828F83A3A3E028FAA3E034008A81
:1094300082F583E014F07510400295C87508007835
:1094400008122A25790B029581740E122CC712C8B6
:10945000997409122CC7E0600302959CE508A2E309
:10946000500302959C7407122CC7E06401607A795E
:109470000085188285198312D33B12313F8A0A8BEB
:109480000BA80AA90BE849601C88828983A3A3A3BF
:10949000A3A3E06401605288828983A3A3A3A3A34A
:1094A000E064026044EE242D12B0568518828519BE
:1094B0008312D33B1234698A828B83E582458360B1
:1094C0000FA3A3E0F9123487E96005C3940840199B
:1094D0007410122CC712D33B122EBDE970030295F3
:1094E000777409122CC77404F0E4F5097809122A7C
:1094F00025741E122CC7AC82AD83740F122CC712B8
:10950000D33B740A122CC7E0F91231517401122AAC
:1095100034E9600F7510208E828F83A3A312B04FA1
:10952000543FF0741D122CC7E06023740E122CC738
:1095300012B05C741E122CC7AA82AB831232B9859A
:10954000188285198312DA2F74404510F5107407BC
:10955000122CC7E06401601579007410122CC71238
:10956000B05C740E122CC712D33B1230F1E508A286
:10957000E35037794080357508007808122A25793C
:1095800002740F122CC712B05C7411122CC712D3C4
:109590003B1233BB7401122A34029733E508A2E36D
:1095A00040030294E974400294EA79007410122C8A
:1095B000C712B05C740E122CC712D33B12307FE975
:1095C000600674204510F5101232EFE9F509851890
:1095D00082851983E064FE7003A3E0F470037509CB
:1095E0000090098DE064016003029681EE2413125D
:1095F000BB5FF47003A3E0F47003029681740E1253
:109600002CC7C3E094F9A3E094FF507512B8AB7473
:1096100010122CC7E0687003A3E069606474101234
:109620002CC712D33B122EC98A0A8B0BA80AA90B8E
:10963000E849604D88828983A3A3A3A3E064016005
:109640000D88828983A3A3A3A3E0640270337426E8
:10965000122CC7740112DFA5F8A3E0F97431122CA3
:10966000C712C89D7426122AA2122E8DE9601274A8
:1096700029122CC7AA82AB83122EDBE96003123FAA
:10968000BBE508A2E74003029733E50970030297A0
:10969000338E828F83A3A3A3A3E0FA7B00123D63E2
:1096A0008A0A8B0BEA450B7003029733EE2404F50C
:1096B00012E43FF5138E828F83A3129788122A1D1E
:1096C000851282851383E0FC7D00123C9D74031299
:1096D0002A347407122CC7E0C0E07402122CC7D0E1
:1096E000E0F07403122CC7E4F0A3F07402122A9A7B
:1096F000880C890D780C122A217810122A21E5098C
:10970000F5087808122A2512CA7D1228458512828A
:10971000851383E0F97407122CC712B05CAA0AAB58
:109720000B1232AD7407122A34E96007AA0AAB0B98
:10973000123D697433122A347F0C0226BDF582E48F
:1097400012E7D222790012CA8112B0607407221285
:10975000B22764062212B22D64072212D0FCEE2436
:109760001312B6286822EE242BF582E43FF583120B
:10977000B64A241312985322E012977D22F8A3E0F0
:10978000F985188285198322A3129792750E0078A5
:109790000C22E0F50CA3E0F50D2212B22D64032299
:1097A000A3E4F0A3F0A3F0A322F01297AE22EE24DC
:1097B00025F582E43FF58322F0EE243112B628220B
:1097C000F0EE243012B6282274F412242EEAFEEBB6
:1097D000FF8C088D0990098AE0600F12DAE87003A7
:1097E000A3E069700512306D804C790012D32E12FF
:1097F000313F8A828B83E58245836032A3A3A3A392
:10980000A3A3E054186027E508241C12C88012287E
:1098100045E508241312C880122845EE2418129832
:109820003812983D1231577404122A348008790096
:1098300012983D123097802B12B628F9228E828F13
:1098400083A3A3A3A3A3A3A3A3A312B64A240B1287
:10985000985322F582E43FF58312E9A8FB2274189D
:10986000122A347F040226BD74F012242E74EA12E8
:109870002AC88A0A8B0BEA2402F50EE4350BF50F91
:109880000A0AFB122ECF8A088B09AE08AF097508A9
:1098900001850A82850B83A3E0F509750C01AC0EE6
:1098A000AD0F740B122CC7AA82AB8312479B7413A3
:1098B000122CC7129B547415122CC77402F0740832
:1098C000122CC7E4F090156DE0700EEE4F700AE5B3
:1098D0000970067508C3029AA8900556E0640860EE
:1098E000067508C2029AA4850A82850B83A3A3A3E6
:1098F000A3A3A3A3A3A3A3E0A2E1500EA2E3500558
:10990000750C04800C750C038007A2E35003750CE2
:1099100002EE4F70030299B48E828F83A3A3A3A398
:10992000E06404600D8E828F83A3A3A3A3E064038D
:10993000700C7404650C602C7403650C60268E82B8
:109940008F83A3A3A3A3E06402600D8E828F83A301
:10995000A3A3A3E0640170357402650C6006740172
:10996000650C701C8E828F8312D33B123397E97083
:10997000438E828F8312A63F122CC712C89D80345B
:109980008E828F83A3A3A3A3E06402600D8E828FD7
:1099900083A3A3A3A3E06401700A8E828F8312A71E
:1099A000A6124AEEE50A2402FAE4350BFB122EDB7E
:1099B0007E007F007413122CC7E064FE7003A3E0E6
:1099C000F4704E122E99E97048E5096023900593D2
:1099D000E06402701B90157412D33B123397E97048
:1099E0000F90157412A63F122CC7E8F0A3E980204F
:1099F000850A82850B83A3A3A3A3A3A3A3A3A3A3E5
:109A0000E05402F91230A97413122CC7EAF0A3EB48
:109A1000F07413122CC7E064FE7003A3E0F4700529
:109A20007508C7807FE509F50D780D122A25850A8E
:109A300082850B83A3A3A3A3A3A3A3A3A3A3E0F95A
:109A4000E50A2402FCE4350BFD7414122CC712D372
:109A50003B122FEF7401122A34E97048A90CE50A71
:109A60002402FCE4350BFD7413122CC712D33B12F5
:109A70002EAB8A0E8B0FAE0EAF0FEE4F601E740230
:109A80006509700D8E828F83A3A3A3A3A3E0D2E305
:109A9000F07415122CC7E4F0F50880087413122C2A
:109AA000C7129B54E5097009AA18AB1912487980AE
:109AB0000AFCA90CAA18AB19123337E9F8EE4F606B
:109AC00053E50960208E828F83A3A3A3A3A3E0D2D2
:109AD000E6F074026509700D8E828F83A3A3A3A3A1
:109AE000A3E0D2E5F0850A82850B83A3A3A3A3A3F9
:109AF000A3A3A3A3A3E0A2E6500D8E828F83A3A30A
:109B0000A3A3A3E0D2E7F08E828F83A3A3A3A3A392
:109B1000A3E004F0E5087003E86034FC7D007A01FE
:109B20007B1012477DEE4F600CE50A2402FAE43503
:109B30000BFB122EDB7413122CC7E064FE7003A320
:109B4000E0F4600B7413122CC712A7A6124AEE742D
:109B50001602C12574FEF0A304F02274F712242E1D
:109B600074F7122AC8EAFEEBFF900556E064036022
:109B70000DE064016008E064096003029C858E8248
:109B80008F83A3E06003029C5B7C007D007A027BF4
:109B90000012477D129C8A8A828B8312B8B490058A
:109BA0004712C89D795312486D790090055412D31D
:109BB0003B122FE9900556E06409600990055412A4
:109BC000D33B123463851882851983740112C9E767
:109BD000794212486D9005567404F07401122AA25D
:109BE000794A1248677401122AAA7A4C7B051247F7
:109BF0009B90099AE060046401701F90054AE0643C
:109C0000FE7003A3E0F4602A79007401122AAA907E
:109C1000054A12D33B122EAB8018E06402701390F9
:109C2000054712B05C7A037B0012477D12A56612CD
:109C3000477D900541E0A2E35004D2F08002C2F0DB
:109C400012C9DD795212486D90099AE064027032AF
:109C50009015C512D33B12319F80278E828F83A32C
:109C6000AE82AF83FC7D007A037B1012477D8E822B
:109C70008F83E0F990055412D33B122FE9900556DB
:109C8000E4F012320B740902B154EE2402FAE43FFC
:109C9000FB22C082C08390051712CB81701F9005F4
:109CA00056E014600924FC600A14600C800F9005D3
:109CB00020803490051C802F90051E802AE8496082
:109CC0000890051812A2CC700C8A828B83A3E0F94D
:109CD000122FD1801D900517129CF5640270051299
:109CE00033F7800E9005D812CB81600612C5EB12B7
:109CF0004AEE02C160E0F8129CFB22A3E0C82406F1
:109D0000F582E438F583E02274F412242E74FB12F9
:109D10002AC88A088B097A0F7B00123CC18A0A8BF9
:109D20000BAE0AAF0BEE4F7003029E278E828F831D
:109D3000740212C9E7795012486785088285098341
:109D4000A3E06003029E0A900554E0F47003A3E0D0
:109D5000F46044900554E064FE7003A3E0F46037BF
:109D6000851882851983129E2C7003A3E0696027F1
:109D7000850882850983A374EAF07A477B057953C5
:109D800012486D7A4A7B05794B12486D7A547B05EF
:109D9000795012486D807385188285198312DBB95A
:109DA00012C89D7A477B0579531248679005471280
:109DB000ACFF12C89D7A4A7B05794B1248677A49F5
:109DC0007B0579E112486790055BE0C3940F501D55
:109DD000900549E0C0E07402122CC7D0E0F0740492
:109DE000122CC77401F004122AA2124891750A00BD
:109DF000780A122A25780A122A259015FBE0F91212
:109E0000A9EE1232F57402122A348508828509837C
:109E100012D64EA3F09005567403F0EEFAEFFB90C5
:109E200005A1E0F9123CCD740502986012DBBDE09B
:109E3000682274F412242E74E8122AC8EAFCEBFD9E
:109E40008C828D83A3A3A3A37808122C70780812A8
:109E50002C029005577808122B6C7F7F7E7F79004B
:109E60009005577808122C70E97808122A69E508DD
:109E7000A2E0502978009005A28014850882850907
:109E800083A3A3E069700108E508241412C88012B6
:109E9000A6C970E7E8C39F5004E8FFE9FE09E9C3DB
:109EA000941B40BC8C828D83A3A3A3A3122CA4E893
:109EB000494A4B607DEC2404F508E43DF50985082A
:109EC00082F583122CA4900557122CB07C187D00CB
:109ED0007900AA18AB19123CA9850882850983125A
:109EE0002CA4851882851983122CB07404122CC7F7
:109EF0007401F090055DE0C0E07405122CC7D0E05D
:109F0000F07407122CC7E412C9E7124885807090DC
:109F1000055412D33B12301F8A0A8B0BA80AA90BD7
:109F2000900554E8F0A3E912CB8E687003A3E069B2
:109F3000602D9005A212A6C9602585088285098337
:109F4000129E2C7003A3E069700C8508828509833A
:109F5000A3A3E06E60B9E508241412C88080D6EE91
:109F6000900549F01231EDE96015900556E4F09046
:109F7000052212CB81600879C412C5EB124AEE02A9
:109F8000985E74F412242E74E8122AC88A828B8395
:109F9000A3A3A3A3A3A3A3A3A312B8B4E8FAE9FBC2
:109FA00079009005577808122C70E97808122A6910
:109FB000E508A2E05031EA29F582E43BF583E0F8B8
:109FC000901573E0C398501F750801750900750A54
:109FD00000750B00E978081229C17808122C02904C
:109FE00005577808122B6C09E9C3941B40B49005FF
:109FF00057122CA4E8494A4B604E7C187D0079002A
:10A00000AA18AB19123CA9900557122CA4851882E6
:10A01000851983122CB07404122CC77401F07407D4
:10A02000122CC77401F090055DE0C0E07405122C9D
:10A03000C7D0E0F07407122CC7E412C9E7124885B4
:10A040009005567406F0801E900556E4F0FCFD7AEB
:10A05000047B1012477D90052212CB81600879C4E1
:10A0600012C5EB124AEE02985E74F512242E74D1DA
:10A07000122AC88A088B098A828B8312B8B8741C8A
:10A08000122AAA8A828B83A3A3A3A3A3A3A312B297
:10A090000312D33612321D741C122CC7E0702C85AB
:10A0A0000882850983A3A3A3A3A3A3A3A3E0C394C6
:10A0B0000B40188E828F83A3A3A3A3A3A3A3A3E023
:10A0C0006402700712C86BE0F4600302A2BE900540
:10A0D00056E06402700302A1A0E06406700302A1CE
:10A0E000A090051712CB81600812A2CC700302A1C8
:10A0F000D5900556E064086008E06404600302A29D
:10A10000BE741E122CC712A2C3A3A3A3A312B8B875
:10A11000900517E0F8496007129CFB640260779095
:10A120000554E06E7003A3E06F600302A2BE7401E9
:10A130006A60167423122CC7AC82AD837A687B05E3
:10A14000124795E9600302A2BE7A007B029005A146
:10A15000E0F9123E3BEA4B4C4D600302A2BE900573
:10A1600057122CA4851882851983122CB090055D96
:10A17000E0C0E07404122CC7D0E0F07405122CC7C4
:10A180007401F07406122CC7740212C9E7122F531F
:10A19000E9600302A2BBEEFAEFFB1233F102A2BEAA
:10A1A00090051712CB81702D7508007808122A25AA
:10A1B0007808122A25EE2410F582E43FF58312CBAD
:10A1C00075A3A3A3A3A3A3A3A3A312ADD01232F597
:10A1D0007402122A348E828F8312B8B47407122C40
:10A1E000C7E8F0A3E912AD0912B8B47409122CC77C
:10A1F00012C9D6240D12BB5FC0E0740B122CC7D05D
:10A20000E0F012C86B12ACE2740F7808122C527492
:10A210000C122CC7E508F07420122CC7E0C0E074C3
:10A220000D122CC7D0E0F07422122CC7E0C0E074ED
:10A230000E122CC7D0E0F0741D122CC7E0C0E074E1
:10A2400010122CC7D0E0F0741E122CC7E0C0E074CE
:10A250000F122CC7D0E0F0EE241012BB5FC0E074E8
:10A2600011122CC7D0E0F07421122CC7E0C0E074AA
:10A2700012122CC7D0E0F0742E122CC7E0C0E0748C
:10A2800013122CC7D0E0F07423122CC7A982AA8322
:10A2900089088A09750A007808122A1D7C087D0041
:10A2A0007417122CC7AA82AB83123C9D7403122A26
:10A2B000347407122AA2122FE38003122F59742F2D
:10A2C00002EF3BE0FA8E828F83A3A322129CFC64F0
:10A2D000012274F612242E74C9122AC89005D212D3
:10A2E000CB81600612C5EB124AEE900556E0640879
:10A2F000700302A38F900593E06402702390509046
:10A30000E493900538F0905090E493900536F090E7
:10A31000055F7401F01297A004F0A3E4F0A3806C31
:10A32000900567E0F8749328F582E4340EF583E035
:10A33000FA900538F0749428F582E4340EF583E041
:10A34000F9900536F07508FF7509FFEA7808122BB9
:10A35000DEE508F4FCE509F4FD3395E0FE90055FC9
:10A36000ECF0A3EDF0A3EEF0A3F07508FF7509FF84
:10A37000E9C39A7808122BDEE508F4FCE509F4FD40
:10A380003395E0FEA3ECF0A3EDF0A3EEF0A3F07C98
:10A39000237D0079007414122AA2123CA99005674B
:10A3A000E07009741E122CC774018006741E122CF2
:10A3B000C7E412A4D4740FF090157212C9E779465D
:10A3C00012486D7401122CC7E4F09015D4E0C0E07F
:10A3D0007402122CC7D0E0F0900544E0C0E0740392
:10A3E000122CC7D0E0F07404122CC7E4F0740512EC
:10A3F0002CC7E4F07407122CC7E4F0900567E0C3A3
:10A40000940F500CE0C0E07406122CC7D0E0800717
:10A410007406122CC7740FF07C687D057408122C2A
:10A42000C7AA82AB8312479B7C037D0079FF74101F
:10A43000122CC7AA82AB83123CA99005A0E0C0E011
:10A440007413122CC7D0E012C7DF7401122AA212B3
:10A4500032177AA47B05794512486D123325900591
:10A460005BE0C0E0741C122CC7D0E0F090055CE00B
:10A47000C0E0741D122CC7D0E0F0900549E0C0E0A8
:10A48000741A122CC7D0E012849D7418122CC712B3
:10A49000C89D7420122CC7E4F090055EE0C0E07403
:10A4A0001F122CC7D0E0F07434122CC7E4F07429CA
:10A4B000122CC7E4F07A477B05795312486D7A4A2B
:10A4C0007B05794B12486D7414122AA212488B74C2
:10A4D0003702C4D112A4D822F085188285198322AC
:10A4E000C082C0838A828B83A3E09005566004E417
:10A4F000F080707408F0900567E0702890052212D3
:10A50000CB816008790012C5EB124AEE9005541217
:10A51000B05C7A057B0012477D90055412D33B1244
:10A52000346380187900122FDD90054712B05C7AF1
:10A53000067B0012477D12A56612477D9005DE124C
:10A54000CB81601F90098EE0640170179080CC125F
:10A5500028417A007B409005A1E0F9123E2974045D
:10A56000122A3402C16090054A12B0607A047B005E
:10A570002274F412242E74EA122AC8EAFEEBFF12A7
:10A580009C8A122ECF8A088B09EA4509700302A61D
:10A590003A8A828B83A3A3A3A3E0640160278A8203
:10A5A0008B83A3A3A3A3E06402601A8A828B83A394
:10A5B000A3A3A3E06403600D8A828B83A3A3A3A358
:10A5C000E064047075EE2402FCE43FFD740B122C71
:10A5D000C7AA82AB8312479B85088285098312A68E
:10A5E0003F122CC712C89D7415122CC77401F07449
:10A5F00008122CC7E412C9E712487F890AAC0A7D09
:10A60000007A077B0012477D850882850983A3A312
:10A61000A3A3A3E0C2E012C0CCA3A3740112E291F1
:10A620005001097A027B00122247E88508828509D9
:10A6300083A3A3A3A3A3A3A3A3F0741602986012F9
:10A64000D0FC74132274F212242E74F8122AC8EA71
:10A65000FEEBFF8C0A8D0B890C908062AC18AD1953
:10A660007408122962F50DEEFCEFFDAA18AB191261
:10A670004795E97003750D019005A2801AEEFCEF75
:10A68000FDE508240BFAE43509FB124795E9702330
:10A69000E508241412C88012A6C96024E50DA2E0C2
:10A6A00040DB850882850983E0650A7004A3E065C4
:10A6B0000B70DD850882850983A3A3E0650C70D04B
:10A6C000AA08AB09740802D10A12ACE6E5084509EC
:10A6D00022C082C0839005A202C15D74F712242EAD
:10A6E0009005A212E9A8800C12D3C712B8BB123D84
:10A6F00069EEFAEFFBEA4B70EF9005A2E4F0A3F0ED
:10A7000002B15774F412242EEAFEEBFFEE2413126A
:10A71000BB5F6403700CEE240BFAE43FFB122ECFF8
:10A72000800EE06402707C12C86B12D33B122EC9FB
:10A730008A088B09E508450960698E828F83A3E04A
:10A74000700F850882850983A3A3A3A3A3A3E48034
:10A750005164F1600A8E828F83A3E064E1702785E3
:10A760000882850983A3A3A3A3A3A3E064017016B1
:10A7700085088285098312A7A6124AEEEE240BFAF9
:10A78000E43FFB122EDB850882850983A3A3A3A3E4
:10A79000A3A3E0600E850882850983A3A3A3A3A3D6
:10A7A000A314F002986312985990053012C8B12290
:10A7B00074F112242E8A088B09ECFEEDFF890A122F
:10A7C000D63BEEF8EFF9A30EAF838A828B83A3A367
:10A7D000E0C454F0FA88828983E04A12A89112D624
:10A7E0004F12A88CE0333354FCF88E828F83E048FC
:10A7F00012A88CA3E033333354F8F88E828F83E0B1
:10A8000048F0EEF8EFF9A30EAF838508828B83A39F
:10A81000A3A3A3A3A3E0A2E0E4331313FA888289DD
:10A8200083E04AF0E5082407F50CE43509F50D75D9
:10A830000E00780C122A1D7C087D00EEFAEFFB1248
:10A840003C9D7403122A34EE2408FE50010FE508E3
:10A85000240FF50CE43509F50D780C122A1D7C0344
:10A860007D00EEFAEFFB123C9D7403122A34E50AD8
:10A87000C3940F4012E5082412F582E412DEC58E5F
:10A88000828F83A3A3A3F07F070226BD12A891A302
:10A8900022F08508828B83A3A3A32274F112242EB5
:10A8A000EAFEEBFF890A8C088D098E828F83E08C8B
:10A8B000828D8312B65AAE82AF83E012BEFA12C006
:10A8C000E8C412BEFA12A965E054038C828D83128B
:10A8D000C0E6A2E2E4338C828D8312C0E513131329
:10A8E000541F12BEFA12C0E4A2E7E4338C828D83B7
:10A8F000A3A3A3A312A9658E0C8F0D750E00780C6F
:10A90000122A1D7C087D00E5082407FAE43509FBBE
:10A91000123C9D7403122A34EE2408FE50010F8E5F
:10A920000C8F0D780C122A1D7C037D00E508240F86
:10A93000FAE43509FB123C9D7403122A34E50AC37C
:10A94000940F40158E828F83A3A3A3E0C0E0E50897
:10A95000241212C880D0E08008E508241212C880B2
:10A96000E4F002A887A3A312B65E0EAF832274F5AB
:10A9700012242E8A088B098A828B83A3AE82AF832E
:10A98000E0F91230078E828F83E064EB6024850843
:10A9900082850983A3E064E16018850882850983C4
:10A9A000A3E064F1600C850882850983A3E0641A42
:10A9B0007009850882850983A3E4F09015C512D338
:10A9C0003B12319F750A01780A122A258508828573
:10A9D0000983A3E0F5087808122A25790012A9EE68
:10A9E0001232F57402122A3412323502EF3E90050B
:10A9F0005412B06090054A12985922C082C083E96F
:10AA00009005B47003E4800274018065E0F902C12E
:10AA10006074F712242EEAFEEBFF8E828F8312C938
:10AA2000AF12DA1412DA2F123379E98E828F836033
:10AA30000512AA42800312AA5712AA6012489D0268
:10AA4000B15712AA49E4F0A322E0F8A3E0C8240D0C
:10AA5000F582E438F5832212AA497401F0A3E422B6
:10AA6000F07C8D7D318E828F8312985922EAF0A37B
:10AA7000EBF002C16074F612242E9005B4E0701B56
:10AA80007C0079017A007B00123265EA4B600C8A07
:10AA9000828B8312CB81600312319302C4D4C082B3
:10AAA000C083790412325FE9F890509DE493C39813
:10AAB000401079FF12325FE9F890509CE493C398FC
:10AAC000500479018002790002C16074F012242ED2
:10AAD0008A088B09890B750C008A828B83A3A3A338
:10AAE000A3A3A3A3A3E0F912326B8A0E8B0FAE0EC1
:10AAF000AF0F750A01EE4F600302AB9B850882859C
:10AB0000098312ACEEA3A3A3A3A3A312BC3412D354
:10AB10003B1232538A0C8B0DAE0CAF0DEE4F70030F
:10AB200002ACD48E828F83A3A3A3A3E4F0A3F0E5A9
:10AB300008240CFAE43509FB8A828B83E0C0E0121A
:10AB4000E287D0E0F0123385EE240D12DA29E50811
:10AB500012DEB7350912B8B212B61C12C89D750CB8
:10AB600001EE240612BB63547FF0A3E054FC12E60E
:10AB7000885404600302AC129015CDE0F508750905
:10AB80000074077808122BDE8E828F83A3A3A3A301
:10AB9000A3A3E04508F0A3E04509F08E828F83A3CC
:10ABA000A3A3A312ACE074077808122C52E5085452
:10ABB00007F508E50B606B8E828F83A3A3A3A3A385
:10ABC000A3A3A3A3740212C0E912AFCB600B90053C
:10ABD0004212ACFFA3A312C89DE508700302ACA00B
:10ABE000EE240612EDC0547FFCA3E054FCFDE50802
:10ABF00024FFF508E434FFF50974077808122BDE0A
:10AC0000EC4508F8ED4509F98A828B8312C89D024C
:10AC1000ACA08E828F83A3A3A3A3A3A3E04480024E
:10AC2000AB9AE5087005750A0080758E828F83A344
:10AC3000A3A3A3A3A3E05420600C123CBBEA547F5F
:10AC40007900245F80198E828F83A3A3A3A3A3A37B
:10AC5000E05410601A123CBBEA540F7900240A50E9
:10AC600001098E828F83A3A3A3A3F0A3E9800D8E95
:10AC7000828F83A3A3A3A37401F0A3E412AD09748C
:10AC800004F07A207B009005A1E0F9123E3BEA4BEC
:10AC90004C4D700C7A207B009005A1E0F9123D0329
:10ACA000E50CA2E050318E828F83A3A3A3A312D31D
:10ACB0003FF9EEFAEFFB123259E9601B12B14C1268
:10ACC000CB7F600912B23B12D33B123D69EEFAEF23
:10ACD000FB123D69750A00A90A02C1288E828F8382
:10ACE000A3A312ACE622E0F508A3E0F50922A3A392
:10ACF000A3A3A3A312B060850882850983A32212AF
:10AD0000D0FC8E828F83A3A32212C88DA3A3A3227B
:10AD100074F412242E74F7122AC87E0012326BEAE1
:10AD20004B700302ADC98A828B83A3A3A3A3A3A301
:10AD3000A3A3A3E06406600302ADC98A828B83A348
:10AD4000A3A3A3A3A3A3E0FF8A828B8312ADDBE0BE
:10AD5000C0E07408122CC7D0E012B22012C89A12B8
:10AD60003289EF5408606085188285198312B05CBF
:10AD70007A007B0012324D8B0BEA450B704912EFC3
:10AD8000351248B57C007D007A007B0080258E82DC
:10AD90008F8312B04FF47003A3E0F4602A9005543F
:10ADA00012ADD01248AFE9641A601C7C007D00EE41
:10ADB000FAEFFB12324D8A0A8B0BAE0AAF0BEE4F45
:10ADC00070CC79001248BB7E01EEF97409029860DC
:10ADD00012B0608E828F831298592212B8A612ADDB
:10ADE000E2222408F582E438F58322C082C083EA97
:10ADF0004B70059005B580068A828B83A3A312AFA2
:10AE0000FF60258A828B83A3A3A3A3A3A3A3E054FB
:10AE10000860E5EC4D60158A828B8312B04F6C7030
:10AE200003A3E06D70D280047A007B0002C16074DD
:10AE3000F212242EEAFEEBFF890A8C088D097A11A2
:10AE40007B00123D63EA4B603E8A828B83A3A3A3FF
:10AE5000A3A3A3A3A3A3E412B214A3E50A12DBCC19
:10AE6000A3A3A312F0168A828B83A3A3A3A3E4F067
:10AE7000A312B23512AE9512DA1C12B72AE4F01200
:10AE8000AE8AA3A3F0A3F002D10DA312AE8F22F0DD
:10AE90008A828B8322A3F012EDEC3BF583E4F0224F
:10AEA00074F412242EEAFEEBFF89088C0A8D0BEE57
:10AEB0004F700302AF5474016508701279011232A9
:10AEC0005FE9F89050A2E493C3985022801674046E
:10AED00065087014790412325FE9F890509DE4938C
:10AEE000C398500A7911806E7402650870668E826C
:10AEF0008F83A3A3A3A3A3A3A3A3A3E50812BE6563
:10AF000012D6338E828F83A3A3E4F0A3F09005B50D
:10AF100012CB8160178003E0F8A312C9B6A3A31275
:10AF2000AFFF88828983A3A370ED80039005B512DB
:10AF3000DA207A207B009005A1E0F9123E3BEA4B33
:10AF40004C4D700C7A207B009005A1E0F9123D0376
:10AF50007900800279C1029863C082C083E9F879E0
:10AF6000009005B5801D8A828B83A3A3A3A3A3A30E
:10AF7000A3A3A3E068600574FF687001098A828B4F
:10AF800083A3A312AFFF70DE02C16074F712242EF8
:10AF9000EA4B70059005B580068A828B83A3A312C5
:10AFA000AFFF60208A828B83A3A3A3A3A3A3A3A341
:10AFB000A3E06970E4EC60108A828B83E012AFCB6F
:10AFC00070D780047A007B0002B15712AA4AE0547D
:10AFD0000422C082C0839005B580068A828B83A339
:10AFE000A312AFFF60128A828B83A3A3A3A3A3A3A0
:10AFF000A3A3E06970E580047A007B0002C16012BF
:10B000009859EA4B2274F712242EEAFCEBFD9005C6
:10B01000B580068A828B83A3A312AFFF60218A8248
:10B020008B8312B04F6C7003A3E06D70E68A828B45
:10B030008312862A12CA9CA2E0E43370D680047A76
:10B04000007B0002B157EE241DF582E43FF5831228
:10B05000B22722EE2413F582E43FF58312B060227A
:10B0600012B06422E0FCA3E0FD2274F212242E8AC6
:10B070000A8B0B8C0C8D0D750800750900EA450BC9
:10B0800060309005B580068E828F83A3A312B8BB73
:10B09000EE4F601EAC0CAD0DEEFAEFFB850A82851B
:10B0A0000B83124AEEE9640170DDEEF8EFF98808CF
:10B0B0008909AA08AB0902D10D79000229E674F7C3
:10B0C00012242E9005B512B8B47C007D00800DE8E6
:10B0D000FCE9FD88828983A3A312B8B4E8496030F3
:10B0E000EA687002EB6970E79005B512D33BE86A35
:10B0F0007002E96B88828983A3A3700812B8B490A8
:10B1000005B5800912B8B48C828D83A3A312C89DA3
:10B11000804574F712242EEAFEEBFFEE4F602B12EF
:10B12000328312B241123D698E828F8312D33B1259
:10B130003D6912B14C12CB7F600912B23B12D33B76
:10B14000123D69EEFAEFFB123D69800BEE240DF51E
:10B1500082E43F22122A347F010226BD74F71224B2
:10B160002E8A828B8312B20C9005B512B8B4750882
:10B17000007E00803388828983A3A3A3A3A3A3A313
:10B18000A3A3E0640570180E88828983E0FFA3E022
:10B19000F5838F82E06C7003A3E06D700205088870
:10B1A000828983A3A312B8B4E84970C99050991258
:10B1B000E3DC500890509512D27C400F8A828B833A
:10B1C000A3A3A3A37401F0A3E4800C900542E0F8CC
:10B1D00012B203E8F0A3E912B235740512B214E01A
:10B1E000440812B220F47003A3E0F4600E900554FA
:10B1F00012D5361248AFE9641A700579011248BBBE
:10B2000002B157A312B604A3A3A3A32212B227FC30
:10B21000A3E0FD2212B2182212DBD4A3A3A3A3221F
:10B2200012AE8F12B22722E0F812B22D22A3E0F55F
:10B23000838882E02212B218A3A32212B14CF583B4
:10B240002212B248129857228E828F83E0F8A3E030
:10B25000C8241FF582E43822C082C083EAFCEBFDDB
:10B26000EC4D6017EC24FBF582ED34FF12CB7F70C0
:10B270000712B2B2E0F46007123CC7790580309043
:10B2800005A1E0C0E012B2B2D0E0F090508DE4939E
:10B29000F97AB77B05123CFDE9640170107A007BF6
:10B2A000209005A1E0F9123D0379008002790402A3
:10B2B000C160EC24FFF582ED34FFF5832274F412B3
:10B2C000242EA2AFE433F508C2AF9005B712B8BB85
:10B2D000EE4F603AEE24FBF582EF34FF12CB7F7A1B
:10B2E000007B209005A16007E0F9123D038005E096
:10B2F000F9123D09E4F50AF50B780A122A21EEFC51
:10B30000EFFD7AB77B05123CF77402122A34E50888
:10B31000A2E092AFEEFAEFFB02986374F012242ED3
:10B3200074DB122AC8EAFEEBFF750B00750A007584
:10B3300008FE7509FF12323BE9600302B5F7EE24FF
:10B340001512BB5F60469015E8E0C43354E0F8E0A6
:10B35000333354FC48C0E012D320D0E012B65A1266
:10B36000D33A79FF122D5B8B0DEA450D6011750BF9
:10B37000017508FF12B621440412C8BAD2E0F09059
:10B38000099AE0600464017003750A408E828F831D
:10B3900012D339123379E9600312C98DEE241312E6
:10B3A000BB5F700D905098E493C0E012CA7DD0E06E
:10B3B000F08E828F83E0A2E7500454038019EE24BC
:10B3C0001412BB5F7012900533E0C0E012ED9ED006
:10B3D000E0F0900533E004F012EDB770199015D647
:10B3E000E0600D90053EE0700D8E828F83E0700668
:10B3F000EE241112C99090099AE06004640170482B
:10B40000900541E0A2E15040E50BA2E040218E8290
:10B410008F8312D339123379E9602D8E828F83E0C6
:10B42000600DEE240B12B049F9123355E960191280
:10B43000B630700302B5A8EE241312EDBA60030211
:10B44000B5A812B62154FBF08E828F83E0640170A0
:10B450000DEE240B12B0496402700312B63D12B611
:10B4600030600302B521E50BA2E0500302B5219044
:10B47000099AE060076401600302B521900541E08C
:10B48000A2E1400302B521E50AF50B780B122A254B
:10B49000EE2406FCE43FFD8E828F8312D339EE2426
:10B4A000121298381231517401122A34E9600612CE
:10B4B000C98D12B6368E828F83A3A3A3A3A3A3E064
:10B4C000603CEE2402F50CE43FF50D850C8212B6CB
:10B4D000442407FAE43FFB1232B98A088B09850C31
:10B4E00082850D83E065087004A3E06509700C8E09
:10B4F000828F83A3A3A3A3A3A3E4F012B63D8E82FD
:10B500008F83E064016008A90A12B64F1230F1A9D6
:10B510000A8E828F8312B64F12307FE9600312B613
:10B5200036AC18AD19EEFAEFFB1232B38A0A8B0B68
:10B5300074FE6508700474FF6509700312ACDCEAE0
:10B54000450B700302B5FB8E828F83E0C0E074016F
:10B55000122CC7D0E0F07402122CC712DA2074014A
:10B56000122A9A880C890D780C122A2112B61C1204
:10B570002845EE240E12BB5FF50C780C122A25909C
:10B5800005471228457407122CC7E0F9AC08AD092D
:10B590001232AD7407122A34E9FE74106E705EAA7E
:10B5A0000AAB0B123D698055EE241312BB5FC0E05D
:10B5B0007415122CC7D0E012EE1B740D122CC7129A
:10B5C000C9D6240412B60B12B8B4740F122CC712C9
:10B5D000C9D6241412BB5FC0E07416122CC7D0E089
:10B5E00012E27D12B60412B05C7404122AA2123167
:10B5F00021E9600302B448791180047E10EEF974E9
:10B600002502C125E0F98A828B832212B60F22F827
:10B61000E43FF9E8FAE9FB8A828B8322EE12C9A2A1
:10B620002212B62522EE240FF582E43FF583E022B4
:10B6300012B62554402212B6254420F02212B62517
:10B640004440F022F58312B64A2212B064EE22A3DF
:10B65000A3A3A312D34B1298592212B65E22F08EE6
:10B66000828F83A322C082C08374DC122AC88A829C
:10B670008B83A3A3A3A312B8B4740E122CC7E8F053
:10B68000A3E912D0F3740C122CC712C89D12B72A6A
:10B69000E0C0E0741A122CC7D0E0F012B7343B12AD
:10B6A000B8B27420122CC712C89DEA12D3283BF5F9
:10B6B00083E0C0E07408122CC7D0E0F0EA241CF547
:10B6C00082E43B12B8B27412122CC712C89DEA244D
:10B6D00011F582E43BF583E0C0E07409122CC7D079
:10B6E000E0F0EA2412F582E43BF583E0C0E0740761
:10B6F000122CC7D0E012A4D474FFF07401122CC72E
:10B7000074FFF07402122CC774FFF09080D01228DE
:10B71000417404122AAA7407122AA2122FCB7404AD
:10B72000122A34790074240284A7EA240DF582E4F5
:10B730003BF58322EA12EDED2274EE12242E74EF13
:10B74000122AC88A0E8B0F8C088D09890C750A1075
:10B750007A217B00123D6312D153E849700302B88D
:10B760009F750B007C217D007900851882851983E7
:10B77000E0FA123CA97426122CC712B8BB90099AA1
:10B78000E060046401703EAA08AB09122EC98A1059
:10B790008B11A810A911E849602388828983A3A38B
:10B7A000A3A3E06401600D88828983A3A3A3A3E01F
:10B7B00064037009EE5440700474044FFFEF5404A6
:10B7C0006003750B0190055412D33B8518828519CF
:10B7D0008312B8A62409F582E43812DA2D742312F4
:10B7E0002CC712B8B4740F122CC7E8F0A3E912B832
:10B7F000C112EDE312B8C112ADE2740212BC3E12E6
:10B80000C5E9E508F0A3E50912B8C112EDAEE50CF3
:10B81000F07425122CC7E0F508851882851983126B
:10B82000EDF3E50812B8C1241FF582E438F583E58D
:10B830000EF0A3E50FF07406122CC712DA2074087C
:10B84000122CC7E508F07428122CC712C5E8C08274
:10B85000C083740C122CC7AC82AD83D083D08274A9
:10B8600003122962A90BAA18AB19123241E964012B
:10B87000702190099AE0600464017012E50BA2E067
:10B88000500CA90812326BEA4B600312328F750A12
:10B8900000800C85188285198312D33B123D69A95B
:10B8A0000A741102BE7212D101C822EE2413F5826D
:10B8B000E43FF58312D0FC22A3A3A3E0FEA3E0FFA4
:10B8C0002212D162C82274EE12242EEAFEEBFF8C03
:10B8D000088D098E828F83A3740812C9C9E060089D
:10B8E0008E828F83A37410F012BB5C60098E828FEE
:10B8F00083A3E02408F0EE241512BB5F60088E825B
:10B900008F83A3E004F08E828F83A3A3A3A3A3A3BA
:10B91000E060198E828F83A3A3A3A3A3A3A3E0C394
:10B92000332402F88E828F83A3E028F0EE241112D4
:10B93000BB5F6005750B0E8003750B008E828F83D5
:10B94000A3E0F8EE240D12BB5F28250B8C828D83BB
:10B95000F0EE241112BB5F601190053FE0F9122E4A
:10B9600009850882850983E029F085088285098395
:10B97000E0C39475400975080075090002BB55E0E5
:10B98000FA7B00123D638A088B09EA4509700302BD
:10B99000BB558E828F83E0FA90054412BB6D740212
:10B9A000780C122BDEEA450CFAAB0DEE241212BB1A
:10B9B0005F5403F50C750D007406780C122BDEEA4B
:10B9C000450CFCEBFDEE241512BB5F600478018092
:10B9D000027800EE2416FAE43FFBE8F9ED49FDEEAB
:10B9E000241112BB5FF50C7409780C122BDEED45A7
:10B9F0000DFD8A828B8312BB6D740B780C122BDECB
:10BA0000ED450DFD12BE4212BB6D740C780C122B6D
:10BA1000DEED450DFD8E828F83A3A3A3A3A3A31206
:10BA2000BB6D740A780C122BDEECF8ED450DF9E8CD
:10BA3000850882850983F0E9A3F0EE240212BB6336
:10BA400085088285098312BB91F0EE2404F8E43F57
:10BA5000F98882898312C093A312BB91A3A3F0EE4D
:10BA6000241312BB74F0EE241412BB74A3F0750AF5
:10BA7000088A828B83E06015EE241812B056E50820
:10BA80002408FAE43509FB12479B750A1012BB5CC7
:10BA9000601BEE241A12B056850A0CE508250CFA34
:10BAA000E43509FB12479B7408250AF50A8E828F3C
:10BAB00083A3A3A3A3A3A3E06058EE2407F510E497
:10BAC0003FF511851082F583E0C0E012C879D0E01F
:10BAD00012BB81E0C0E012C879D0E012BB8112979E
:10BAE00088122A1D851082851183E025E0FCE4334D
:10BAF000FD850A0CE508250CFAE43509FB123C9D8E
:10BB00007403122A34851082851183E0C333250A19
:10BB1000F50AEE241512BB5F6008C0E012C879D0A8
:10BB2000E0F012C86B129789122A1DEE240D12BB89
:10BB30005FFC7D00850B0A8E828F83A3E0F8E50809
:10BB400028F8E43509F9E8250AFAE439FB123C9DA6
:10BB50007403122A34AA08AB0902BE75EE24171228
:10BB6000B62822F8E43FF988828983E022E0F50CC8
:10BB7000750D0022F582E43FF58312BB9AA3A3A3BF
:10BB800022F0050A8E828F83A3A3A3A3A3A3A3A35A
:10BB900022A3A312DFAB12BB9A2212C097A3A32247
:10BBA00074F412242E74FD122AC88A088B09ECFE44
:10BBB000EDFF7401122A9A880A890B780A122A2149
:10BBC0007402122AAAEEFAEFFB1230CD7402122A86
:10BBD00034E97057851882851983E08508828509C4
:10BBE00083F07401122CC7E0F812BC34A3A312BC7A
:10BBF00042602914850882850983A312BC3E12D7AE
:10BC0000147401122CC7E028F8A3E039F9E824FEE7
:10BC1000F582E934FFF58312E9A8800C8508828556
:10BC20000983A3E4F0EEFAEFFB80047AFE7BFF7455
:10BC300003029860A3E0F98508828509832212BC7B
:10BC40004A22E8F0A3E912BC4A2212BC4E2212A4F6
:10BC5000D8E02274EE12242E8A0A8B0BECFEEDFF44
:10BC6000750F01E9C39408500302BDDA8E828F83F9
:10BC7000E912AE8B12C0BE1232C5E96003750F0027
:10BC800012C0A08E828F8312C0F0EE12B7353F1221
:10BC9000C0DAC0E0EE2411F582E43FF583D0E01273
:10BCA000C0D2C0E0EE2412F582E43FF583D0E0126A
:10BCB000B65A740812BE65A3A3A3E06018E50A246F
:10BCC00008F8E4350BF912CA7D12C89D8E828F8365
:10BCD000A3E02408F08E828F83A3A3A3A3A3A3A32E
:10BCE000A3E0601C8E828F83A3858208858309125E
:10BCF000C0B3EE241512E25FA3E912CB8E2408F044
:10BD00008E828F83A3A3A3A3A3E0600F12BE4C8EE9
:10BD1000828F83A3A3A3A3A312BE6CEE241912C91E
:10BD200090EE241B12C990A3F0EE241812BB5F7092
:10BD30000302BDCA12BE4CFAEE2419F582E43FF5A7
:10BD400083EA12BE6CF8E50A28F582E412E256F89E
:10BD500012CB92E812BE6CE8C39AEE506824191216
:10BD6000BB5FF890508CE493C398500575110C801C
:10BD700008EE241912BB5FF5118E828F83A3E0F8C1
:10BD8000E50A28F50CE4350BF50D750E00780C125C
:10BD90002A1DAC11EC2CFCE433FD7A337B13123CEE
:10BDA0009D7403122A34EE241BF582E43FF583745C
:10BDB00033F0A37413F0E511C333F88508828509C5
:10BDC00083E028800412C989E4F08E828F83A3E087
:10BDD000F88E828F83E0C398500479008062A3E0DC
:10BDE000FAE50A28F8E4350BF9EE241D12E25FA308
:10BDF000E912C0E9C39AC0E012BE42D0E012C8887E
:10BE0000603CEE2417F8E43FF9880889098882F538
:10BE100083E024F2F0EE241D12BB63240EFAA3E0AB
:10BE20003400FB8882898312DA2F90053FE0F912F3
:10BE30002E09E9F8850882850983E0C398F0A90FE7
:10BE40008033EE2417F582E43FF583228E828F83C0
:10BE5000A3858208858309E0F8E50A28F582E435A0
:10BE60000BF583E02212B65EA3A3A32212CB9C049F
:10BE7000F022122A347F0A0226BD74F412242E8A7C
:10BE8000088B09EA12BF01F0EA1313543F12BEFAFD
:10BE9000A3A3A3F0EAC4131312BF01A3A3F0EB12F0
:10BEA000BF0C12BF147409780A122C5212BF0A1266
:10BEB000BF13740A780A122C52E50A5401C0E0EC50
:10BEC0002418F582E43DF583D0E012BF19740B7895
:10BED0000A122C5212BF0AA312BF13740C780A1252
:10BEE0002C5212BF0AA3A3A3A3A3A3A3A3F0740D70
:10BEF0007808122C52A908029863540F8C828D8303
:10BF00002254038C828D83A3A322E50A54018C82E0
:10BF10008D8322A3A3A3A3A3A3F08A0A8B0B22C021
:10BF200082C08379008A828B83A3A3A3A3A3A3E007
:10BF300090053E600EE070228A828B83A3A3E0709E
:10BF4000198016E060148A828B8312D332900547E1
:10BF5000E06A7003A3E06B60010902C16074F01233
:10BF6000242E8A0A8B0B890C8C088D098A828B837C
:10BF700012C0BE1232C512C0A08508828509831284
:10BF8000C0F0E50812B735350912C0DAC0E0E5089F
:10BF9000241112C880D0E012C0D2C0E0E5082412FB
:10BFA00012C880D0E012EE46740812C0CCE0601EC9
:10BFB000E50A2408F8E4350BF9E508241312C880D3
:10BFC00012C89D850882850983A3E02408F08508AE
:10BFD00082850983A3A3A3A3A3A3A3A3E0601B85D6
:10BFE0000882850983A312C0AFE508241512C88012
:10BFF000E8F0A3E912C0E92408F0850882850983E6
:10C00000A3A3A3A3A3E06019850882850983A3AE37
:10C0100082AF8312BE5785088285098312C0E4046B
:10C02000F0AA08AB091232CBE9F50D7061850882E0
:10C03000850983A3A3A3A3A3A312C093701AE0FA54
:10C04000E50A2AF8E4350BF9E508241D12C8801228
:10C05000C89DE50CC39A802A12C0AFE8240EF850A0
:10C060000109E508241D12C88012C89D90053FE013
:10C07000F9122E098E828F83E0F8E50CC39824F222
:10C08000C399C0E0E508241712C880D0E0F0A90DDC
:10C0900002C12812C09722E0850882850983A32265
:10C0A000850A82850B83A3A312C106E0F9EA22AEBA
:10C0B00082AF83E0F8E50A28F8E4350BF922E0FACC
:10C0C000A3E0F8E4C8F9EA28E439FB2212EE29A338
:10C0D000A32212C119A3A3A3E022F583E812C1127F
:10C0E000A3A3E022A3A3A3A3A3F08E828F83E022C5
:10C0F000A3A3A3A3A3A3A3A3A312C11212C106A324
:10C10000A3E0F9EAF822E0FA850A82850B83A3A36B
:10C11000A322F0A3E912C11922F0850A82850B83BC
:10C12000A3A3A3A322122A347F080226BDC082C083
:10C13000837AC57B0579E21248677AC57B05802042
:10C14000C082C0839005478014C082C08390054A96
:10C15000800BC082C083794A124867800312D33BA8
:10C16000D083D0820229E674F612242E9005CDE009
:10C17000FE04F0EEF912326B8B09EA450970EDEE20
:10C1800060EAF902C4D474EE12242EEAFEEBFF8CAE
:10C190000E8D0F890A750B00750C001234698A0820
:10C1A0008B097412122CC7E0F5107413122CC7E01F
:10C1B000F50DEA45097017E50D600302C2AAA90A48
:10C1C000AC0EAD0FEEFAEFFB12348D02C3B8E50DE5
:10C1D000700302C27090099AE060046401700E90CE
:10C1E00005DA12CB81600612C5EB124AEEE510703B
:10C1F0000B850882850983E4F002C2A590099AE0C4
:10C2000060076401600302C2CD900541E0A2E140F5
:10C210000302C2CD9005DC12CB81600CA910AA08E4
:10C22000AB0912C5EB124AEE850882850983E0FA54
:10C2300012E272500109C3EA98E499A2D265D033A0
:10C240005009850882850983E004F0850882850904
:10C2500083E0F89050A3E493687072750B01EEFAD6
:10C26000EFFB12315D850882850983A3E4F0805DD0
:10C27000E5107021EA2402F582E412DEC5850A0E7B
:10C28000250EF8E4340013E813F070098A828B83DA
:10C29000A3A37401F08A828B83A3A3E0F89015FB1B
:10C2A000E0C3985028750C0180237401650D701D42
:10C2B000E510601990099AE060046401700F900520
:10C2C00041E0A2E15007EEFAEFFB12315D90099ACE
:10C2D000E06402600FE060046401702A900541E0B0
:10C2E000A2E140227401650D701CE5109005EC6020
:10C2F00013E004F09015CEE0F89005ECE0C3984010
:10C3000005750B01E4F0E50CA2E092F0E50BA2E06C
:10C3100072F0400302C3B890099AE06004640170AF
:10C3200041900541E0A2E15039EEFAEFFB122EC92F
:10C330008A088B09A808A909E8496026E50CA2E04B
:10C34000500D88828983A3A3A3A3A3E0C2E0F0E5F4
:10C350000BA2E0506388828983A3A3A3A3A3E0D2A6
:10C36000E0F0E50BA2E0505090099AE0600464010F
:10C37000701D900541E0A2E15015EEFAEFFB122E80
:10C38000B7E9600BEEFAEFFB7900123001802990DB
:10C39000054AE06E7003A3E06F701DEEFAEFFB79C3
:10C3A0000112300190099AE06402700C7A017B005E
:10C3B0009005A1E0F9123E3502BE7574F412242EE8
:10C3C00074016A4B700E7A017B009005A1E0F912AE
:10C3D0003D0380379015C512DA2FEA4B60218A0899
:10C3E0008B09E4F50AF50B7808122A197A017B000B
:10C3F0009005A1E0F9123E297404122A34800C7AC7
:10C40000017B009005A1E0F9123E35029863C082DD
:10C41000C0839015C702AA6DC082C0839015C9025F
:10C42000AA6D74F612242E75083375090578081262
:10C430002A217C6E7D007A217B00123DDB74021282
:10C440002A34E9F508122E3FE9420890099AE06083
:10C450000464017006122EF3E9420890071012CB13
:10C4600081600912C5EB124AEEE94208122D7FE9FC
:10C47000FE124309E9F8E5084E48F9805774F612B0
:10C48000242E1247777508337509057808122A217A
:10C4900075086E7509007808122A217C007D007AE3
:10C4A000217B00123DE77404122A34122E459009B4
:10C4B0009AE0600464017003122EF990071212CB07
:10C4C00081600612C5EB124AEE122D8512431B80C5
:10C4D00003122A347F020226BD74F612242E74FF42
:10C4E000122AC87E007508337509057808122A21BA
:10C4F0007C6E7D007A217B00123DDB7402122A34AF
:10C50000E9600302C5BC7808122A2175086E8E09FD
:10C510007808122A217C007D007A217B00123DEDF3
:10C520007404122A34E9600302C5BC900547E06434
:10C53000FE7003A3E0F4700302C5BC0E900556E044
:10C5400064086005E06404706F851882851983EEC5
:10C5500012C9E7794212486D7A5E7B057943124829
:10C560006D7A5B7B05794712486D7A4C7B05794A79
:10C5700012486D7A4A7B05794B12486D7A547B05D7
:10C58000795012486D7A477B05795312486D7A5C71
:10C590007B05795412486D7A497B0579E112486D23
:10C5A000900541E0A2E35004D2F08002C2F012C92B
:10C5B000DD795212486D80041247771E122E4B907F
:10C5C000099AE0600464017003122F0B90071412A3
:10C5D000CB81600612C5EB124AEE122D91EEF97472
:10C5E0000102C4D18E828F83E0F8A3E0F5838882B4
:10C5F0002274F612242EE9FEA2E050267508337547
:10C6000009057808122A2175086E75090078081244
:10C610002A217C007D007A217B00123DE774041200
:10C620002A34EEA2E35003122E5190099AE06004DE
:10C6300064017008EEA2E15003122F11EEA2E25045
:10C640000E90071612CB81600612C5EB124AEE025D
:10C65000C4D474F612242E74EC122AC87401122A5F
:10C66000AA901572E0F97AA47B0512321D90059309
:10C67000E06402707C7405122CC7E4F07407122C7D
:10C68000C7E4F07A04F9122EA58A08905090E4933A
:10C69000FAC3E5089AEB9400400302C727122E99CB
:10C6A000E9600302C72790508312C78360157A049C
:10C6B0007903122EA5905090E493FC90508312C7FA
:10C6C0008D50087405122CC77401F090508112C768
:10C6D0008360157A027901122EA5905090E493FCA4
:10C6E00090508112C78D503F7407122CC77401807F
:10C6F0003590055F122CA4E8494A4B600474018010
:10C7000001E4C0E07405122CC7D0E0F0900563127C
:10C710002CA4E8494A4B600474018001E4C0E07431
:10C7200007122CC7D0E0F0901572E0F97CA47D05CB
:10C730007401122AA21232177AA47B057945124895
:10C740006D7407122CC7E070117405122CC7E070CD
:10C7500009851882851983E48008851882851983E4
:10C760007401F090156EE0F890156DE058F885189A
:10C7700082851983E05812C9E7794112486D741413
:10C7800002C4D1E493F8740193F9E84922E493F8E0
:10C79000740193F9ECC398F8E499F9C3EA98EB991A
:10C7A0002274F712242E74ED122AC8E9FE9005A017
:10C7B000F0AC18AD19901572E0F97AA47B0512322D
:10C7C0001D7412122CC7EE12C7DFAA18AB19123251
:10C7D000177AA47B05794512486D741302B154F0A1
:10C7E000901572E0F97CA47D052274F412242EEADF
:10C7F000FEEBFF901574E064FE7003A3E0F4706834
:10C800007A167B00123CC18A088B09EA45096058F8
:10C810008A828B83740112C8888A828B83A3600406
:10C8200074028002740112C8A3A3E08A828B83A3DE
:10C83000A3A3A3A3A3A3A3A312C8B9FCA3E0FDEAE7
:10C840002402FAE43509FB12479BE508241312C8B9
:10C8500080E4F0AA08AB099005A1E0F9123CCD12E2
:10C86000C86B12D0EC12C89D02986312C86F22EEFA
:10C87000240BF582E43FF58322850A0CE508250C9C
:10C88000F582E43509F5832212C88DE022F08E820C
:10C890008F83A3A3A3A3A3A322E012977DE8F0A311
:10C8A000E9F022F0EE241DF582E43FF58312C8B1D1
:10C8B0002212D101F583888222A3F0EE241512B64C
:10C8C000282274F212242E74FD122AC88A088B09B9
:10C8D000890A8C0B7401122CC7740412C9E7123335
:10C8E0005B8A0C8B0DAE0CAF0DEE4F700302C97E50
:10C8F000EE12B7353F12C9AD7407F0A3A882A98321
:10C90000E5082413FAE43509FB8A828B8312C9BE39
:10C910008A828B8312C9BDE50812D32812DEC5882E
:10C9200082898312C9C97401F0E508240BF8E43543
:10C9300009F9EE12C98912C9D612EDC61232D71200
:10C94000DA26EE241312EDC87403650A600674013A
:10C95000650A700712C9997404800412C999E4F039
:10C9600090157412ACFF12C89D7401650B7006EE31
:10C97000241112C990EEFAEFFB122F4180027910B8
:10C98000901574129B5402D10812EE1222EE24125A
:10C99000F582E43FF583E4F02212C9A17440F0A3CC
:10C9A00022EE12DEB73FF5832212EDEC3BF5831247
:10C9B000C9B322E0F8A3E0F98882898322A3E08842
:10C9C000828983F0A308A98322F0EE2416F582E47D
:10C9D0003FF58322A3A3E8F0A3E9F0EE22A2F0E45E
:10C9E00033851882851983F0AA18AB192274F412C2
:10C9F000242EEAFEEBFF7A007B049005A1E0F912F9
:10CA00003E3512CA8B12C89D9005567409F0123239
:10CA1000D78A088B09AC08AD0912CA7D12D33B1224
:10CA20004795E9640170537A0F7B00123CC18A0874
:10CA30008B09EA450960438A828B837402F012CA2B
:10CA400095FC88828983A3A3E0FBEC8A8285098315
:10CA5000A3A312DA3088828983A3A3A3E08A828504
:10CA6000098312C8B9FAA3E0FB794A12486DAA08F3
:10CA7000AB099005A1E0F9123CCD02986312CA817E
:10CA800022EE2413F582E43FF5832290051912D09B
:10CA9000FC9015C922EE241DF582E43FF58312CDEA
:10CAA00066E02274F412242E74FD122AC88A088BC0
:10CAB000097401122CC7740212C9E712335B8A0A87
:10CAC0008B0BAE0AAF0BEE4F700302CB6D12EE3143
:10CAD000700888828983A37420F085088285098381
:10CAE000A3A3A3A3A3E06401700988828983A3E0C0
:10CAF000D2E6F0850882850983A3A3A3A3A3A3E0BC
:10CB00006401700A88828983A3E0D2E7800312ED72
:10CB1000A812EE227019850882850983A3A312CB7F
:10CB2000816006EE241612EDC812EE0412C89D852F
:10CB30000882850983A3A3A3A3A3A3A3E064017030
:10CB40000312EDD985088285098312D33B1233790C
:10CB5000E9600312EDD212EDC51232D712CB871263
:10CB6000CB7312C9D4FAEFFB122F41800279100265
:10CB7000BC2FE0F8A3E0F98E828F832212B248F531
:10CB80008312D0FCE8492212CB92EAF0A3EB12CB3D
:10CB90009C22EE241AF582E43FF58322F085088278
:10CBA000850983E02274F512242E74F3122AC889B1
:10CBB0000AEAFEEBFF7508007509007C0D7D00791F
:10CBC00000AA18AB19123CA9EE12D71C3FF583122C
:10CBD000CD52741F58600C7AD37B0012437B7900CE
:10CBE00002CCA4E8A2E55008740C122CC77401F022
:10CBF000E8A2E75008740B122CC77401F0E8A2E613
:10CC0000740A5008122CC77401F08008122CC7E077
:10CC1000640170138E828F83A3A3A3A3A3A3A3E0B5
:10CC20006032EE241380128E828F83A3A3A3A3A36A
:10CC3000A3A3A3E0601EEE2415F582E43FF5831262
:10CC4000A6C96010AC08AD097402122CC7AA82AB49
:10CC50008312479B12C86B12C899740A122CC7E042
:10CC60006401703712D32E123379E97035EE240B3C
:10CC700012B8AE90054AE0687003A3E0697023E53E
:10CC800008450960161232D7EAFCEBFD7402122C3B
:10CC9000C7AA82AB83124795E96007AA18AB19129D
:10CCA0002FFBA90A02EF3974F712242E74D2122A2C
:10CCB000C8EAFEEBFF8E828F83129CF5A2E0400350
:10CCC00002CD4D12CD59E054FE12E680740D122AA9
:10CCD000AA12CD761232D1E97073742A122CC712BF
:10CCE000CD7070697C0D7D007900AA18AB19123CDB
:10CCF000A97416122CC712C899742A122CC712CD07
:10CD000052A2E55008740B122CC77401F0E8A2E798
:10CD10005008740A122CC77401F0E8A2E65004749B
:10CD20002080027422122CC712B05C7402122CC72D
:10CD3000AA82AB8312479B8E828F83A3A3E0C0E0BD
:10CD4000740C122CC7D0E012C9E7122FF5742E0212
:10CD5000B15412C8B1A3E0F8228E828F8312CD663F
:10CD6000A3A3A3A3A32212D101F988828983A322BA
:10CD700012B227640422EA241EF582E43BF583E024
:10CD8000F9EA241FF582E43B12985722E9F879006A
:10CD9000740468600A740A686005740368700109A5
:10CDA0000229E674F612242E8A828B837420F0A363
:10CDB000A37401F0122F478A088B09AE08AF09EE61
:10CDC0004F60168E828F837401F0900594E0700995
:10CDD00012EDC51232D712DA26EEFAEFFB02C4D4F6
:10CDE000C082C08390054402AA0CC082C083901503
:10CDF0007302AA0CC082C083E990157302AA71C0A5
:10CE000082C0839005B97401F0E9A2E35003740372
:10CE1000F0E9A2E15004E0D2E2F002C16074F6123F
:10CE2000242E79007C008A088B097808122703F8E1
:10CE3000FF074ECE4CCE4CCE4CCE4CCE44CE48CE40
:10CE40004ECE49CE7C0480060C0C80027C089005F6
:10CE5000B9E05C6003098003EC60010902C4D4748A
:10CE6000F412242EEAFEEBFF8908122ECF8A0A8BD9
:10CE70000BA80AA90BE849604188828983A3A3A370
:10CE8000A3E06036C39405503174016508601A88C8
:10CE9000828983A3A3A3A3E06401600D88828983B0
:10CEA000A3A3A3A3E06402700A8882898312A7A6C1
:10CEB000124AEEEEFAEFFB122EDB02986374F612C2
:10CEC000242E8A828B83E07012A312CB81600C8A9D
:10CED000828B8312D33A124A4180047A007B00028B
:10CEE000C4D4C082C083900593E06402700B9005A7
:10CEF00056E06408700312339D02C160C082C08393
:10CF00007C00EC12CFAF7003A3E06B7011905093D4
:10CF1000E493C0E012CF7ED0E0F079C580510CECF4
:10CF2000C3940340DD7C00EC75F003A4F8A9F07411
:10CF3000BD28F582740512974064FE7003A3E0F4E7
:10CF4000600F0CECC3940340DE7C00EC12CF7270D7
:10CF500015EC12E31912DA2F905093E4938882892A
:10CF600083F0790080090CECC3940340DE79C7029A
:10CF7000C16075F003A4F8A9F012CF7EE02274BC62
:10CF800028F582740539F58322C082C0837D00EDC7
:10CF900012CFAF7003A3E06B700912CF79600479F0
:10CFA0000180090DEDC3940340E5790002C160756D
:10CFB000F003A4F8A9F074BD28F582740512E7D235
:10CFC0006A2274F212242E74DD122AC8EAFEEBFFE4
:10CFD000750A0090099AE060076401600302D0E6D8
:10CFE000900547E06E7003A3E06F701EEE4F700374
:10CFF00002D0DA9005CE12CB81700302D0DA750A26
:10D000000112C5EB124AEE02D0E6122EC98A088B35
:10D0100009EA4509700302D0DA8A828B83A3A3A3AD
:10D02000A3E0640160108A828B83A3A3A3A3E064BE
:10D0300002600302D0DA851882851983E412D0F3E6
:10D04000740B122CC7E8F0A3E912C9E7122E8DE980
:10D05000700302D0DA85088285098312D0EC12C8E9
:10D060009D79001230A985088285098312DA2F7410
:10D0700003122CC7AC82AD837418122CC7AA82ABE2
:10D080008312479B85088285098312B8B4742012E5
:10D090002CC712C89D7422122CC7E4F07C028508AC
:10D0A00082850983A3A3A3A3E0F9740D122AA21217
:10D0B000333785088285098312B8B47401122CC7EE
:10D0C000E8F0A3E912C9E7122E93750A01E50824D6
:10D0D0000C12C8801297A1F0800C90055412B6462D
:10D0E000FAEFFB123451A90A7423801E12D0FC906F
:10D0F00015742212AE8F12D0FA22A3A312D101F915
:10D1000022E0F8A3E022A90A7403122A347F06025F
:10D1100026BDC082C08374FE122AC890099AE060BE
:10D120000464017029790190052C12C5E8124AEEB9
:10D1300012D153900547E8F0A3E912C9E7795312D9
:10D14000486D85188285198312D33B123F617402A2
:10D150000284A7851882851983EAF0A3EB12D162B5
:10D16000F92212BC4EF8A3E02274F512242E74F3B7
:10D17000122AC88A088B09ECFEEDFF750A12EA45EF
:10D18000097005790002D276900547E065087004C1
:10D19000A3E0650970191232D7EAFCEBFDEEFAEF55
:10D1A000FB124795E97005750A018003750A008531
:10D1B0001882851983E4F004122CC7E508F0A3E572
:10D1C0000912C9E7122E81E960297403122CC7AA3B
:10D1D00082AB83122E5DE964017018750A01740335
:10D1E000122CC7AC82AD83EEFAEFFB124795E970C3
:10D1F0001E801F7412650A7019900593E064027016
:10D2000011EEFCEFFDAA08AB09122EB1E96003751F
:10D210000A00EEFCEFFDAA08AB0912346FE9F874BE
:10D220000A687005750A01804274A0687037EEFCC8
:10D23000EFFDAA08AB091234817E008023EE75F061
:10D2400017A4F8A9F012E7E87004A3E06509700FCD
:10D2500012E924122E5DE9700612E4C312345D0E49
:10D2600012D27940D87401650A70097900AA08AB16
:10D27000091233AFA90A02EF3990508BE493F8EE0C
:10D28000C3982274F612242EEAFEEBFF8908900957
:10D290009AE060046401701E12339DE508F5097878
:10D2A00009122A25790DEEFCEFFD7AFC7BFF123383
:10D2B000BB7401122A3402C4D474F712242EEAFE7D
:10D2C000EBFF8E828F83A3A3A3A3A3A3A3A3E060FA
:10D2D0001312D32012984A1233A9E964017005127F
:10D2E000C86B802D8E828F83A3A3A3A3A3A3A3E0E7
:10D2F000602912CA7D12D33FFAA3E0FB1233A9E9D9
:10D30000640170178E828F83A3A3A3A3A3A3A3A3F7
:10D31000A312D33B12339179018002790002B157F5
:10D32000EE12D3283FF583222415F582E4228E8263
:10D330008F83A3A3A3A3A3A3A3A3A31298592212E9
:10D34000D34BA3A3A3A3A3A3A3E02212B0648E8212
:10D350008F83A3A32274F212242E74FD122AC88A8A
:10D36000088B09ECFEEDFF890B750A017401122C84
:10D37000C7740412C9E712335BEA4B604774111299
:10D380002CC7E0601AEA2417F582E43BF583E41227
:10D39000DBDB8A828B83E0D2E7F012D3C7E4F012A2
:10D3A000C9A9740312D635EE88828983A3A3F0EF4E
:10D3B00088828983A3A312AE8AA3A312F016122F28
:10D3C00041E9F50A02D106EA2414F582E43BF5832B
:10D3D0002274F012242EEAFEEBFF890A750B01126B
:10D3E000CA95F50C88828983A3A3E0FA8882898391
:10D3F00012D50E12BB5C6404600A7AD37B00124320
:10D400007B02D509E50C1228CA0200021ED4030BC8
:10D41000BED4030CA5D40D7DD40EBED4BCD49009CB
:10D420009AE060076401600302D4BE900541E0A267
:10D43000E1400302D4BE7900AB0912313FEA4B60F0
:10D44000318A828B83A3A3A3A3A3A3E054186022F1
:10D4500012C86B1228458A828B83A3A312284579B0
:10D46000008E828F8312D52D1231577404122A3404
:10D47000802E7901AA08AB0912300D804190099ADB
:10D48000E0600464017037900541E0A2E1502FABE9
:10D490000912338BAA08AB09123391E964C5701ED7
:10D4A000750B00801990099AE060046401700F9078
:10D4B0000541E0A2E15007123F858002880AEE2470
:10D4C00009F50EE43FF50FAC08AD09A90C850E82F5
:10D4D000F58312D33B123025850E82850F8312D33C
:10D4E0003B123379E96022EE241112BB5FC3940230
:10D4F000401712C86B12DAF57003A3E069600AE501
:10D500000BA2E05004A90A8002790002C128A3A35B
:10D51000A3E0F8E4C8F9EA28F508E439F50922E5BA
:10D5200008240CF582E43509F58312B604A3A3A3FD
:10D53000A3A3A3A3A3A312B0608A828B83129859DA
:10D540002274EE12242E74F5122AC88A0A8B0B89D3
:10D550000C8C0E8D0F7E01EE122CC7740AF0741D18
:10D56000122CC7E0F50DE9700FE50DC333240AC096
:10D57000E0EE122CC7D0E0F0AA18AB1912335B8A88
:10D58000088B09EA4509700302D62A12B734350917
:10D5900012D7B7740912D7C3450D12D655AC0EADCC
:10D5A0000FEEFAEFFB12479BEE2408FE50010FE549
:10D5B0000C70247C00741E122CC712B8B48012ECBC
:10D5C00012DAE1E82AFAE93BFB12D63BA30EAF835D
:10D5D0000CECC3950D40E8E508241712C8807401CF
:10D5E000F01232D7E508241AF582E4350912DA2D53
:10D5F0007403122AAAAA0AAB0B122E69E96019E574
:10D6000008241612C8807401F07403122A9AE508DF
:10D61000241812C88012C89D85088285098312D6F5
:10D6200031AA08AB09122F41E9FEEEF9740B02BED4
:10D6300072A3A3E50AF0A3E50BF0228A828B831282
:10D64000D64F12D6558A828B8312D64EF022A3E093
:10D650008E828F8322F0A3AE82AF832274F01224D5
:10D660002E74F8122AC88A088B0912D71B350912A2
:10D67000D83CF50B880AA3AE82AF83EEFCEFFDAA7F
:10D6800018AB1912479BEE2408FE50010FAC18ADE1
:10D69000197A687B05124795E9607474E0550A7041
:10D6A00067AA0BEA2AFA7B00123D638A0C8B0DEA0B
:10D6B000450D605B7C00801E8E828F8312C0BEECA5
:10D6C00012D714E50C28F582E50D3912DA2DEE2477
:10D6D00002FE50010F0CECC3950B40DC780C122AB3
:10D6E00021780B122A257403122AAA7900E508244E
:10D6F0000B12C88012D33B1233D37403122A34AAFC
:10D700000CAB0D123D6980077AD37B0012437B740A
:10D710000802C12525E0F8E433F922EA241DF58248
:10D72000E42274F012242E8A0A8B0B890C8C088D4B
:10D73000099007E512CB81607B7410122CC7E0F5CD
:10D740000D12D714E8240EFAE439FB123CC18A0EFC
:10D750008B0FAE0EAF0FEE4F605A8E828F8374D454
:10D76000F0A3A3E50AF0A3E50B12BE65E50CF0AC4F
:10D7700008AD09EE2405FAE43FFB12479B12B23BC9
:10D78000E50DF07411122CC712DBC57808122A1DA2
:10D79000AC0DEC2CFCE433FDEE240EFAE43FFB125E
:10D7A0003C9D7403122A34EEFAEFFB9007E512C594
:10D7B000E8124AEE02C128F583E0FEA3E0FF8E8264
:10D7C0008F8322F0A3E50CC43354E02274F61224B4
:10D7D0002E74F8122AC8890812D71B3B12D83CF9BC
:10D7E0008809A3AE82AF837401697042EEFCEFFD3D
:10D7F000AA18AB1912479BEE2408FE50010FAC1873
:10D80000AD197A687B05124795E9602974E05509DE
:10D81000701C8E828F83A3E0FA8E828F83A312C046
:10D82000C08E828F83E0F91233EBA90880097AD386
:10D830007B0012437B7900740802C4D1F583E02495
:10D8400001FEA3E03400FF8E828F83E0F8741F583E
:10D850002274F612242E74DF122AC8EAFEEBFF129D
:10D86000CB7C60508E828F8312D33BAC18AD1912E3
:10D87000CD761232BF7409122CC712DAF57003A3E9
:10D88000E069603012C5E41228457508FE7509FF8D
:10D890007808122A21741C122CC7E0F9740D122C7E
:10D8A000C712B05C740F122CC712D33B12315774DD
:10D8B00004122A34742102C4D174F712242EE9FC14
:10D8C0007A007B007E00800B12D95BE02AFAA3E08D
:10D8D0003BFB0E90509012D27C5029EE75F016A4AE
:10D8E000F8ADF0EDF912E7D7F460E774A528F582FA
:10D8F000740E3912CB7F60DAEC60CD12D95BE4F0A4
:10D90000A3F080CE7E00800B12D948E02AFAA3E073
:10D910003BFB0E12D279502DEE75F017A4F8ADF046
:10D92000EDF912E9357003A3E0F460E6747828F5A8
:10D930008274103912CB7F60D9EC60CC12D948E4E4
:10D94000F0A3F080CD02B157EE75F017A4F8EDF911
:10D95000747828F582741039F58322EE75F016A4D8
:10D96000F8EDF974A528F582740E39F5832274EC6C
:10D9700012242E890CEAFEEBFF9005A0E0C3950C63
:10D98000503B12332B9005D012DA2090053AE0F587
:10D9900008E4F509F50AF50B9080B47810122C70A4
:10D9A0007808791012233F7808122A197A007B022E
:10D9B0009005A1E0F9123E297404122A3402973826
:10D9C00074F612242EEAFEEBFF9005BA80138882CB
:10D9D0008983E06E7003A3E06F603688828983A339
:10D9E000A312CB8170E87A047B00123D638A088B16
:10D9F00009A808A909E84960188882898312DA20F1
:10DA00009005BA12DA14A3A312DA2F9005BA12C83D
:10DA10009D02C4D412985988828983228A828B837A
:10DA2000EEF0A3EFF022EE241AF582E43FF583EA4C
:10DA3000F0A3EBF02274F412242E7E009005BA803D
:10DA4000070E88828983A3A312CB8170F4EE12DAC9
:10DA5000E1123D638A088B09EA4509607E7F0090E8
:10DA600005BA80218882898312B05CEF12DAE1E581
:10DA7000082AF582E5093BF583ECF0A3EDF00F8869
:10DA8000828983A3A312CB8170DA90059C12DAF508
:10DA90007003A3E0697808701C122A21EEF50A7859
:10DAA0000A122A257C687D05790090059C12D33BDB
:10DAB0001233D3801A122A21EEF50A780A122A2587
:10DAC0007C687D05790090059C12D33B1233C774A6
:10DAD00003122A34AA08AB09123D69122F59029881
:10DAE0006325E0FAE433FB228E828F83A3A3A3A3F2
:10DAF000A3A3A3A3A312D0FC900547E06822C08291
:10DB0000C08380128A828B83A3A312B8B49005BA13
:10DB100012C89D123D699005BA12AFFF70E602C1AE
:10DB20006074F512242E90055412B8BB9005D012E3
:10DB3000DBB912C89D7AD07B05795012486D9005EB
:10DB4000D012DBC5801512E37765087004A3E06589
:10DB500009600612E4CB12345D050A12DBAE5018E0
:10DB6000E50A12E4B77003A3E06F70DA746D28F56C
:10DB700082741012F01380E19005D012B8BB9007A8
:10DB8000E712CB8160257A067B00123CC1EA4B602C
:10DB90001A8A828B8374D5F0A3A3E412DBCC04121F
:10DBA000DBDB9007E712C5E8124AEE02EF3E905029
:10DBB0008BE493F8E50AC3982212DBBD2212D1014F
:10DBC000F99005542212ACE6750A002212DBD0222D
:10DBD00012DBD42212AE8FA3A3A32212DBD0A3EEBA
:10DBE000F0A3EFF022C082C0839005D27415F0A399
:10DBF0007434F09005D4740FF0A37434F09005D60B
:10DC0000742DF0A3743402AA71C082C083900547BA
:10DC1000E064FE7003A3E0F4600E900541E0A2E131
:10DC2000500612347512341B02C16074F012242E97
:10DC3000900595E06053F50CE4F50DF50EF50F90A9
:10DC400080A47808122C70780C790812233F123CBB
:10DC5000BB8A088B09A808A90990507DE49358F560
:10DC600008A3E49359F509E4F50AF50B780C790853
:10DC7000122B92780C122A197A007B019005A1E0F0
:10DC8000F9123E2F7404122A3402C12874EE1224B1
:10DC90002E7E007F008E0A8E0B122F1D8E0D803E71
:10DCA000850D08AA087B00122F178A088B09A8087F
:10DCB000A909E849602688828983A3A3A3A3E06019
:10DCC000046404701788828983A3A3A3A3A3A3A3D6
:10DCD000A3A3A3E0F9123487E960010F050D90506A
:10DCE00090E493F8E50DC39840B612344B8A0E8B3E
:10DCF0000F8E0C8023AA087B001234578A088B09E8
:10DD0000A808A909E849600EE8240F12973DF91206
:10DD10003487E960010E050C850C08C3E508950EF3
:10DD2000E4950F40D0EF2EFE700302DE258E0875BD
:10DD3000090074027808122BDEAA08AB09123D63B1
:10DD40008A0A8B0BEA450B700302DE23750C008EEA
:10DD50000875090074027808122BDEAC08AD097949
:10DD6000FF123CA9750D00805D850D08AA087B0097
:10DD7000122F178A088B09EA450960488A828B832B
:10DD8000A3A3A3A3E06004640470398A828B83A3F5
:10DD9000A3A3A3A3A3A3A3A3A3E0F9123487E960D9
:10DDA00023050C780A122A21EEFD85088285098355
:10DDB000A3A3A3A3A3A3A3A3A312DECB1234217412
:10DDC00002122A34050D905090E493F8E50DC398A3
:10DDD0005006E50CC39F4091750C00850C08C3E507
:10DDE00008950EE4950F503DAA087B001234578A1F
:10DDF000088B09EA45096027EA12DEB712DEC5F989
:10DE0000123487E96019780A122A21EEFDE5082408
:10DE10000E12C88012DECB1234217402122A34058D
:10DE20000C80B87E00750E6290053FE0600CF91220
:10DE30002E09E9F87454C398F50E75F003E50E84C5
:10DE4000F50D94204003750D1F850A08850B097593
:10DE50000C00E50E6006750C20750E00E50DC39EE6
:10DE60005004AF0D8008EEFFE50CD2E6F50CAC08CF
:10DE7000AD09AA0CEFF9123427E9F50FE50CA2E67B
:10DE8000401A1F7800800BE5082404F508500205AD
:10DE90000908E8C39F40F0EFCEC39EFEE97006E597
:10DEA0000CA2E650AAE50A450B6007AA0AAB0B12C2
:10DEB0003D69A90F02BE75240FF582E42274002586
:10DEC00008F58274143509F583E022E0FC850882A8
:10DED0008509831298592274F212242EEAFEEBFF70
:10DEE00089088C098D0A7C007D00740E122CC712E3
:10DEF000D33B8C0B800DEAFCEBFDEA2404FA5001C5
:10DF00000B050BE50BC3950A400302DFA28A828B47
:10DF100083E0F47003A3E0F46077EC4D600C8C8236
:10DF20008D83C3E09EA3E09F50CC8A828B8312E254
:10DF3000E6EE98EF9950BFEAF8EBF988828983E022
:10DF4000F47003A3E0F46010E82404F8500109051C
:10DF50000BE50BC3950A40E3E8FCE9FDE824FCF877
:10DF6000E934FFF9888289831297928C828D83E548
:10DF70000CF0A3E50D12DFA58C828D83A3A312E61E
:10DF80007AE08C828D83A3A3A3F0C3EA98EB994037
:10DF9000C712DA1C8A828B83A3A3E50912DBCCE5C6
:10DFA00008F002D10D12DFABA3E022F08882898352
:10DFB000A32274F212242E74FD122AC889088A0939
:10DFC000ECFEEDFF750A0175F003E9A42402C0E040
:10DFD0007401122CC7D0E012C9E712335BEA4B6020
:10DFE0007812C9A97408F0741F55084509A3F0E810
:10DFF0002402F8500109750A0080388E828F83E070
:10E0000088828983F0A3A882A9838E828F8312C914
:10E01000BD8E828F83A3A3E05407C4FC8E828F83BE
:10E02000A3A3A3E054074C12C9BFEE2404FE500181
:10E030000F050AE50AC3950840C18A828B83A3A312
:10E0400074FCF0A374FFF0EA2413F582E43BF5833B
:10E050007401F0122F41E9F50A02D10674F112247D
:10E060002E8A0A8B0B7508007AFE7BFF7CFE7DFFF3
:10E07000E50A12D71C350B12CA9CF509741F550905
:10E08000F50CE82402F8500109E509A2E7406FE524
:10E090000A2417F582E412E256FE75F003E50CA49B
:10E0A00024026E7059E50C600B88828983E0FEA320
:10E0B000E0FBEEFA750D00801DE05407F50EA3A8F5
:10E0C00082A983EEFC900547E06E7003A3E06F70B9
:10E0D00003850E08050DE50DC3950C502B8882892C
:10E0E00083E0FEA3E0FCE4CCFDEE2CE43DFFE8245D
:10E0F00002F850010988828983E0548860BB7AD392
:10E100007B0012437B02E24BE508700BA909123435
:10E1100033E9700302E24B12E26812D33B122EC9BC
:10E120008A0C8B0DAE0CAF0DEE4F605A8E828F8332
:10E13000A3A3A3A3A3A3A3E4F09050A393F88E8278
:10E140008F83A3A3A3A3A3A3A3A3E0C398402412F4
:10E15000E2725001097A027B00122247E88E828F18
:10E1600083A3A3A3A3A3A3A3A3F0E508C394075089
:10E170000205088E828F83A3A3A3A3A3A3A3A3A3B3
:10E18000E508F002E24B7CFF7DFF12E26812D33B10
:10E1900012343F8A0C8B0DAE0CAF0DEE4F704F1248
:10E1A00034458A0C8B0DAE0CAF0DEE4F700302E2BE
:10E1B0004B7C177D007900123CA912E26812CB72E9
:10E1C0001284998E828F83A3A3A3A3A3A3A3A312D4
:10E1D000C9D412B61D74AA12E2915001097A027BC9
:10E1E0000012224712B23BE812E27D7401F0905017
:10E1F000A3E493F8EE240D12BB5FC398401912E21A
:10E20000725001097A027B0012224712E25CE50893
:10E21000C394075002050812E8E3E50812E282E41D
:10E22000F0129C8A122E5DE97021850A82850B838B
:10E23000A3A3A3A3A3A3A3A3E06010E50A12D3287A
:10E24000350B12B644129C8B12479B02A8877400B0
:10E25000250AF5827414350BF583E022EE240DF5C2
:10E2600082E43FF583E8F022E50A12EDED350BF587
:10E2700083229050A3E49379002401F822F012E85D
:10E28000E722F012E28722EE240CF582E43FF583C8
:10E2900022F09050A3E49379002401F82274F7123D
:10E2A000242EE9FE74FE6A700374FF6B60347460A0
:10E2B0005E6460602DEEA2E5401CA2E6900547502A
:10E2C0000DC3E09AA3E09B5019790002B157C3E057
:10E2D0009AA3E09B40F390054712E2E6EC98ED9993
:10E2E00040E7790180E512D0FCC32274F712242E96
:10E2F0007E00800712E4C312345D0E12D27940F41E
:10E300007E00EE12E319129B5488828983E4F00E9A
:10E31000EEC3940340EC02B15775F003A4F8A9F0E2
:10E3200074BC28F8740539F988828983A32274F7AC
:10E3300012242E7F0080010F90508BE493F8EFC3DE
:10E3400098502DEF75F017A4F8A9F012E7C36A7082
:10E3500003A3E06B70E112E3776C7003A3E06D60E0
:10E360000A74FF6C700374FF6D70CC12E4CB8004F0
:10E370007A007B0002B15712E37B22746D28F5828C
:10E38000741012E7D22274F612242E7CFF7DFF7ADD
:10E39000FE7BFF12343FEA4B703C7508008032E58B
:10E3A0000875F017A4F8A9F0747228F58274101299
:10E3B0009740600512E7B87016746328FE74103930
:10E3C000FF8E828F8312D33B12315DEEFAEFFB0595
:10E3D0000812E3D940C902C4D490508BE493F8E505
:10E3E00008C39822C082C0837A007B007D00801021
:10E3F00012E92D7003A3E0F460050AEA70010B0D29
:10E4000090508BE493F8EDC39840E502C16074F43A
:10E4100012242E8A088B09ECFEEDFF800B12345D6E
:10E42000EEFCEFFDAA08AB0912343FEA4B70EE0296
:10E43000986374F612242E7D007E0080020D0E1269
:10E44000D2795018EE12E92E7003A3E0F460EF8D3C
:10E4500008EA65084B70E612E4CB80047A007B0082
:10E4600002C4D474F712242EEAFEEBFFEE4F601ABA
:10E470007C177D007900123CA98E828F8374FEF098
:10E48000A30412AD09A314129B5602B15774F712DC
:10E49000242EEAFEEBFF7508008014E50812E4B7AD
:10E4A0007003A3E06F600612E4CB12345D0508121E
:10E4B000E3D940E702B15775F017A4F8A9F012E3C9
:10E4C0007B6E22EE75F017A4F8A9F0746328FA7435
:10E4D0001039FB2274F412242E8A088B09ECFEED0D
:10E4E000FF90099AE0600464017020900554E06E8A
:10E4F0007003A3E06F7014122EC98A0A8B0BA80A4E
:10E50000A90BE8496005E82408801AEEFCEFFDAA93
:10E5100008AB0912343F8A088B09A808A909E84901
:10E520006009E8240DFAE439FB80047A007B0002DC
:10E53000986374F412242E8A0A8B0BECFEEDFF759F
:10E5400008007509008034E50912E91D122E5DE905
:10E550006027E50975F017A4F8A9F012E7E2700446
:10E56000A3E0650B700375080AEEFCEFFD12E924C9
:10E57000124795E960034308A0050990508BE49386
:10E58000F8E509C3985004E50860BC02BEF574F6CE
:10E5900012242E7E00805C8E08AA087B00122F17A2
:10E5A0008A088B09A808A909E849604688828983F6
:10E5B000A3A3A3A3E06401603988828983A3A3A3F2
:10E5C000A3E06402602CE8240712973DFA74012A44
:10E5D000F0900596E0C39A501988828983A3A3A37B
:10E5E000A3A3A3A3A3A3A3E412E671A312E680123C
:10E5F000315D0E90509012D27C409C7E008059EE8E
:10E6000075F017A4F8AAF0EAF912E9357003A3E04F
:10E61000F46044746328F8741039F9E8240C1297F4
:10E620003DF8740128F0900596E0C3985029EE75E6
:10E63000F017A4F8EAF9746328F8741039F9E812AD
:10E64000DEB739F583E4F0E8240EF582E439F5838A
:10E65000E412E68012315D0E12D27940A27B00EB0B
:10E6600012CF72600214F00BEBC3940340F102C4AA
:10E67000D412E67AA3A3A3A3A32212DFABA3A322FF
:10E6800012E688FAA3E0FB22F088828983E02274F4
:10E69000F312242E8A088B09ECFEEDFF750C007B2B
:10E6A000007C01740D122CC7E0F50AA3E0F50B8085
:10E6B00010123CBBE50CF5F0EA84ABF0750C007C65
:10E6C000007D0080010D90508BE493F8EDC39850CD
:10E6D0004912E92D7003A3E0F460EA12E7E8700440
:10E6E000A3E0650960DF12E7C36E7003A3E06F600B
:10E6F000D412E7E27004A3E0650B60C912E7B860CA
:10E70000C4C3940750BFEC050C70BAE50CC39B4022
:10E71000B4746328F582741080787A0080010A90BE
:10E720005090E493F8EAC3985070EA75F016A4F894
:10E73000A9F012E7EE64FE7003A3E0F460E012E7D4
:10E74000EE65087004A3E0650960D312E7EE6E7011
:10E7500003A3E06F60C812E7EE650A7004A3E065EA
:10E760000B60BB749E28F582740E12974060AFC395
:10E77000940750AA12E7D7640160A3E06402609E88
:10E78000EC050C7099E50CC39B4093749528F582B9
:10E79000740E39F58312D33B8019E50C6011EB70D0
:10E7A0000E7401650C600302E6B17B0102E6BC7ADF
:10E7B000FE7BFF7F050226BD747128F5827410125E
:10E7C000E7D22212E7C722746328F582741012E799
:10E7D000D22239F583E022749928F582740E12E76B
:10E7E000D22212E7C7650A2212E7C765082274958C
:10E7F00028F582740E12E7D22274F512242E8A08AC
:10E800008B09ECFEEDFF750A008002050A12DBAEF3
:10E810005022EEFCEFFDE50A12E91D124795E96072
:10E82000EAE50A75F017A4F8A9F0746328F5827474
:10E830001012F01302EF3EE9F87907C3940D40047B
:10E8400079018019E8C3940740047903800FE8C375
:10E850009403400419198005E8700279000229E642
:10E8600074F012242E8A088B098C0A8D0B890C12E5
:10E8700034458A0E8B0FAE0EAF0FEE4F60627C17E1
:10E880007D007900123CA98E828F8312F0168E8251
:10E890008F83A3A3A3A3A3A3A3A312D631E50C60E4
:10E8A0000712B61CE50C800512B61C7401F0900529
:10E8B000D412CB81601590059BE06401700612E8CC
:10E8C000E3E4800C12E8E37407800512E8E37401C6
:10E8D00012E2915001097A027B0012224712E25C97
:10E8E00002C12812E8E722EE240EF582E43FF58308
:10E8F0002274F712242E7E00801BEE12E92E700384
:10E90000A3E0F4600F12E924122E5DE9700612E410
:10E91000C312345D0E12D27940E002B15775F01780
:10E92000A4F8A9F0746528FA741039FB22ED75F08B
:10E9300017A4F8A9F012E7C764FE22C082C0839032
:10E9400005D8749FF0A37434F09005DA74A5F0A391
:10E950007434F09005DC74ABF0A3743402AA7174C3
:10E96000F712242EEAF8EBF990051712E9A8CA2449
:10E9700006F582E43AF583E0702B88828983A3A3AD
:10E98000A3A3A3A3A3A3A312284590051712E9AD3F
:10E99000122C9888828983A3E0F91230197402122C
:10E9A0002A34122F5902B157E0FAA3E02212E9A843
:10E9B000F5838A8222C082C08390059E12EA78F095
:10E9C00090059E12CB81700579011233E502C1607A
:10E9D00074F612242E74FC122AC8E9FE905094E4B6
:10E9E00093700874E16E600302EA73EA2408F8E4A5
:10E9F0003BF98882898312EA7812EA81700E9005C9
:10EA00009EE4F0A3F079011233E5806790099CE061
:10EA10006061FA90059E12E2E6EA98E49950547912
:10EA2000001233E58A088B09AC08AD09ECF8EDF962
:10EA3000E875F064A4F8AAF075F064E9A42AF990E6
:10EA4000059E12D33B12224FE8941AE9940040230A
:10EA50009007DF12CB81601B90059E12C89974024B
:10EA6000122CC7ECF0A3ED12C9E79007DF12C5E83E
:10EA7000124AEE740402C4D1E02401F0A3E0340091
:10EA80002212E688F8A3E0F9E84922C082C0837424
:10EA9000F8122AC890805AAC18AD1974081229626D
:10EAA000AC18AD19124795E9640170047900800231
:10EAB00079010284A574F612242E740C122CC7124C
:10EAC000B8BB743A6E7001EF6006743B6E4F7023F2
:10EAD000740A122CC71228458C088D097808122A4E
:10EAE00021EAFCEBFDEEFAEFFB123DED7404122A75
:10EAF000348002790A02C4D4C082C0839005DE74D7
:10EB000023F0A3742FF09005E07429F0A3742FF084
:10EB10009005E274C9F0A37434F09005E474CFF06A
:10EB2000A37434F09005E674D5F0A37434F0900526
:10EB3000E874DBF0A37434F09005EA74E1F0A37498
:10EB400034F074C9443460031234C902C16074F4EF
:10EB500012242E74E9122AC88A088B097404122C14
:10EB6000C77402F004122AA212335B8A0A8B0BAE1E
:10EB70000AAF0BEE4F700302ED9412EE317008886D
:10EB8000828983A37420F0850882850983A3A3A3C7
:10EB9000A3A3E06401700988828983A3E0D2E6F030
:10EBA000850882850983A3A3A3A3A3A3E0640170BE
:10EBB0000A88828983A3E0D2E7800312EDA812EECF
:10EBC000227019850882850983A3A312CB81600670
:10EBD000EE241612EDC812EE0412C89D8508828537
:10EBE0000983A3A3A3A3A3A3A3E06401700312ED6D
:10EBF000D985088285098312D33B123379E96003F2
:10EC000012EDD212EDC51232D712CB87FAA3E0FB78
:10EC10008E828F83A3A312DA2F123379E960031255
:10EC2000C98DEE241312BB5F700D905098E493C011
:10EC3000E012CA7DD0E0F08E828F83E0A2E750041C
:10EC400054038019EE241412BB5F7012900533E058
:10EC5000C0E012ED9ED0E0F0900533E004F012ED3C
:10EC6000B770199015D6E0600D90053EE0700D8EDE
:10EC7000828F83E07006EE241112C990AC18AD1992
:10EC8000EEFAEFFB1232B38A088B09EA45097003EA
:10EC900002ED887A217B00123D637406122CC712A4
:10ECA000DA2F7406122CC712CB81700302ED7C9010
:10ECB000099AE060046401700812B61CA3E04404E1
:10ECC000F07401122AA279501248677401122CC7FD
:10ECD00012B8B47406122CC712E9A8CA2409F58226
:10ECE000E43AF58312C89D90054712B8B474151222
:10ECF0002CC712C89D7406122CC712B8A612EDE3D9
:10ED0000F07406122CC712ADDB740212EE1B7406EF
:10ED1000122CC712E9AD12BC42C0E07406122CC717
:10ED200012B8A612EDAED0E0F0EE240E12EDC0C087
:10ED3000E07406122CC712EDF3D0E0F07406122C2A
:10ED4000C712862812F014EE240F12B8AE740C12FB
:10ED50002CC712C89D8A828B83E0C0E0740E122CEF
:10ED6000C7D0E0F07406122AA212322FE9F50A7415
:10ED700006122CC712D33B123D698003750A10AAF4
:10ED800008AB09123D698003750A10EEFAEFFB1219
:10ED90003D698003750A10A90A7417029860EE2471
:10EDA00014F582E43FF5832212CA81740122241EE5
:10EDB000F582E438F58322EE241112B6286401228C
:10EDC00012B60FE022EE2417F582E43FF5837401BA
:10EDD000F02212B6254404F02212C9A17401F0A356
:10EDE000E4F02212EDED38F583740222EA240BF5EB
:10EDF00082E42212EDF72212D101C8240CF582E43C
:10EE000038F5832285088285098312D0FAEE12EE46
:10EE100012222418F582E43FF5832212B65E12D046
:10EE2000FB2212EE29E064012212EE4AA3A3A3A35F
:10EE30002212C86F12C9B37404F0A3E412EE46A301
:10EE4000A3A3E064012212EE4A22F085088285091C
:10EE500083A32274F612242E7E00801F7C047D0082
:10EE600079FF8E088D0974027808122BDE74002554
:10EE700008FA74143509FB123CA90E90509A12D26C
:10EE80007C40D902C4D474F512242E74F7122AC817
:10EE9000750A00801E850A08750900740278081238
:10EEA0002BDE74022508F582741412C88312EF2C2D
:10EEB000F0050A90509A12DBB1506D850A08750969
:10EEC0000074027808122BDE12DEBDF47003A3E09A
:10EED000F460DE850A0875090074027808122BDEDA
:10EEE00074022508F5827414350912CB7F70A6745C
:10EEF00008122CC77402F0850A08750900780812F8
:10EF00002BDE74002508FE74143509FF8E828F8372
:10EF100012C89912EF351248B57C047D0079FFEED6
:10EF2000FAEFFB123CA980897409800FE024FFF0FE
:10EF3000A3E034FF2212F0A322740D122A347F03BF
:10EF40000226BD74F012242E74F7122AC8EAFEEBD2
:10EF5000FF8C088D09750CFF7408122CC712F095F0
:10EF60001248AFE9641A700302F00F750E00800BAF
:10EF700074FF650C7003850E0C050E90509AE49397
:10EF8000F8E50EC3985048850E0A750B0074027898
:10EF90000A122BDE12E24EF47003A3E0F460D18576
:10EFA0000E0A750B007402780A122BDE12E24E6E06
:10EFB0007003A3E06F70C2750F007402780E122BFD
:10EFC000DE7402250EF5827414350FF5838030E46B
:10EFD00093650E702D74FF650C602E850C0A750B01
:10EFE000007402780A122BDE7400250AF8741435B6
:10EFF0000BF98882898312DA2088828983A3A3127D
:10F00000F0167901740902C12512EF351248B5795D
:10F010000080F139F583E508F0A3E509F02274F4E6
:10F0200012242E74F7122AC8EAFEEBFF7408122C81
:10F03000C712F0951248B5750A008002050A905073
:10F040009A12DBB1504C850A0875090074027808E1
:10F05000122BDE12DEBDF47003A3E0F460DE850A3D
:10F060000875090074027808122BDE12DEBD6E707E
:10F0700003A3E06F70C67C047D0079FF8D0B7402E2
:10F08000780A122BDE7400250AFA7414350BFB1271
:10F090003CA902ADCB740212A4D8EEF0A3EFF0129B
:10F0A000F0A32290055412B064AA18AB1922C082B2
:10F0B000C08374F8122AC885188285198312DA2F42
:10F0C0007402122CC7E4F0A3F07404122CC774016C
:10F0D000F07405122CC77401F07406122CC7E4F00A
:10F0E0007407122CC7E412C9E71234C30284A57452
:10F0F000EE12242E8A088B09ECFEEDFF750C00EE53
:10F1000065087003EF6509600C123DE18A0A8B0BFC
:10F11000EA450B7006750C0102F1ABEEFAEFFB123B
:10F120003DE18A0E8B0FAC0EAD0FEC4D6007EEFA91
:10F13000EFFB123DF3E4F50EF50F780E122A21AC29
:10F140000AAD0BEEFAEFFB123DDB7402122A34E932
:10F150006059AA0AAB0B123D638A0E8B0FEA450F6A
:10F160006046780E122A21780A122A217C007D003E
:10F17000AA08AB09123DED7404122A34E9701D7817
:10F180000E122A21780A122A217C007D00EEFAEF65
:10F19000FB123DE77404122A34E96003750C01AADE
:10F1A0000EAB0F123D698003750C10A90C02BE75E1
:10F1B00074F712242E9007188008EAFEEBFF8A826B
:10F1C0008B8312FCA3EA4B603BEA2408F582E43B04
:10F1D000F583E014F070E312FE41EA687002EB6917
:10F1E0008A828B83700B12FE4A12F919123D6980D4
:10F1F000C412FE448E828F8312F919123D698E82E9
:10F200008F8380BE12F78C601AE0C812F783E01477
:10F2100012F77BE0700D12FCA0123D6990071AE412
:10F22000F0A3F090071812F78F700512F78C602684
:10F230009080A41228417A087B0090071EE0F91202
:10F240003E297404122A34E9600C7A087B00900786
:10F250001EE0F9123D037F010226BD74F612242E32
:10F2600074FA122AC8EAF8EBF97E0088828983A32F
:10F27000A3E0602B146034146031146034146025F2
:10F2800024F4603314700302F35B14700302F3552B
:10F2900014700302F36114700302F39D02F3EA1287
:10F2A000398B02F3EC12399102F3EC12399702F325
:10F2B000EC12399D02F3EC88828983A3A3E0FFE876
:10F2C0002403F850010988828983A3AA82AB83882A
:10F2D000828983E0606314605514602F1470668A1D
:10F2E000828B83A3A3E0F98A828B83E0FCA3E0FBFB
:10F2F000ECFA124831E960087403122CC7E4800765
:10F300007403122CC77401F0E080328A828B83E090
:10F31000F912389BEA4B600C124837851882851920
:10F3200083E480298518828519837401801F8A826D
:10F330008B83E0F9124825800312482BE985188257
:10F340008519838008851882851983740212FF5AF3
:10F35000EFFA02F3E31239AF02F3EC1239B502F31C
:10F36000EC88828983A3A3A3A3E0C0E07401122CDC
:10F37000C7D0E012F976A3A3A3A3E0C0E074021201
:10F380002CC7D0E0F07401122AA288828983A3A33B
:10F39000A3E0F91238CB12FF537A138046908118FC
:10F3A0007401122AAA740212296204122AA2888203
:10F3B0008983A3A3A3E0F91238C57401122CC7E016
:10F3C000C0E07404122CC7D0E0F07402122CC7E025
:10F3D000C0E07405122CC7D0E0F07404122AAA7B96
:10F3E000037A14796412396780020E0EEEF97406FE
:10F3F000122A347F020226BD74F212242E74FF12E8
:10F400002AC88A088B0912F4A0F50A7A067B001232
:10F410003D638A0C8B0DAE0CAF0DEE4F603F8E82BC
:10F420008F83A3741EF0A37407F0EEFCEFFDE508D4
:10F430002403FAE43509FB123979E9851882851924
:10F4400083F0700FEEFAEFFB123865E985188285BC
:10F450001983F0E06007EEFAEFFB123D69AC18ADDE
:10F46000197B01AA0A79641239677401122A347F60
:10F47000060226BD74F712242E74FF122AC812F455
:10F48000A0FE8A828B83A3A3A3E0F912386B12FF3C
:10F4900053EEFA79641239677401122A3402F25673
:10F4A000851882851983741012F98D2274EA12244A
:10F4B0002E74F2122AC88B0D851882851983740167
:10F4C00012F96FE0F5128A828B83A3A3E0F50FEAAD
:10F4D0002403F50C5002050D7402650F7071850C44
:10F4E00082850D83E0F8740A122CC7E812F75D7468
:10F4F00003687021850C08850D09750A00780812CB
:10F500002A1D7C087D007405122AA2123C9D7403FA
:10F51000122A34800912F91F122CC712F919E50CAE
:10F520002408F50C5002050DF582850D83E0C0E03E
:10F53000740B122CC7D0E012F75DE0FAA3E0F9EAF1
:10F54000F8740C122CC712F751503A050D8036741E
:10F550000A122CC77402F0850C82850D8312F91FE4
:10F56000122CC712F7515002050DF582850D83E06C
:10F57000C0E0740B122CC7D0E012F75D740C122C93
:10F58000C7E4F0A3F0850C82850D83E0F912389B67
:10F590008A108B11850C82850D83A385820C85834F
:10F5A0000D12F770F508E439F509E50C2402F50CA5
:10F5B0005002050DF582850D83E0C0E07401122C28
:10F5C000C7D0E012F767E0F50BA3E0F50AA3858248
:10F5D0000C85830D7402650F701A12F770FEE43902
:10F5E000FFEE2414F8E43FF9E50C2402F50C501664
:10F5F000050D8012E0FE7F00A385820C85830D241B
:10F600000AF8E43400F9E51045116011C3E894FBF1
:10F61000E99400500302F6F112F78C600B85188212
:10F62000851983740202F731EE2418FAE43FFB12C5
:10F630003D6390071AEAF0A3EBF012F78C8518826D
:10F640008519837005741002F731E4F090071AE011
:10F650002418FAA3E03400FB12FFB3EAF0A3EBF0A6
:10F660007402122A9A880C890D750E00780C122AE1
:10F670001D7C0C7D0012FF62123C9D7403122A3423
:10F6800012FFA7E510F0A3E511F012FF9BE508F0CB
:10F69000A3E509F012FF86EEF0A3EFF07401122C3F
:10F6A000C7E0C0E012FF922414F582E438F583D05D
:10F6B000E0F012FF7AE50BF090071AE0F8A312FFD2
:10F6C0006FE50A12F77B740FF09080A41228417A3C
:10F6D000087B0090071EE0F9123E297404122A34B8
:10F6E000E9604F7A087B0090071EE0F9123D038025
:10F6F00041780A122A257402122A9A8814891578E8
:10F7000014122A21780C122A218E0C8F0D780C12DB
:10F710002A217808122A21A90BAC10AD11740B1202
:10F720002AA21238897409122A34E98518828519A7
:10F7300083F074E055126420700DAC18AD197B0194
:10F74000AA0F7964123967740E122A347F0E0226CA
:10F75000BDE8F0A3E9F0E50C2402F50C2212F767EE
:10F7600085820C85830D22F0850C82850D83A32272
:10F77000E0FAA3E0F8E4C8F9EA2822F012FF9212B6
:10F78000F783222417F582E438F5832290071AE0E4
:10F79000F8A3E0F9E8492274EC12242E74F2122A3C
:10F7A000C8EAFEEBFF851882851983740112F912ED
:10F7B000A3E0F50EEE2403FE50010F7C0C7D0079D2
:10F7C000007402122AA2123CA9740A122CC77402F5
:10F7D000F08E828F8312F91F122CC712F919EE24B2
:10F7E00002FE50010F8E828F83E0C0E0740B122C5A
:10F7F000C7D0E012F912E0F9A3AE82AF8312389BB2
:10F800008A0A8B0B8E828F8312FE5BEE2402FE50DF
:10F81000010F8E828F83E0C0E07401122CC7D0E00C
:10F8200012F912E0F50FA3E0F512A3E0F513A3AE71
:10F8300082AF8325E0FAE433FB123D638A088B092B
:10F84000EA4509700302F8F27C00802412F773E4A1
:10F8500039FBEC25E0F8E433F9E50828F582E50901
:10F8600039F583EAF0A3EBF0EE2402FE50010F0C11
:10F87000ECC395138E828F83E0FAA340CFAE82AFA4
:10F8800083E50A450B700A85188285198374028006
:10F89000577808122A21E513F5107810122A25E569
:10F8A00012F5107810122A257405122A9A881089E8
:10F8B000117810122A218E108F117810122A218AA5
:10F8C000107511007810122A21780C122A21A90F24
:10F8D000AC0AAD0B740E122AA212388F740C122AC5
:10F8E00034E9851882851983F0AA08AB09123D69AD
:10F8F00080098518828519837410F0AC18AD197BC6
:10F9000001AA0E7964123967740E122A347F0C0230
:10F9100026BDF08E828F83A322E8F0A3E9F022E0D7
:10F92000FAA3E0F9EAF8740222C082C08374FD12DF
:10F930002AC812F97DC0E07401122CC7D0E012F978
:10F9400064C0E07402122CC7D0E0F0AC18AD197B93
:10F95000037A8079441239677403122A34D083D031
:10F96000820229E612F969E02212F96FA3A322F0BC
:10F970008A828B83A322F088828983A3228A828B46
:10F9800083A3E085188285198312F98D2212F96FFD
:10F99000A3E02274E912242E8A108B11EA2420128B
:10F9A000FC3112FE53E50A2414F508E4350BF50981
:10F9B000751681751200751300EA12FC4BE0F9EA26
:10F9C000241012FC3112FCA3124831E97017E51023
:10F9D000240E12FC31E06403600BC3E50894F1E5EA
:10F9E000099400400E751682E508240AF508E435EE
:10F9F00009F509C3E50894FBE50994004036E50ADA
:10FA00002409FAE4350BFB123D638A128B13EA4595
:10FA100013700302FC2CEA2409F8E43513F98A82F6
:10FA20008B83A3A312F919C3E508950AF508E50924
:10FA3000950BF509AA08AB09123D638A148B15EAE8
:10FA400045157010E51245136007AA12AB13123D5D
:10FA50006902FC2CAE14AF15E510240212FCB5248B
:10FA60000412FCA912FC9374826516705CE51024E4
:10FA70000E12FC3D12FC9388828983E0640370259A
:10FA8000E5102406F50CE43511F50D750E00780C23
:10FA9000122A1D7C087D00EEFAEFFB123C9D7403D8
:10FAA000122A34800E12FC3912FC8D12F97612FCE7
:10FAB0008DA3F0EE2408FE50010FE51012FC4B124E
:10FAC000FCC5241012FCA9800D12FC3912FC830E17
:10FAD00012FCBE12FC4B12FCC5241412FC7CAE823C
:10FAE000AF83E510241512FC3112FCC5241612FC5C
:10FAF0003112FCC5241912FC3112FCC5241AFAE497
:10FB00003511FB8A828B83780C122C7012FC5512F3
:10FB10002C70E50D8E828F8312FC5B122C7074109A
:10FB2000780C122A6912FC55122C707418780C1279
:10FB30002A698E828F83E50CF0A30EAF83748265F1
:10FB400016700EE4F0A3E50AF0A3E50BF0A30E8017
:10FB50000BE510241F12FC7CE50AF0A30E0EAF8308
:10FB6000E5124513700302FBEB12FE4185128285FC
:10FB7000138312F919900718E512F0A3E513F08525
:10FB80001282F583A3A3A3A3A3A3A3A3740FF0904E
:10FB900080A41228417A087B0090071EE0F9123EEB
:10FBA000297404122A34E9600C7A087B0090071E3D
:10FBB000E0F9123D03E510241A12FC31122CA48541
:10FBC0001282851383A3A3A3A3122CB012FC671285
:10FBD0002A1DAC0AAD0B851282851383A3A312FCE8
:10FBE000A3123C9D7403122A34801E12FC67122A51
:10FBF0001DAC0AAD0BEEFAEFFB123C9D7403122A0A
:10FC000034EE250AFEEF350BFFE510242412FCB577
:10FC1000242612FC3112FC88AC14AD15AB08AA16D0
:10FC20007944123967AA14AB15123D697F0F022679
:10FC3000BDF582E43511F58322E510240612FC415E
:10FC400022F8E43511F98882898322240FF582E4B1
:10FC50003511F583228E828F83E50CF0A30EAF83DE
:10FC60008A828B83780C22E5102422F582E43511F8
:10FC7000F583E0F50CA3E0F50D780C22F582E43570
:10FC800011F58312FC88A32212FC8DF022E08E82F3
:10FC90008F832212FC972212FC8DF0A30EAF8322D9
:10FCA00090071AE0FAA3E0FB2212FC4112FC9788AD
:10FCB000828983A32212FC4112FC88A3AE82AF8307
:10FCC00088828983A312FC97E5102274EB12242EFC
:10FCD0008A088B0990071812FE537A01751400E503
:10FCE000082403F50850020509F582850983E0F52B
:10FCF0000CE4F50DF50EF50FA3E0F510E4F511F5A4
:10FD000012F513740878101229C1780C7910122B8F
:10FD100092850882850983A3A3E0F510E4F51174A8
:10FD20001078101229C1780C7910122B9285088254
:10FD3000850983A3A3A3E0F510E4F51274187810E5
:10FD40001229C1780C7910122B9280078C828D8336
:10FD500012FE53E50A450B6059AC0AAD0B8C828D3F
:10FD600083A3A3A3A3780C122ADE70E0E508240481
:10FD7000F50850020509F58285098312FE5B8508A6
:10FD800082850983A3A3E0F514704512FE41EC6857
:10FD90007002ED698C828D83700512FE4A80071215
:10FDA000FE448C828D8312F919AA0AAB0B123D69AD
:10FDB0007A00EA850882850983F0A3E514F0AC088F
:10FDC000AD097B027A1279641239677F0D0226BD74
:10FDD0002402FAE43400FB123D638A0E8B0FAE0E50
:10FDE000AF0FEE4F70077A1075140080C58E828FAA
:10FDF00083E4F0A3E514F0850A82850B83A3A3E0D6
:10FE0000250CF508A3E0350DF509750A00780812F0
:10FE10002A1D851408AC087D00EE2402FAE43FFB9D
:10FE2000123C9D7403122A34EEFCEFFD740225147B
:10FE3000FB7A127964123967EEFAEFFB123D6980A2
:10FE40008A900718E0F8A3E0F922E0F8A3E0F9901F
:10FE5000071822E0F50AA3E0F50B22E0FAA3E0F888
:10FE6000E4C8F9EA28F50CE439F50D2274F51224FA
:10FE70002E74FF122AC88518828519837401F0EA4E
:10FE80002403FA50010B8A828B83E0FCA3E0F8E4A0
:10FE9000C8F9EC28FEE439FF8A828B83A3A3E0FC37
:10FEA000EA2403FA50010B12F78C700B8518828537
:10FEB0001983741002FF3FEC705E12FF6FE0F508CB
:10FEC0007808122A2590071AE02414F508A3E034D4
:10FED00000F5097808122A2112FFB312284512FFF3
:10FEE0008612284512FF9B12284512FF7AE0F9126C
:10FEF000FFA7E0FCA3E0FD12FF621238897409122B
:10FF00002A34E9851882851983F012FCA0123D6914
:10FF100090071AE4F0A380278A088B09750A0078F5
:10FF200008122A1D7D0012FFB3E02EFAA3E03FFB6A
:10FF3000123C9D7403122A34851882851983E412B9
:10FF4000FF5A7A1179641239677401122A347F03D7
:10FF50000226BDE9851882851983F0AC18AD197B9E
:10FF6000012290071AE02402FAA3E03400FB22E009
:10FF7000C82416F582E438F5832212FF922415F581
:10FF800082E438F5832212FF922412F582E438F5D8
:10FF9000832290071AE0F8A3E0C82212FF922410EF
:10FFA000F582E438F5832212FF92240EF582E438BC
:10FFB000F5832290071AE0F8A3E0F583888222C037
:10FFC00082C0831249218010C082C08312492780D9
:10FFD00007C082C083124957D083D0820229E6C06D
:10FFE00082C08312495D80F07409F5D575D49E7482
:10FFF00009F5D375D2A6D2B80229E6FFFFFFFFFFAD
:020000040001F9
:10000000C082C0831238D19004E074BFF0A3744A58
:10001000F09004E274B9F0A3744AF09004E474B36D
:10002000F0A3744AF09004E674ADF0A3744AF002B1
:10003000A4B674F712242EE9FE9004D2E4F0EE90F8
:1000400004D1F09015E512929612A9877C8F7D0954
:100050007AD57B0412479B9015E7E09004DDF09081
:1000600004DE747AF0A3740902B18874F412242EA9
:100070008A088B09EB5480700302813E9004D1E022
:10008000F9123CD98A0A8B0BAE0AAF0BEE4F700304
:1000900002813512B874E0F912A94E9004F012B43E
:1000A0009BA3A3A3A3A3A3A3A3E0640270378A82A4
:1000B0008B8312A96980078C828D8312AB94EC4DDF
:1000C00060208C828D83E06A7003A3E06B70E88C03
:1000D000828D83A3A3E06970DE9015ED12C5C3F095
:1000E000804C124A838E828F83E064017034EE2448
:1000F000181281A7122A2512AE66122841EE241288
:100100001281A7122A2512BEEC122A2112A40B1268
:100110002845EE241712BEF812387D740A122A34CC
:10012000800CE064027007EEFAEFFB123B17EEFA68
:10013000EFFB123CC7AA08E5096480FB80669009C2
:100140009AE0600464017019EAA2E050149004E897
:1001500012B1AB600612C8AC124AEEE50864018029
:100160003AEA5402600C90156B7401F0EA6402FAEA
:100170008032EA54086029124A898B0BEA450B70D9
:10018000169004F2E4F0A3F0A3F0A3F07A08FB9039
:1001900004D1E0F9123E35E5086408FAAB098004A1
:1001A0007A007B00028BCF12BDE0F50A780A227438
:1001B000F412242EEA4B9004E86026ECF0A3EDF054
:1001C0008A088B09E4F50AF50B7808122A197A01D6
:1001D0007B009004D1E0F9123E297404122A348085
:1001E0000FE4F0A3F07A01FB9004D1E0F9123E3560
:1001F000028BCF74F412242E8A088B098A828B8397
:1002000012C74D12BDBB38F583E02409FA7B0012FA
:100210003CC18A0A8B0BAE0AAF0BEE4F7003028211
:10022000B98E828F837402F0A3E412B007A3A3A354
:10023000A3E8F0A3E912A98BA3A3A3A3A3A3A3F00C
:10024000E5082403F8E43509129AAE12BDBB3AF56D
:100250008312B494F0EE2409FAE43FFB8E828F837C
:10026000A3A312A210F5838882E0A2E58E828F8379
:10027000A3A3A3A3A3500474018001E4F0E5082420
:1002800003F88882898312A969EA12C5A93BF5831C
:100290001282BE122A1DEA12BDBB3B12A4148E822A
:1002A0008F8312A967123C9D7403122A34EEFAEF71
:1002B000FB9004D1E0F9123CCD028BCFA3A3E0F573
:1002C00008A3E0F509750A0078082274F212242EBA
:1002D0008A088B09ECFAEDFB740E122CC7E0FC12B5
:1002E00039018A0C8B0DAE0CAF0DEE4F6031AC08AE
:1002F000AD091238EFE96027AC08AD09EEFAEFFB63
:100300001238F5E970158E828F83128324EEFAEF8E
:10031000FB1238E9AA08AB09123919790080027971
:10032000B4800EA3A3A3E0F508A3E0F50922122AE6
:10033000347F060226BD74EF12242E74F7122AC8E9
:100340008A0A8B0BECFEEDFF750DB3750C00751072
:10035000008002051090509EE493F8E510C3984089
:1003600003028445851008AA087B001239618A08B7
:100370008B09EA450960DC8A828B83A3A3A3A3A32C
:10038000E0250CF50CF50EC3E50A950EE50B94007F
:1003900050C17C157D007900EEFAEFFB123CA98577
:1003A0000882850983A3A3A3A3A3E0F8E50AC39564
:1003B0000C2825E0F8E433F9E50828F582E5093949
:1003C000F58312A9751232D7EAFCEBFDEEFAEFFBCA
:1003D00012479B850882850983A3E06401700A1295
:1003E000AE66740112AF39803DAC18AD1985088234
:1003F00085098312A967123949E960307408122C03
:10040000C7E0C0E012AE66D0E0F07408122CC7E07E
:100410006403700CAC18AD1912B48212479B800CA7
:1004200085188285198312AE7612A9878508828580
:1004300009831299CAA3A312AF41C0E012BABBD07C
:10044000E0F0750D00A90D7409122A347F09022607
:10045000BD74F712242EE9FE8A828B83A3A3A3A383
:10046000A3A3E0540860338A828B83A3A3A3A3A32E
:10047000A3E0540260218A828B83A3A3A3A3A3A336
:10048000A3A3A3E06406600F74E96E600A74CD6EE6
:10049000600574F06E7003124AA102ACD774E812C2
:1004A000242E74F8122AC87406122CC712C787ECBF
:1004B000FEEDFF89177515001286E412390D8A0AC0
:1004C0008B0BEA450B7003028696EE241012B66081
:1004D000A90A1230378A128B13EA45137003028679
:1004E00096EE2403F50CE43FF50DEE2406F508E442
:1004F0003FF5097C0085088212BE141239138A1058
:100500008B11850C82850D831286D91298B68512BF
:1005100082851383A3A3A3A31294B11286D9A3A3A4
:10052000A3A312B89E851282851383A3A3A3A3A3BA
:10053000A312CB9E12AF2D122A1D12BDBA3F12A4D8
:1005400014851282851383A312A961123C9D740342
:10055000122A347514007423122CC7E0F516742483
:10056000122CC7780C122C7002861B851082851104
:100570008312A96712394F850882850983A3EAF09F
:10058000A3EB1286F5A3A312AA3512898FA2E65017
:100590000F850882850983A3A3A3A3A3E0D2E1F07A
:1005A000E515706685088285098312C0F5900547B8
:1005B000E0687003A3E0697051850882850983A310
:1005C000A3A312B6657510007810122A25780C12B4
:1005D0002A19E516F5107810122A257426122CC750
:1005E00012284590055412284579007410122CC722
:1005F00012A96D122CE9740A122A34850882850921
:1006000083A3A3A3A3A3E04405F074012514FC1263
:1006100086E41239138A108B110514E51045116018
:1006200050851408C3E508950AE4950B5043E5147A
:1006300075F006A4F8A9F0E51228F8E51339F9E8F1
:10064000240CF508E439F509850882F583E412D80D
:1006500020E06401600302856B75150185088285C1
:10066000098374011286F512BB0DE8F0A3E9028537
:1006700082AA12AB1312303D7812122A21AD1674E1
:1006800024122CC7E0FCA917EEFAEFFB124AA7745C
:1006900002122A34803E8E828F83A3A3A3E0C0E09F
:1006A0007403122CC7D0E0F0EE241212BDD9C0E0C2
:1006B0007404122CC7D0E0F0E50A450B70097405EC
:1006C000122CC774B980077405122CC7741012A4B9
:1006D00034122CE37408028CFEE0851282851383A9
:1006E000A3A3A3228E828F8312BE228E828F83A326
:1006F000A3A3E0F92212D824A32274E812242E74B2
:10070000F2122AC8E9851882851983F08A0A8B0BB0
:100710008C168D177426122CC7129102AA0CFB128C
:10072000302BE9F514AA0CAB0D123031E9F515E5C3
:10073000147003028977751300800F8E828F83A354
:10074000A3A3A3A3E0D2E3F00513E50C12A942355D
:100750000DF583E0F8E513C398400302896EE514B4
:10076000700302896EE51375F006A4F8A9F0E50C94
:1007700028F8E50D39F9E8240CFEE439FF8E828F64
:1007800083A3A3A3A3A3E0A2E040BD750E0090093C
:100790009AE060046401704A8E828F83E070431295
:1007A000A968122EC98A088B09A808A909E8496016
:1007B0003188828983A3A3A3A3E06401600D8882AA
:1007C0008983A3A3A3A3E0640370178E828F83A3FE
:1007D000A3A3A3A3E0D2E7F0750E01E51570030211
:1007E0008748750F00750808750900E517600375DF
:1007F0000F207C087D0079007401122AA2123CA906
:100800008E828F83E0603C900597E064017018E56C
:100810000FD2E3F50F75091012C0F17401122CC745
:1008200012A0CD74FF803A430F0C75080C8E828F96
:1008300083A312898512A9837401122CC774FFF057
:10084000A3801E851882851983E06009E50FD2E632
:10085000F50F75080A12C0F17401122CC7E8F0A355
:10086000E9F07403122CC7E50F12BB40C0E0740519
:10087000122CC7D0E0F07406122CC77401F0122AB3
:10088000A2124A65740D122CC7E0600302894974F4
:1008900009122CC71298938E828F83A3A3A3A3F06F
:1008A0007409122CC71289981290F8E51612898FD4
:1008B0006011900597E0C0E07409122CC712910EE8
:1008C000D0E0F0850C82850D83A3A3A3E0C0E07483
:1008D00009122CC712BE44D0E012AC41C0E074092A
:1008E000122CC7129118D0E0F07409122CC712898B
:1008F0008512C76512BB4912A96912C746EAF0A35F
:10090000EB12BB2FC0E012C73ED0E0F07409122CEE
:10091000C7128AC712897C129CE53B12BB1C12BD10
:10092000B3128D127512007810122A1D12A40FEA4C
:1009300012A93B3BF58312A969123C9D7403122A4C
:10094000347401122AA2124A3B8E828F83A3A3A37E
:10095000A3A3E0D2E0F0740D122CC7E0600302877D
:100960003BE50EA2E05002151515140287487900E8
:10097000AA0CAB0D124A9B740E028CFEA3A3A3A378
:1009800012C0FAEA2212C0FA850A82850B8322126B
:1009900089932212C2EEE022129D0412AE6039F554
:1009A00083E508F0A3E509F02274F012242E74E91F
:1009B000122AC8EAFEEBFF89088E828F83A3A3A3C5
:1009C000A3A3A3A3A3E0F91230558A0C8B0DEA452B
:1009D0000D7003028AC2E50870157C048E828F8335
:1009E000A3A3A3A3A3A3A3A3E0F912305B804F7C2E
:1009F000088E828F83A3A3A3A3A3A3A3A3E0F912CA
:100A0000305B8A0A8B0BEA450B6033E508F5097801
:100A100009122A25850C82850D83A3A3A3A3A3A372
:100A2000A3E0FD8A828B83A3A3A3E0FC8A828B834D
:100A3000A3128AC7E0F91238777401122A3412A47B
:100A40000512B1A9607C8882898312A96574061297
:100A50002CC7128AD112A9697408122CC7128AD124
:100A6000A3A3E0C0E07410122CC7D0E0F0850C8284
:100A7000850D83A312A961740E122CC712C7877447
:100A800011122CC7E412898FFAA3E0CA241FF58241
:100A9000E43AF583129AB9E0C413135403FC7002CC
:100AA0007C0488828983E0F9780C122A2174205909
:100AB000FD744059F97402122AA2124AA774021254
:100AC0002A3474170296B212BE28850A82850B83D7
:100AD00022EAF0A3EB129E89A3A32274F712242E1C
:100AE00074FA122AC8E9FE7F018F087D0080047520
:100AF00008000D1293BCE0F8EDC3985027ED75F097
:100B000006A4F8A9F0EA28F8EB39F9E812BB3A395B
:100B1000F583E0A2E050D8540C60D4E0A2E250D2B9
:100B20007F0080CE8A828B83A3A3A3A3A3A3E070BC
:100B30003EE508A2E0400574016E70338A828B8323
:100B4000A3A3A3A3A3A3740112C607E0C0E0740388
:100B5000122CC7D0E012C5FFE0C0E07404122CC70D
:100B6000D0E0F07405122CC7EF12A434122CE374F9
:100B70000602ACD4C082C0837901124A9B02A4B69B
:100B800074F412242EEA4B602D900593E0640270F9
:100B90002590156BE4F08A088B09F50AF50B7808A7
:100BA000122A197A027B009004D1E0F9123E2974CE
:100BB00004122A34801290156B7401F07A027B00C3
:100BC0009004D1E0F9123E3580057402122A347F78
:100BD000040226BD74E812242E74FC122AC8740282
:100BE000122CC7E4F0A3F09004F012B76B851882C2
:100BF000851983E4F0A3F0751401900541E0A2E3A8
:100C00005003028C8B123E4D8A088B098C0A8D0B87
:100C10008A0C8B0D8C0E8D0F9004F2780C122A82A8
:100C2000128D067810790C122C2250077A017B0065
:100C3000028CFC850C14850D15850E16850F177812
:100C40001479101223BFA814A9159015EDE0C398CC
:100C5000E4995003E0F514128D06780C79101223F4
:100C6000BFE4F512F51378087910122B319004F2D5
:100C70007808122C61801412C0F69004F012A98733
:100C8000EEFAEFFB123D69AE08AF09EE4F60658EDC
:100C9000828F83A3A3A3E0F8E514C3985029EE2420
:100CA00003F582E43FF583A814E0C398F060217453
:100CB00002122CC712C2DA12B4B6EEF0A3EF12A6DB
:100CC000A7FEA3E0FF80C48E828F83A3A3A3E4F0DA
:100CD0008E828F83A312832385188285198312B194
:100CE000AB8E828F83A3A3A3A3608C12A2A2129ABD
:100CF000C2A380897402122CC712A9697404122A33
:100D0000347F100226BD9015EB128D12E4F512F51A
:100D10001322E0F510A3E0F5112274F212242E8ABA
:100D20000A8B0BE9FE7A007B009004F01283269078
:100D300004F012B1AB601E0A850882850983A3A363
:100D4000A3A312B1AB600E0AEA70010B88088909EF
:100D5000E8450970E39015EE12C0F6C3EA98EB99E6
:100D60004003028E057A067B00123D638A0C8B0DD0
:100D7000A80CA90DE8497003028E0588828983E5D5
:100D80000AF0A3E50BF0EE88828983A3A3F0901507
:100D9000ED129D30A3A3129E84E4F0A3F09004F022
:100DA00012B18C600B85088285098312A983801F8C
:100DB0009004F012A987900541E0A2E34011123E91
:100DC0004DEAF8EBF9ECFAEDFB9004F2122CB0903E
:100DD0000541E0A2E3502E7A087B009004D1E0F9AF
:100DE000123E3BEA4B4C4D701C9015EB12D25978D9
:100DF00008122A197A087B009004D1E0F9123E2FDC
:100E00007404122A3402833174F212242E74F31201
:100E10002AC8EAFEEBFF8E828F83A3A3A3A3A3A31A
:100E2000A3A3A3A3E0F50A90156BE0700579BA02BD
:100E300090EC750801750900750C00750D007C08B3
:100E40007D007900AA18AB19123CA97405122CC7B1
:100E50007401129124540460127402122CC7E0D25F
:100E6000E612912454087003750803E054106006DC
:100E700074404508F508E0540860227402122CC73B
:100E8000E044C01291245420600A7403122CC7E07D
:100E9000D2E080087403122CC7E0D2E1F08E828F7A
:100EA00083A3A3A3A3A3A3A3A3E070161232DD859B
:100EB000188285198312C7877402122CC7E0D2E208
:100EC000802C640F70107402122CC712912C7404C1
:100ED0004508F508807B8E828F83A3A3A3A3A3A3D9
:100EE000A3A3E064028E828F83700612A050F0806C
:100EF00060A3A3A3A3A3A3A3A3E06403700DAC18F2
:100F0000AD19EEFAEFFB124A4780468E828F83A31B
:100F1000A3A3A3A3A3A3A3E064017035900597E066
:100F200060107402122CC712912C750910750AFFFB
:100F300080187402122CC7E0440C12B4B674FDF091
:100F4000A374FFF074044508F5088E828F83129114
:100F500002EE241512BDD9A2E0503F7402122CC734
:100F6000E0540C701B8E828F8312A9691242F1E942
:100F7000700579BB0290EC7402122CC7E0D2E5F048
:100F8000EE241512BDD9A2E050107402122CC7E055
:100F9000540C64047004E0D2E5F0EE241112BDD9C3
:100FA000C0E07404122CC7D0E012A434124A657455
:100FB0000C122CC7E060030290E57408122CC712D3
:100FC0008998EE241812BDD9C0E01290F8D0E01232
:100FD000BB24E0C0E07408122CC712C75012BDD069
:100FE00038F583D0E012A05864017011900597E0A5
:100FF000C0E07408122CC712910ED0E0F0740812F1
:101000002CC712B4A52417FAE43FFB8A828B83E035
:10101000FCE8241CF582E439F583ECF0A3E412B17A
:10102000BBE0C0E0E82422F582E439F583D0E0F0AB
:101030007408122CC7129118E50AF07408122CC714
:10104000129D00129CE539F583E50CF0A3E50D1225
:10105000BE68FCA3E0FD12C770ECF0A3ED12954C46
:1010600012AB981290F13912C162C0E0E8242FF55A
:1010700082E439F583D0E0F0EE241B12BDD9C0E044
:101080007408122CC712C759D0E0F0EE241A12BD12
:10109000D9C0E07408122CC712C75012B65638F5E2
:1010A00083D0E012C78D1282BF122A1D12AE4C12DD
:1010B000AB98740B122CC712A02E123C9D74031215
:1010C0002A34EE241512BDD9544060129005001246
:1010D000B1AB600AAA18AB1912C8AC124AEEAA1832
:1010E000AB19124A3B740C122CC7E0F9740D028341
:1010F0002EE82428F582E422E82412F582E439F56A
:10110000832212910622E0F50CA3E0F50D2212C70E
:101110005412BAA538F5832212C7542423F582E469
:1011200038F58322F0EE241512BDE022E0D2E3125E
:10113000C2EE1291362212A2AAE8F0A3E9F02274BC
:10114000F712242E7E638A828B83E0600C7905126D
:101150002E09E9F87456C398FE90053FE0600CF93B
:10116000122E09E9F8EEC39824F2FEEEF902ACD78C
:1011700074F612242E74FE122AC8851882851983EB
:1011800012C787E9FEECFAEDFB90070A12B1AB60DB
:1011900035A818A919880889097808122A217D011B
:1011A000740E122CC7E0FCEEF990070A12A51F126C
:1011B0004AEE7402122A348B09EA45096004790068
:1011C000800679B2800279B60298BE74F712242E96
:1011D000E9FE9004E012B1AB601F7409122CC7E065
:1011E000F5087808122A25EEF99004E012A51F12DE
:1011F0004AEE7401122A34800279B602ACD774F731
:1012000012242E8908ECFEEDFF79B5E508245F6015
:101210000C14603114601224F86041804A9004D3A9
:1012200012BB01E8F0A3E9801990070C12B18C60A1
:101230003690070C12A51F124AEE8E828F83EAF0B9
:10124000A3EBF080209004E212C002601AEEFCEFE3
:10125000FD9004E212A51F124AEE800B9004DE12EC
:10126000A96D12479B790002ACD774F712242EE9BE
:1012700079B5245F600624F6600E80178C828D831A
:1012800012929612A98780099004DE12A96912476A
:101290009B790002ACD712C0FA9004D32274F212E8
:1012A000242E8A088B09ECFEEDFF750A0190054794
:1012B000E065087004A3E0650970101232D7EAFCFB
:1012C000EBFDEEFAEFFB12479B802A1232E38A0C09
:1012D0008B0DE508650C7004E509650D7009EEFAE3
:1012E000EFFB1232E9800EEEFCEFFDAA08AB09120B
:1012F0002E69E9F50AA90A02833174F512242EEA4F
:10130000FEEBFF8C088D09750A011232D7EAFCEB5F
:10131000FDEEFAEFFB124795E96401700B9005476B
:10132000129ACE12A987800EAC08AD09EEFAEFFB37
:10133000122E6FE9F50AA90A02CCF074F612242ED7
:10134000EAFEEBFF7A0C7B00123D63EA4B606AEE2B
:10135000242012BDD98A828B83F0EE24211293C4FB
:10136000F0EE24221293C4A3F0EE24231293C4A31C
:10137000A312B66B1293CD12A983EE1290F23FF531
:10138000831293CDA3A3A3A3A3A3E8F0A3E912B66A
:101390007A8A828B83A3A3A3A3A3A3A3A3F0EE249F
:1013A0002F12BDD9C0E01293BCD0E012AC4AF8A312
:1013B000E0F98A828B8312A97E0298C3EA12A946B9
:1013C0003BF5832212BDE08A828B83A32212C0FAEE
:1013D0008A828B832274F612242EECFEEDFF79B301
:1013E00090053EE0702A900570E064017022EE24C2
:1013F0001112BDD9F9122DF18A088B09A808A90983
:1014000012AE5412A987E84960047900800279A1DC
:101410000298C374F412242E74FE122AC8ECFEED56
:10142000FFEE241612BDD96405700DEE2406FCE40F
:101430003FFD124A4DE96074AC18AD1912BAC512DD
:1014400042F785188285198312B1AB605BE875F0AD
:1014500009A4F8AAF075F009E9A42AF9747628F825
:1014600074F639F9E8FAE9FB8A828B837808122C42
:10147000701296A47808122C32402985188285199A
:101480008312B4A512AE551294B17808122C709044
:1014900080E07808122BCB8A828B837808122C612B
:1014A0007900800A79A2800679A1800279C8028B2E
:1014B000CA129139EE1296A92274F412242E74FFE6
:1014C000122AC8EAFEEBFF90053EE0706C900570B2
:1014D000E06401706475083A7509007808122A21E1
:1014E0007402122A9A880889097808122A217C0134
:1014F0007D007A007B001234B77404122A34E9703C
:101500003512AFD67401129629C0E012AE4CD0E06D
:1015100012954C743A12B89E900508122CA412969B
:10152000A4122CB09080E07808122C7090050878F6
:1015300008122B7F800312953E7401028BCCEE249F
:101540000FF582E43FF583E4F0A3F022F0EE12AE53
:10155000592274F012242E74F6122AC8ECFEEDFF04
:101560007402122AAA124A4DE97003029624AC189A
:10157000AD197402122AA21242F7851882851983C6
:1015800012B1AB7003029624E875F009A4F8AAF032
:1015900075F009E9A42AF9747228F874F639F9E8A3
:1015A000FCE9FD12AFD6E4129629F8A3E0F912AED9
:1015B0005412A9878C828D83122CA41296A4122C0B
:1015C000B09080E07808122C708C828D837808129D
:1015D0002B7F8C828D837808122C709080A4780CDD
:1015E000122C707808790C1223BFE50C450D450EBE
:1015F000450F7030851882851983129D0075F0099A
:10160000A4F8AAF075F009E9A42AF9747A28F582F9
:1016100074F639F5837401F07A007B089007AAE02C
:10162000F9123D03740A0296B2F085188285198377
:10163000E02274F012242E8A088B09ECFEEDFF12D2
:10164000953E908110780C122C701296A4780C1292
:101650002ADE604CEE240E12BDD964017005124AD8
:1016600035803FE07015124A2FE960368E828F83F5
:10167000A3A312A45A5403700C802764027013129F
:101680004A2FE9601DEEFCEFFDAA08AB0912432DBD
:101690008010E064037005124A2F800679A1800251
:1016A00079A38011EE1296A9222412F582E43FF567
:1016B0008322122A347F080226BD74F612242EEAF1
:1016C000FEEBFFEE240AF508E43FF509850882F5F4
:1016D0008312AB98EC12AE603DF583E4F012AC38A7
:1016E000124A23850882850983E02406FCA3E0349E
:1016F00000FD8E828F8312A969124A4D850882856A
:10170000098312B1A07054129898124795E9701D80
:101710001232D78A088B09AC08AD099004DE12A9F1
:1017200069124795E97006122CD7E9602E8E828FD8
:101730008312AB8E8E828F8312A969124333E960C4
:10174000158E828F83A3A3A3A3A3A3A312C74D12B5
:10175000B8A3E4F0A3F0129AEFE4F012B192701A79
:1017600012977D12A969124A298508828509831278
:10177000B1A0700612AFC874A1F00298C3EE240A9B
:1017800012984D8882F5832274F612242EEAFEEB1D
:10179000FFEE240A12984D7A187B00123D638508EB
:1017A00082850983EAF0A3EB1298B6E84970030238
:1017B0009847EEFAEFFB1249ED12B192607212985F
:1017C0008564018E828F83A3A3A3A3A3A3700712B2
:1017D0009877740E802012B1AB700F129898124750
:1017E00095E97006122CD7E9600712986D740D8088
:1017F0000512986D740512AC4A5403640170071207
:1018000098567405800B90053FE0C0E0129856D0C2
:10181000E012A421F812C8ABA3E0F9122E09850842
:101820008285098312C75012BADB38F583E9801A22
:1018300085088285098312A969123D698508828518
:101840000983E4F0A3800312A66EF08076F8E43FEB
:10185000F988088909228E828F83A3A3A3A3A3A357
:10186000A3A312986622A3A3129F93A3228E828F12
:1018700083A3A3A3A3A3A3A3A3A3A312C75412A6A2
:101880005F38F583228E828F83A3A3A3A3A3A3A390
:10189000A3A3A3129B01E0229004DE12AB9C8E82D4
:1018A0008F83A3A3A3A3A3A3A3A3A3A3E02406FAC4
:1018B000A3E03400FB2212A425F8A3E0F92274026D
:1018C000122A347F020226BD74F112242E8A0A8B5A
:1018D0000B8C088D097A187B00123D638A0C8B0DE6
:1018E000AE0CAF0DEE4F70030299C28E828F8374DF
:1018F00001F0E508240DF8E43509F988828983E0D0
:10190000FAC3E49AFA95E0FBE50812C5A935091275
:1019100099CEFB8E828F83A3A3A3A312C6338E829C
:101920008F83A3A3F0EEFAEFFB122DB58508828515
:10193000098312C5CC70098E828F83A3740580063B
:1019400090053F1299CAF0EE2417F8E43FF9880C8D
:10195000890D8E828F83A3E0F9122E09E9850C820E
:10196000850D83F0EE2416F8E43FF9E508240EFA1D
:10197000E43509FB8882898312A67CE5082410FAE5
:10198000E43509FB850C82850D83E0FC8882898320
:10199000E0F88A828B83E0C398C39C12C2E3F0EE26
:1019A000FCEFFDAA0AAB0B1249F3E9F508700AEE49
:1019B000FAEFFB122DC1E9F508EEFAEFFB123D69D3
:1019C0008003750810A90802AF5C12A99222F58362
:1019D000E02AFAA3E03B2279010229E674F41224FA
:1019E0002EEAFEEBFF8E828F83A3A3A3A3A3A3A360
:1019F000A312BE0AF58312C5CC702A1298857025F1
:101A0000129ADCE06405701D129ADCA3E0F8740100
:101A10006860057406687007129AEF7402800512F8
:101A20009AEF7403F012977D12A51FE4F0EE2408DC
:101A3000129AAB242DF582E43AF583E0C0E08508E4
:101A400082850983129AB9A3A3D0E012C637FAA3FC
:101A5000E0CA242AF582E43AF583E0C0E0850882F2
:101A6000850983129AC2D0E012C637F8A3E0C812E3
:101A7000A94238F583129ACE129AB912A98312326A
:101A8000D78A0A8B0BAC0AAD0B850882850983E0E7
:101A9000240612A29112479B85088285098312A908
:101AA00069122DC112A718F0028BCFF8E43FF98814
:101AB000828983E0FAA3E0CA22E0FAA3E0F5838AF0
:101AC0008222E0FAA3E0F5838A82A3A3A322129ADA
:101AD000D22212C0FE850882850983228E828F83DE
:101AE000A3A3A3A3A3A3A3A312A035129F8F228E07
:101AF000828F83A3A3A3A3A3A3A3A3A3A3129B0146
:101B00002212A21BC8240EF582E438F58322EA12C1
:101B1000C5A33BF583220299D7C082C0839004F607
:101B200074E7F0A37449F09004F874DBF0A37449EF
:101B3000F09004FA74D5F0A37449F09004FC74E1B9
:101B4000F0A37449F002A4B674F412242EEAFEEB5A
:101B5000FF129B9EF5081232DD8A0A8B0BA80AA998
:101B60000B8E828F83129AB9E0687003A3E06960DC
:101B70002AE508A2E550248E828F83A3E0FB90041F
:101B8000F612A51F124AEE8E828F8312C750240AC6
:101B900012B1A57006129B9EC2E5F0028BCF8E8219
:101BA0008F83129868A3E02274F412242EEA24088A
:101BB000FCE43BFD8C828D83129D0012A665E0FE45
:101BC00074035EF50912A9413912B4A3888289838E
:101BD000F0A3A882A983E50960097402650960037E
:101BE000029C73740C5EF508601774086508601138
:101BF000740465087013740265097005EEA2E44070
:101C00002A129D092423129D36740C650870161241
:101C10009CF22424129D1BFCA3E0CC129CE53CF515
:101C200083A3129D3C740265097005EEA2E4404353
:101C3000129CF22426129D1BFFA3E0CF12B65CA3D8
:101C4000129D3C129CF62428129D4B1290F23CF5FA
:101C500083A3129D3CE508601274086508600C744B
:101C60000C65086006740465087008129D0924223A
:101C7000129D36129D09129CD97005EEA2E1500CFE
:101C8000129D0912B6563C129CEB800E9004D212A3
:101C90009CED9004D2E00412A220A3A882A983EEB6
:101CA000A2E75032129CF22421129D4B129CD96063
:101CB00025129D092430129D36EEA2E150188A8229
:101CC0008B83A3A3A3A3A3A3A3A3129AB32431F545
:101CD00082E43A129CEB028BCF2421F582E43CF59E
:101CE00083E05403222424F582E422F583129D30FC
:101CF000F022EA2408FC8C828D83E0FFA3E0CF224F
:101D0000129D042212C0FEE8228A828B83A3A3A321
:101D1000A3A3A3A3A3E0FCA3E0CC22F582E43FF5B8
:101D200083129D30F0A3A882A9838C828D83E02248
:101D3000E08882898322F582E43CF583129D40226B
:101D4000E088828983F0A308A98322F582E43FF525
:101D500083129D408C828D83E0FCA3E0CC22C08264
:101D6000C0838A828B83129BA2F8740358F98A82FB
:101D70008B83A3A37401F0E9600574026970617438
:101D80000C58FC601474086C600F74046C7013744D
:101D900002697005E8A2E4401D8A828B83A3A374C4
:101DA00002F0740C6C700A8A828B83A3A3E0240275
:101DB000F07402697005E8A2E440258A828B83A34F
:101DC000A3E02404F0EC600F74086C600A740C6CDF
:101DD000600574046C70098A828B83A3A3E004F00D
:101DE000E8A2E750318A828B83A3A3E00412C16882
:101DF000F9A3E0F5838982A3A3A3E0540360178AC3
:101E0000828B83A3A3E004F0E8A2E150098A828BCD
:101E100083A3A3E004F08A828B83A3A3E004F002EF
:101E2000A4B6C082C0838A828B83A3A3A3A3A3A3E7
:101E3000A3A3A3A312B1AB600C8A828B83A3A312CA
:101E4000A961123D6902A4B674F712242EEAFEEBD2
:101E5000FF8E828F8312AE6EA3A3A3A3A3A3A3A31B
:101E6000E4F0129E84A3A3A3A3A3A3F0A3F0E8121B
:101E7000C5A339F583E4F01249BDEEFAEFFB124930
:101E8000C902ACD7A3129E892212A220A3A3A3A3A6
:101E90002274F112242E74F3122AC8EAFEEBFF74A6
:101EA0000C122CC77401F01249C38E828F83A3A336
:101EB000A3A3A3A3A3A3A3A312B1AB600612A51867
:101EC000124AEE12BDD66003029F597C087D00794C
:101ED00000AA18AB19123CA97402122CC774011283
:101EE0009F8812A05012A058F8A3E0C812C58D38E0
:101EF000F583E02409C0E07404122CC7D0E0F0742C
:101F000005122CC712A432124A65740C122CC7E0B9
:101F100070477408122CC712AA40740E129F8812C0
:101F2000AB968508828983A3AA82AB8312479B1252
:101F3000A95D1293BC12BE54122A1D12C58712A4A9
:101F400014E5082409FAE43509FB123C9D740312D8
:101F50002A34AA18AB19124A3B8E828F83A3A3A3FB
:101F6000A3A3A3A3A312B1AB600612A95D123D699E
:101F7000EEFAEFFB1249B7740C122CC7E0C0E01266
:101F8000AFC8D0E0F002AF5712B1B5129F8F221246
:101F90009F932212A21BF58388822274F512242EAD
:101FA00074F3122AC8EAFEEBFF7C087D007900AAD0
:101FB00018AB19123CA912A04612A6A7C0E07404DF
:101FC000122CC7D0E0F07402122CC7740112A05872
:101FD000C0E07405122CC7D0E012A69B6401700902
:101FE0007402122CC7E0D2E5F0AA18AB19124A65A8
:101FF000740C122CC7E0702C8E828F831282BC125C
:102000002A1D8E828F83A3A3A3A312A416740B127E
:102010002CC712A02E123C9D7403122A34AA18ABAE
:1020200019124A3B740C122CC7E0F902CCEB12A037
:102030003512BE282212A0392212A21BC8242BF569
:1020400082E438F583228E828F83A3A3A3A3A3A364
:1020500012A2A6E8F0A3E92212B687A3E02274F741
:1020600012242E74FE122AC8ECFEEDFF7508C8ACCF
:1020700018AD19124A47E96401704B851882851919
:102080008312A41BA3A3A3A312A0CDA3A3E4F09047
:102090000997E060198E828F8312A52970108E82B5
:1020A0008F83A3A3A3A3A3A3A3A37401800D8E82F4
:1020B0008F83A3A3A3A3A3A3A3A3E4F0EEFAEFFB50
:1020C0001249A5E9F508A908740202ACD4129139A5
:1020D0008E828F83A3A3A32274F612242E74F4128B
:1020E0002AC8EAFEEBFF12A04612A202129ABAA375
:1020F000E0FA7402122CC7EA12C63712A31E740447
:10210000122CC712AACE6A701312A1F6E012A28F87
:102110007406122CC712C633241A80377402122C8C
:10212000C7E064016005E064067039EE2402129A8B
:10213000AB12BAF13AF583E0C0E07403122CC7D0B9
:10214000E012C637241312A2917406122CC712C6CD
:1021500033241BF8A3E03400F97408122CC7E8F00C
:10216000A3E980297406122CC7E4F0A312A202127C
:10217000A28F7408122CC712A210C8241AF582E488
:1021800038F583E0C0E0740A122CC7D0E0F0740682
:10219000122CC712B1AB602B7406122CC712A9699E
:1021A000122E5DE96401701B1232D78A088B09ACCC
:1021B00008AD097406122CC712A969124795E96483
:1021C000017009AA18AB19122CEF802590099AE02A
:1021D00060046401701BAA18AB191242FDE9640186
:1021E000700FEEFCEFFD7406122CC712A96912499C
:1021F0009F740C0298C0EE2402F8E43FF9888289AB
:102200008322F0EE2402F8E43FF988828983E022F9
:10221000EAF0A3EB12A22012A21B22E0F8A3E02214
:10222000F08882898322C082C08374F9122AC8127E
:10223000A29812A987EA2402F8E43BF988828983EC
:10224000E0240112A2917402122CC712A210F98884
:10225000828983A3A3A3A3A3A3A3A3A3E0FC88824F
:102260008983A3A3A3A3A3A3A3A3A3A3E0FBECFA43
:102270007404122CC712A69412A674C0E07406123D
:102280002CC7D0E012A434122CF5740702A4B32496
:1022900012FAA3E03400FB228A828B83A3A3A3A3B8
:1022A000A3A312A2A62212A2AA2212A21BF9851887
:1022B0008285198322C082C08374FC122AC812A2AC
:1022C0009812A9878A828B83A3A3E02401F8A3E054
:1022D0003400F97402122CC7E8F0A3E912A43412F6
:1022E0002CFB740402A4B3C082C08374FB122AC8FE
:1022F00012A347F87402122CC7E8F0740268701237
:102300008A828B83A3A3E012A31E7403122CC7122C
:10231000A987AA18AB19122D01740502A4B32402CF
:10232000F8A3E03400F922C082C08374FD122AC8E9
:1023300012A347C0E07402122CC7D0E012A43412DA
:102340002D07740302A4B38A828B83A3A3A3A3A340
:10235000A31291368A828B83129866E02274F4125B
:10236000242E74FB122AC8EAFEEBFF8E828F83A311
:10237000A312AE6EE5822409F508E43583F50974ED
:1023800003122AAAA3AA82AB83124A47E964017006
:102390006F851882851983743212A6A724F7C0E0CE
:1023A0007401122CC7D0E0F07402122CC7E412A4FE
:1023B00034122F478A0A8B0BAE0AAF0BEE4F6040E8
:1023C0007403122CC712A41BE8F0A3E912A421C0C5
:1023D000E0EE2420F582E43FF583D0E0F0750A00BA
:1023E0007808122A1D12A40512A41412A40B12A913
:1023F00069123C9D7403122A34EEFAEFFB122F414E
:102400007405028BCCEE12C58D3F2212AE7D2212D6
:10241000C5BB350BF583E0FC7D002212BB05A3A3F1
:102420002212A4252212A42922F08508828509837C
:10243000E0227401F0AA18AB1922C082C0838A82FC
:102440008B8312A45A24FA600624FE6007800812C7
:102450004993800312498702A4B612A4AC22C08219
:10246000C08312A4A2600E24FE600F24FE6010241C
:10247000FB60118012124999800D12498D8008125B
:102480004981800312497B802DC082C08312A4A29F
:10249000600624FC60078008124999800312498174
:1024A000801412A4A824FB228A828B83A3A3129FE8
:1024B00093E022122A34D083D0820229E6C082C05F
:1024C000839015F0E07025900999E0701F8A828B47
:1024D00083A3A3A3A3A3E0701312A52360388A8269
:1024E0008B83A3A312C8ABE06407602A8A828B8324
:1024F000A3A3A3A3A3A3A3A3E070128A828B831236
:10250000A52960097A347B0112437B80099004FE7F
:1025100012A51F124AEE809EEEFAEFFB9004F8120D
:102520009F8F2212A4A864062212A4AC6405227410
:10253000F612242E74FA122AC8EAFEEBFF74031274
:102540002CC712BAAB7403122AA21249B112BDD61B
:10255000600302A65A8518828519837432F07405C7
:10256000122CC712CB91C0E07401122CC7D0E0121C
:10257000A69BC0E07402122CC7D0E012A6A1F8A35B
:10258000E0F9E849601BE812BADB39F583E0FAE8C4
:1025900012A65F39F583E02AF87401122CC7E028EF
:1025A000F0AA18AB19122F478A088B09A808A909A5
:1025B000E849700302A64F8E828F8312A969888230
:1025C0008983A3A312A69412BAF13912AC46C0E0D3
:1025D000E812A665D0E012AC41C0E0E82421F58203
:1025E000E439F583D0E012A6A7C0E0E8242AF582FA
:1025F000E439F583D0E0F07405122CC7E0FCE81252
:10260000A6742C12A291E812A93B39F58312A69464
:10261000242DF582E439F583EC12A6A1FAA3E0FBA0
:10262000EA4B6019E8242BFAE439FB8E828F83A3EE
:10263000A3129D0D12A65F3CF58312A67C8E828F9D
:1026400083A3A3A3A3A3A3A3A3E8F0A3E9800AEE13
:10265000FAEFFB1249B712A66EF074060298C02476
:1026600016F582E4222420F582E439F5832212AFA4
:10267000CC74102212A94639F583E022E0FC8A824C
:102680008B83E02CFCA3E03400FD8A828B83ECF08A
:10269000A3EDF022EAF0A3EBF0E82212A6ACA3E04F
:1026A0002212B1BFA3E02212A6ACE02212A6B022F1
:1026B00012A6B422F08E828F83A3A3A3A32274F662
:1026C00012242EEAFEEBFF12BDD670421249C38ED1
:1026D000828F83A3A3A3A3A3A3A3A3A3A312B1AB9A
:1026E000600612A518124AEE12BDD6700B12A95D33
:1026F000122F4112A7188015EE240812978012A9F4
:1027000069123D69850882850983E4F0A3F0EEFA39
:10271000EFFB1249B70298C312AFCCE92274F6124C
:10272000242EEAFEEBFF8C088D091242F1E97004B9
:1027300079018011AC08AD09EEFAEFFB9004FC12B0
:10274000A51F124AEE0298C374F112242E74F312DC
:102750002AC88A088B09740C122CC712ABB1123C20
:10276000A9850882850983A3A3E06404600302A805
:10277000157404122CC77422F0740C122CC7E0607C
:102780000302A93185088285098312A2A212A987B2
:102790007402122CC7740112AE98C0E07405122C9A
:1027A000C7D0E012AF51F8A3E0F97406122CC7129B
:1027B000AFE9A3A3A3A3A3A3A3E0640170097402D8
:1027C000122CC7E0D2E5F0AA18AB19124A65740CB6
:1027D000122CC7E0600302A9317408122CC712C77B
:1027E0005012A93B38F58312B76B8E828F83740524
:1027F00012A98B12AFFFE849606E850882850983B4
:1028000012BE50122A1D7C1012A94C123C9D74035A
:10281000122A34805F850882850983A3A3E06401BE
:10282000600D850882850983A3A3E06406700A749D
:1028300004122CC7742302A778850882850983A314
:10284000A3E06402600D850882850983A3A3E06488
